:020000040800F2
:1000000000800020C1660008B97300089D660008E2
:10001000BB730008BD730008BF7300080000000038
:1000200000000000000000000000000021C30008E4
:10003000C173000800000000B1C30008F5C3000848
:10004000C3730008C5730008C7730008C9730008AC
:10005000CB730008CD7300084D730008537300087C
:10006000597300085F73000865730008CF730008B8
:10007000D1730008D3730008D5730008D773000844
:10008000D9730008DB730008DD730008DF73000814
:10009000E1730008E3730008E57300086B73000860
:1000A000E7730008E9730008EB730008ED730008BC
:1000B000EF7300084D7A0008F1730008F37300082D
:1000C000F5730008F7730008F9730008FB73000864
:1000D000FD730008F57A0008397F0008FF730008F7
:1000E0008F73000835740008017400080374000859
:1000F000057400080000000000000000000000007F
:1001000000000000000000005FF808F110B5054C89
:10011000237833B9044B13B10448AFF300800123B3
:10012000237010BD100600200000000000F201083E
:1001300008B5034B1BB103490348AFF3008008BD6A
:10014000000000001406002000F2010870470000C3
:100150008168014809F09CBF40B1010838B50446E8
:1001600081680D4809F094FF20690C4D0368002157
:100170001B68984701222846032106F05FFF20698B
:10018000002103685B6898472846BDE83840012293
:10019000022106F053BF00BF4FB10108000002402A
:1001A0000B4B13B51A68B2F5007F04D21A68511CC4
:1001B0001960084B9854084B1C680DF0FFFB002396
:1001C00002460721204600930EF0D8FA02B010BD77
:1001D0002C0800202C0600203008002010B5044612
:1001E0003C2115F03BFF204610BD000070B5154CBA
:1001F0002368092B1FD92268134E023A314613484F
:1002000015F060FE05462068023830440AF03DF8DB
:100210008542014610D10E4D28680CF099FF00234D
:100220003146226828680CF0DFFF10B9094809F050
:100230002FFF0023236070BD2A46074809F028FFDE
:10024000F7E700BF2C0800202C0600200400002047
:100250003408002069B101087DB1010870B5044679
:100260002048214E60602148C4E90312A060204864
:10027000194686B02060636104F1180004F1280576
:1002800005F0D4FF0FCE0FC5336801222B6000218B
:100290004FF400700CF01AFF164B186018B94A2181
:1002A000154806F069F9154B0A21009300231448FC
:1002B0001A460EF041FA134B41F221011860012356
:1002C000CDE900334FF6FF7303A81A4615F0AAFDD7
:1002D0000D4A03AB03CB106020461B88516013818D
:1002E00006B070BD9BB10108ECB10108A5B10108D1
:1002F00008B20108340800208AE50108ED01000871
:10030000ABB101083008002004000020014800685B
:100310000CF0FABF3408002010B50446C068074945
:1003200003685B699847E06804F1280103681B686B
:1003300098470022024B1A6010BD00BFA1010008BF
:100340002C080020C06810B50368084C5B6898470B
:1003500001220221204606F071FE012203212046DF
:1003600006F06CFE0022024B1A6010BD0000024035
:100370002C08002081F001021830082106F018B87E
:1003800081F001021830022106F012B881F001025A
:100390001830042106F00CB881F001021830012158
:1003A00006F006B810B5044681680F4809F070FEE3
:1003B00004F1180005F0EAFF002184F8240020462B
:1003C000FFF7E4FF20460021FFF7DAFF2046002177
:1003D000FFF7D0FF20460121FFF7DEFF2046BDE8F2
:1003E00010400021FFF7D8BFB5B1010810B5044691
:1003F00081681A4809F04CFEA168194809F048FEC6
:1004000020460121FFF7C8FF01212046FFF7B8FF72
:100410004FF496700DF024FC20460021FFF7B0FF4A
:1004200001212046FFF7B2FF4FF496700DF018FC43
:1004300020460021FFF7AAFF01212046FFF79AFF7F
:100440004FF496700DF00CFC20460021FFF792FF50
:100450002046BDE810400021FFF79EBFBFB1010854
:10046000CFB1010807F054BE10B50446406C10B17E
:10047000042115F0F3FD204610BD10B504460068B8
:1004800010B1012115F0EAFD204610BD2DE9F04123
:100490000025069FC0E90112C0E903353946C0E9CD
:1004A0000555C0E90755057045620446164600F13A
:1004B0001C0813F04BFD38B93146074809F0E8FD38
:1004C0002021064806F058F83A464146204613F0E7
:1004D00009FD2046BDE8F08120B201088AE5010847
:1004E00030B58DB014F00CFF044603F0B9F9214685
:1004F00003F0B0FC2E4B2F4A0321009302A82E4B91
:10050000FFF7C4FF02A9204614F09CFD09A8FFF7DD
:10051000B4FF06A8FFF7B1FF284B294A0321009337
:1005200002A8284BFFF7B2FF02A9204614F08AFD6B
:1005300009A8FFF7A2FF06A8FFF79FFF02220023EA
:10054000214D0392214A012102A8CDE90523CDE9DD
:100550000733CDE909338DF8083004950B9313F078
:1005600077FB38B929461A4809F092FD202119482D
:1005700006F002F8012209A902A813F053FB02A910
:10058000204614F05FFD09A8FFF777FF06A8FFF7E4
:1005900074FF2046104B114A114914F021FE00F05F
:1005A00089FA052221460DB0BDE8304003F066BC53
:1005B00075B2010883B201084BB20108E9B2010823
:1005C000E0B201088CB2010813B3010821B301089D
:1005D00020B201088AE501086504000844B3010857
:1005E00068B301082DE9F74FD0E9008AAAEB0804A7
:1005F000A410B4F5705F07460E469346894602D1B3
:10060000224815F0EFFC012C234638BF0123E418E3
:10061000A1EB08031ED204B3B4F5705F28BF4FF4FA
:100620007054A000019309F0CFFD0546019BDBF853
:100630000020EA5043462A1F9E4210D1331DA3EBEF
:1006400008032B441A46D1450ED059F8041B42F832
:10065000041BF8E74FF47054E3E72546E7E753F847
:10066000041B42F8041FE7E7A9EB06061E44B8F195
:10067000000F03D00421404615F0F0FC05EB840484
:10068000C7E90056BC6003B0BDE8F08F6EB3010847
:100690002DE9F04391B014F033FE584F06463D6803
:1006A000574C15F001051AD120461A22294640F868
:1006B000045B18F04FF81A22294604F12400256241
:1006C00018F048F8012320464E4A4F49C4E9105516
:1006D000C4E91255A4F850503B6016F0F1FA94F8B2
:1006E00051301BB11D21494805F046FF0027484DF8
:1006F00030468DF81F7014F097F8304605F080FBF7
:100700002B1F304643490DF11F02009514F02AFBC0
:10071000414808AA05F120012062089709F0A2FAD1
:10072000089B1BB18521394805F026FF30463B491F
:1007300014F0BFFA05463A4FDFF8E880DFF8E8909A
:100740002064ADB10EAB03930DAB02930CAB0193E0
:100750000BAB0093394628460AAB09AA18F08CFF68
:1007600006281FD0314809F093FC01238DF81F3073
:10077000012302223046CDE900322D492D4B0DF1E7
:100780001F0214F0AFFA9DF81F302BB12A4809F070
:100790007FFC102007F0B7FC012384F8513011B022
:1007A000BDE8F0830D2017F07FFF0F9008B92348B4
:1007B000D9E70E9B0D2104930D9B424603930C9B9E
:1007C00002930B9B01930A9B0093099B18F000FF77
:1007D000D4E9121399420BD00F9B41F8043BA1645A
:1007E0002C21284618F0B7FF0028C1D0451CA8E7E7
:1007F00048460FAAFFF7F6FEF2E700BF38080020D0
:100800003C08002000000020690400088AE5010877
:100810004008002083B2010888B30108E0B2010853
:1008200094B301080AB4010880080020A6B30108A7
:1008300013B301088C08002023B40108F6B30108A3
:1008400010B9034809F024BC03C809F087BC00BFF5
:1008500036B4010810B9264809F01ABC017840687E
:1008600001F07002502A01F00F0328D006D8A2B17F
:10087000402A0AD002681F4809F00ABC602AF9D150
:10088000012B0CD101781C4805E01C491C4B0028A9
:1008900008BF19461B4809F0FBBBFFF7D1BF022B6D
:1008A00002D101881848F6E7042B02D101881748C5
:1008B000F1E7082B01680CBF15481648EBE7012B40
:1008C00003D190F900101448E5E7022B03D1B0F9E9
:1008D00000101248DFE7042B03D1B0F900101048D4
:1008E000D9E7082B01680CBF0E480F48D3E700BFBB
:1008F00046B40108C7B401084CB401083BB4010870
:1009000040B401081CB5010858B4010865B40108D9
:1009100072B4010880B401088CB4010897B40108CE
:10092000A3B40108AFB40108BCB4010870B500203D
:10093000002105F03FFA04460F4D104EC4B1617915
:10094000802911D122792168306813F017FF2046E1
:1009500005F068FB2046082115F080FB00200021EF
:1009600005F028FA0446E9E7284609F091FBEEE78E
:10097000034B187870BD00BFE3B40108000D0020E0
:10098000B80D002008B502F06BFFBDE8084002F08A
:10099000AFBF1FB56123CDE9013101A9039204F076
:1009A0002DF905B05DF804FB07B58DF8041001A919
:1009B0008DF805208DF8063004F0CCF903B05DF811
:1009C00004FB000070B5114E346814F001041BD113
:1009D0000F4D1A222846214640F8044B17F0BAFE64
:1009E0001A22214605F124002C6217F0B3FE0123E0
:1009F0002846084A0849C5E91044C5E91244A5F843
:100A00005040336016F05CF9014870BD3808002092
:100A10003C080020000000206904000808B5FFF72A
:100A2000D1FF90F851301BB93321034805F0A4FDE4
:100A3000FFF7C8FF08BD00BF8AE5010870B5154C77
:100A4000154809F025FB2368DB0708D414F072FC75
:100A500080220146114813F0BBFB012323600F4A9B
:100A60000F4B104D1A600CF0A3FF0F4B18600F488E
:100A700009F00EFBFFF7D2FFD0E91146A64205D0E0
:100A8000284654F8041B09F003FBF7E7084B1878D5
:100A900070BD00BF94080020F9B40108E40B0020E9
:100AA000000D00201AB50108A00B00200CB50108AC
:100AB000BC0D002002F0D4BE10B50C4C02F0D0FEEC
:100AC0002368DB070FD400F1580300F1440200F162
:100AD00048010748FFF7C2FB0123064A06490448BC
:100AE000236016F0EDF8024810BD00BF900800200A
:100AF000A80B0020000000204D0100082DE9F04760
:100B0000FFF7DAFF04460121FFF746FC2046FFF716
:100B100003FC0CF04DFF4EF65F283A4F4FF4407245
:100B20003B683949C01A40454FF47A732046374D27
:100B30003FD8FFF7EBFBDFF8D8A0DFF8CC902860B8
:100B40002E68EEB90CF034FF3B68C01A404517D848
:100B5000504609F09DFA01212046FFF711FCC820FC
:100B60000DF07EF831462046FFF70AFC4FF47A7309
:100B70004FF4407249462046FFF7C8FB2860DFE784
:100B80002046FFF7DFFB2B68002B39D001212046E0
:100B9000FFF7FCFB1F4809F07BFA41F288300DF0AB
:100BA0005FF800212046FFF7F1FB1B4B1878BDE8EA
:100BB000F087FFF7ABFB0526DFF85490DFF848809D
:100BC00028602F68002FE1D1013E16F0FF0617D0F4
:100BD000484609F05DFA01212046FFF7D1FBC82005
:100BE0000DF03EF839462046FFF7CAFB4FF47A7302
:100BF0004FF4407241462046FFF788FB2860E0E74B
:100C0000064BD3E7A00B00209C0800209C0B002083
:100C100020B5010848B50108BC0D0020BA0D002020
:100C20002DE9F041444809F033FAFFF745FF044647
:100C30000121FFF7B1FB2046FFF76EFB41F288333D
:100C40004FF440723D492046FFF760FB3C4E306058
:100C50002046FFF777FB3568002D42D1394809F06F
:100C600017FA01212046FFF78BFB4FF47A700CF046
:100C7000F7FF29462046FFF783FB29462046FFF76A
:100C80008BFB314B1D70314809F002FA304D94F85E
:100C90002420304F2C4E002A14BF3A462A462E4BB1
:100CA0002E492F4809F0F4F932782B4B002A14BF53
:100CB0003A462A462B492A4809F0EAF92A4B94F881
:100CC00024102A48002914BF1946294609F0E0F9E2
:100CD000274809F0DDF933785BB3264B1878BDE877
:100CE000F081254809F0D4F90025144FDFF88C80F5
:100CF0003368AB4206D9404617F8011B09F0C8F922
:100D00000135F5E71E4809F0C3F901212046FFF738
:100D10003DFB4FF47A700CF0A3FF00212046FFF753
:100D200035FB00212046FFF737FB0122064B1A70E6
:100D3000A9E7144BD2E700BF65B501089C08002065
:100D40009C0B002020B50108040D00208CB5010883
:100D50005DB5010858B501088AE5010846BD0108DE
:100D60009CB50108B3B5010862B50108B9B5010821
:100D7000CEB50108BC0D002079B5010804DB0108DF
:100D800089E50108BA0D0020F8B5304809F080F96E
:100D9000FFF792FE01210446FFF7FEFA2C4B1A786A
:100DA0006AB10025012120461D70FFF7E3FA41F2E8
:100DB00088300CF055FF29462046FFF7DBFA02F099
:100DC0004FFD036E60301B689847224B224DC3E9EC
:100DD00082012046FFF7A0FA41F288334FF44072B7
:100DE0001E492046FFF792FA28602046FFF7AAFA2C
:100DF0002E681B4FA6B91B4809F04AF9012120466D
:100E0000FFF7BEFA4FF496700CF02AFF31462046E9
:100E1000FFF7B6FA31462046FFF7BEFA3878F8BD3C
:100E200001212046FFF7B2FA4FF496700CF018FF3C
:100E300020460021FFF7AAFA20460021FFF7ACFA6E
:100E40002A680649084809F099F9E7E765B50108F5
:100E500018000020200000209C0B00209C0800208F
:100E6000B80D002020B5010879B501082DE9F04F33
:100E700087B00BF0A7FB04460BF0B2FB21460246FD
:100E80009E4809F005F902F0EBFC04460BF09AFBD2
:100E900005460BF0A5FB29460246984809F0F8F8EC
:100EA000974809F0F5F8FFF707FE0146204615F0D0
:100EB00097FE204615F050FE924809F0E9F8FFF73A
:100EC0000FFBFA200CF0CCFE14F034FA13F0ACFC5B
:100ED000FFF7DEFB204615F055FE8B4809F0D8F8E9
:100EE000FFF79CFD894E05463368894C13F0010FCE
:100EF00004D103F069FE012320603360266802F00C
:100F0000AFFC00F16001304603F03DFD20688149EF
:100F100003F03BFD26682A687F4903A803F01CFD07
:100F200003A9304603F074FD256800230F228DF8D5
:100F300006007A4903A803F0E5FC03A9284603F05C
:100F400067FD774A8DF8070076492068FFF721FD95
:100F5000754A834675492068FFF71BFD744A814630
:100F600074492068FFF715FD734A8246734920686B
:100F7000FFF70FFD704A8DF8020071492068FFF7F6
:100F800008FD702500266F4B8DF8030003A920682B
:100F900003950493059603F031FE6B4B03A98DF87E
:100FA00000002068CDE90436039503F027FE8DF894
:100FB0000100206804F07CFD64498046206804F04C
:100FC00061FD634A8DF8040062492068FFF7E1FC87
:100FD00007462068604A614980F828B0FFF7D9FCCD
:100FE0005F4A05465F492068FFF7D3FC5E4E4B46DB
:100FF000594632788DF805002068FFF7D5FCDFF8F8
:101000006CB149469DF8033032782068FFF7CCFC7C
:101010004946DFF85C9143469BF800202068FFF7C3
:10102000C3FC434699F800209DF803102068FFF7A1
:10103000BBFC3B46414632782068FFF7B5FC53467F
:10104000394632782068FFF7AFFC39469DF8013009
:101050009BF800202068FFF7A7FC3B469DF807207F
:101060009DF801102068FFF79FFC51469DF8023063
:1010700099F800202068FFF797FC2B4699F800208C
:101080009DF802102068FFF78FFC3A4A29469DF828
:10109000043020681278FFF787FC9DF8053032781D
:1010A0009DF804102068FFF77FFC2B4699F800207C
:1010B0009DF805102068FFF777FC29469DF8003061
:1010C00032782068FFF770FC53469DF806209DF8A3
:1010D00000102068FFF768FC206803F0EFFF264847
:1010E00008F0D6FF206801224FF4C87103F080FF9A
:1010F000002007B0BDE8F04F0CF018BBDCB50108CC
:10110000FBB501080FB6010820B6010898080020B9
:10111000E80C0020850900083DB6010846B6010824
:101120003D0A0008C1C20108210C000856B601089A
:10113000890D000869B60108391200086EB6010869
:1011400077B6010823C201088EB601087CC20108E7
:10115000FD0A00089CB60108FD140008A8B60108A5
:101160002D090008B1B60108BC0D0020BA0D002001
:10117000B80D0020BB0D0020C0B60108F8B54B69C2
:1011800005460E46BBB11C7814F0700204D0402A0C
:1011900013D004F00F0403E05A685468F72C05D804
:1011A00030684268062A0AD0204800E02048BDE89E
:1011B000F84008F06DBF1C46F2E70124F0E7D5F8CF
:1011C000F42104F10801C2F5FA77B94201D91948AE
:1011D000EDE70168AF180868A8508A88BA80D5F88A
:1011E000F421D01D2A44C5F8F40194717269284491
:1011F000127812F0700F05BF5B682246224619680C
:1012000018BF596817F07EFAD5F8F42133691444F1
:10121000C5F8F44103B11B78621CC5F8F4212B55C5
:10122000D5F8F8310133C5F8F831F8BDEFB601084B
:10123000DAB6010801B701082DE9F04F89B0FFF7D0
:10124000EDFB00248146FFF737FC8D4B8D4F1B686B
:101250000546102BC7E97D44C7E97F4417D8012113
:10126000FFF79AF801212846FFF78AF84FF49670A5
:101270000CF0F6FC21462846FFF782F828460021AC
:10128000FFF78AF8804B187809B0BDE8F08F7F4AE5
:10129000CDE90544103B0392049303A801F04DFDF2
:1012A000E8B9012103A801F050FDDDE904329A42BA
:1012B000F3D3D7E97D21764808F0EAFE28460121DC
:1012C000FFF76AF801212846FFF760F84FF496709F
:1012D0000CF0C6FC00212846FFF758F8CEE703A81B
:1012E00001F056FA044603A801F01CFD80B10699EE
:1012F000DDE90432674808F0CBFE674808F0C8FE15
:10130000DDE904130398C91A184408F027FFD0E751
:10131000624808F0BDFE63686148197808F0B8FEBD
:10132000A3686048197808F0B3FE23695E481988FD
:1013300008F0AEFE5D4808F0ABFE2068FFF780FACB
:10134000E3685B481B68196808F0A2FEE3681B6845
:101350001A6840F201739A4243D1564808F098FE49
:10136000E368DFF854815B68DFF850A11E69DFF89D
:1013700050B1002E35D033682BB1404608F088FEBE
:101380003068FFF75DFA73682BB15A6850461278DF
:10139000197808F07DFEB36813B1584608F078FE5E
:1013A000F36823B11A784748114608F071FE336993
:1013B00023B193F90010444808F06AFE736933B111
:1013C0004248197808F064FE7069FFF743FAB36980
:1013D0002BB13F4808F05CFEB069FFF731FAF669BF
:1013E000C7E7E3681A68116840F2017291423FD181
:1013F0005B68D9F844800093D9F84830DFF8D4B05E
:101400000193019A4346424532D0186801F0E5FA4B
:101410000646314808F03CFE3046FFF711FA009BC3
:1014200008F10408D3F810A0BAF1000F24D0DAF8BC
:10143000000078B9CEB9584608F02AFEDAF8140050
:10144000FFF708FA51460F48FFF798FE304601F0C3
:1014500077FAD6E74EB1426871688A4205D13168A1
:10146000006817F03FF90028E5D0DAF81CA0DBE7A8
:10147000204601F075F918E7184808F009FEE5E77D
:101480009C0B002020000020B80D0020A4080020A4
:1014900041B8010815B7010832B701083FB7010884
:1014A0004DB701085EB7010872B701087FB70108A0
:1014B00092B70108A4B70108B9B70108C3B701087A
:1014C000DCB70108EAB70108FCB701080BB801084E
:1014D0001DB801085DB801082CB801086BB80108F7
:1014E000D0E97E329A423FBFD0F80032C0188079EE
:1014F000083034BFC0B20020704700002DE9F04F23
:1015000089B0FFF7D9FA0446FFF788FA012180462F
:101510002046FEF741FFFFF7CFFA0121FEF72AFF31
:101520004FF496700CF09CFB764DFFF7C5FA002146
:10153000FEF720FF20460021FEF72EFF2B685C6897
:1015400094B1714808F0A4FD2C6804F02BFC6F499D
:10155000024604AB204612F093FE6C4902469DF809
:10156000100004F00BFC5CE006F076F8684A6D466B
:10157000D2E90036B6F1004F08BF9C4207D0654F54
:10158000C31A61EB06069F4274EB06034EDA04AC05
:10159000C2E90001604808F07BFD14225F49204643
:1015A00014F0D5FC05F0DCF9074614F03DFF0021EE
:1015B0000646204614F0F6FC0521204614F0F2FC05
:1015C0000121204614F0EEFC0021204614F0EAFC34
:1015D0005349384616F094FA16F07EFC01B22046C4
:1015E00014F0F2FC3146204614F0EEFC94E80F00B3
:1015F00085E80F00284614F0E2FC0446E0B14948B3
:1016000008F046FD284614F0D8FC0446284614F09D
:10161000D6FC2146C2B2012004F0B0FB284614F0EB
:10162000D0FC414B187809B0BDE8F08F102221465C
:10163000284617F08FF8DDE73C4ED6E97E329A4215
:101640004DD004F0AFFB98F850308246022B2DD1DC
:10165000D6E982232D4808F01CFE05244FF004082B
:101660003248FFF73DFF00270546DFF8C4B0DFF83A
:10167000BC9055B3AAEB0402D21B954219DD2FBBD7
:10168000584608F005FD4846FFF72AFF48B1D6F84E
:10169000FC210132C6F8FC21D6F800221044C6F81D
:1016A00000024846FFF71CFF0546E2E74FF003083B
:1016B000D6E7164BD6F80012E01918442A463144F2
:1016C00017F020F87B19DFB2DDE747B13C44214633
:1016D000184808F0DDFC40460C49E2B241E7164CE0
:1016E00023783BB1154808F0D3FC00220749104687
:1016F000227036E7124808F0CBFC04F06BFE114B69
:1017000090E700BF000D00207BB80108F40B00201B
:10171000100000200851010091B80108EC0C0020D5
:1017200000007A44B0B80108BB0D00202000002062
:10173000C5B80108D5B80108860E0020EBB801082D
:1017400002B90108BC0D002073B502F089F80368E6
:1017500004469B6898470AF047FF05460AF044FF95
:1017600001262946002500F57052164808F090FC25
:1017700004F030FE4FF496722B46CDE90065124915
:1017800012480BF0DDFE236831462046DB6898479F
:101790004FF4FA7005F02EFA23682946DB682046DC
:1017A00098470B4808F074FC0A4808F071FC0CF0EC
:1017B000ADF840F25231084804F0DEFE284602B08F
:1017C00070BD00BF18B9010831B901086D0E0008DD
:1017D0003AB901084DB901088AE50108FF22014B19
:1017E0001A707047A40B002010B5102008F0ECFC14
:1017F00004461022002116F0ADFF204610BD10B5A2
:10180000044680B1006801F09BF8606801F098F828
:10181000A06801F095F8E06801F077FD2046BDE88A
:10182000104008F0BBBC10BD38B50446FFF7DCFF24
:101830000546204601F07BFA702806D00123E360BC
:101840002846FFF7DCFF002528E0204601F04AFA91
:101850000428F3D1204601F080F82860204601F0EA
:1018600061FA0028ECD1204601F077F86860204644
:1018700001F058FA0028E3D1204601F06EF8A86084
:10188000204601F04FFA0028DAD1204601F0E4FDAD
:10189000E860204601F046FA0028D1D1284638BD3C
:1018A00010B50446012008F08FFC047010BD70B51F
:1018B000044601F04EFA30B9204601F038FA4028CB
:1018C00003D00123E360002070BD204601F00AFA36
:1018D00001280546F5D1204601F02FFA0646294693
:1018E000204636B101F031FAFF20BDE87040FFF725
:1018F000D7BF01F02AFA3046F7E708B108F04EBC2E
:10190000704708B5042008F05FFC0023036008BDA1
:1019100010B5044638B1006801F012F82046BDE861
:10192000104008F03BBC10BD38B50446FFF7E9FF96
:101930000546204601F0FBF9702806D00123E3603C
:101940002846FFF7E5FF00250DE0204601F0CAF923
:101950000128F3D1204601F000F82860204601F06C
:10196000E1F90028ECD1284638BD08B5042008F07C
:101970002BFC0023036008BD10B5044638B1006895
:1019800000F0DEFF2046BDE8104008F007BC10BDA7
:1019900038B50446FFF7E9FF0546204601F0C7F9D0
:1019A000702806D00123E3602846FFF7E5FF0025F5
:1019B0000DE0204601F096F90128F3D1204600F011
:1019C000CCFF2860204601F0ADF90028ECD1284674
:1019D00038BD10B5044698B1006800F0B1FF6068EA
:1019E00000F0AEFF206900F0ABFFA06800F0A8FF98
:1019F000E06800F0A5FF2046BDE8104008F0CEBB2F
:101A000010BD38B50446142008F0DEFB1422002176
:101A1000054616F09FFE204601F089F9702806D091
:101A20000123E3602846FFF7D4FF002531E020467C
:101A300001F058F90528F3D1204600F08EFF286008
:101A4000204601F06FF90028ECD1204600F085FF18
:101A50006860204601F066F90028E3D1204600F0D6
:101A60007CFFA860204601F05DF90028DAD120460D
:101A700000F073FFE860204601F054F90028D1D14E
:101A8000204600F06AFF2861204601F04BF900284B
:101A9000C8D1284638BD10B51C2008F095FB044677
:101AA0001C22002116F056FE204610BD10B504463B
:101AB000C8B1006800F044FF606800F041FFA06812
:101AC00000F03EFFE06801F09BF9206900F0F2FCB5
:101AD000606900F035FFA06901F092F92046BDE889
:101AE000104008F05BBB10BD38B50446FFF7D3FFCC
:101AF0000546204601F01BF9702806D00123E3605B
:101B00002846FFF7D3FF002543E0204601F0EAF81E
:101B10000728F3D1204600F020FF2860204601F07E
:101B200001F90028ECD1204600F017FF686020463C
:101B300001F0F8F80028E3D1204600F00EFFA8607D
:101B4000204601F0EFF80028DAD1204601F067F9CD
:101B5000E860204601F0E6F80028D1D1204600F0E8
:101B6000B3FC2861204601F0DDF80028C8D12046EA
:101B700000F0F3FE6861204601F0D4F80028BFD1E0
:101B8000204601F04CF9A861204601F0CBF800286E
:101B9000B6D1284638BD10B5142008F015FB044610
:101BA0001422002116F0D6FD204610BD10B50446C3
:101BB00098B1006800F0C4FE606800F0C1FEA06843
:101BC00000F0BEFEE06801F075F9206900F0B8FE93
:101BD0002046BDE8104008F0E1BA10BD38B5044613
:101BE000FFF7D9FF0546204601F0A1F8702806D07E
:101BF0000123E3602846FFF7D9FF002531E02046A6
:101C000001F070F80528F3D1204600F0A6FE286008
:101C1000204601F087F80028ECD1204600F09DFE18
:101C20006860204601F07EF80028E3D1204600F0ED
:101C300094FEA860204601F075F80028DAD120460D
:101C400001F053F9E860204601F06CF80028D1D18A
:101C5000204600F082FE2861204601F063F800284B
:101C6000C8D1284638BD08B50C2008F0ADFA0022CE
:101C700002604260826008BD10B5044668B1006829
:101C800000F05EFE606801F015F9A06801F03DFB10
:101C90002046BDE8104008F081BA10BD38B50446B2
:101CA000FFF7E1FF0546204601F041F8702806D015
:101CB0000123E3602846FFF7DFFF00251FE02046F1
:101CC00001F010F80328F3D1204600F046FE28600A
:101CD000204601F027F80028ECD1204601F005F954
:101CE0006860204601F01EF80028E3D1204601F08C
:101CF000B3FBA860204601F015F80028DAD1284689
:101D000038BD10B5242008F05FFA044624220021D3
:101D100016F020FD204610BD10B50446F8B100684D
:101D200000F00EFE606801F06BF8A06800F0EDFDB9
:101D3000E06801F0BFF8206901F062F8606900F026
:101D4000E4FDA06900F0E2FAE06900F0F9FD206A24
:101D500000F0F6FD2046BDE8104008F01FBA10BDA7
:101D600038B50446FFF7CDFF0546204600F0DFFFFB
:101D7000702807D001232846E360FFF7CDFF002538
:101D8000284638BD204600F0ADFF0928F2D1204694
:101D900000F0E3FD2860204600F0C4FF0028E9D1F0
:101DA000204601F03CF86860204600F0BBFF0028A8
:101DB000E0D104226021204600F060FDA8602046AA
:101DC00000F0B0FF0028D5D1204601F08EF8E86081
:101DD000204600F0A7FF0028CCD1204601F01FF8D4
:101DE0002861204600F09EFF0028C3D10822602110
:101DF000204600F043FD6861204600F093FF002874
:101E0000B8D120460E4A0F4900F0A9FAA861204631
:101E100000F088FF0028ADD1204600F09EFDE8616B
:101E2000204600F07FFF0028A4D1204600F095FD59
:101E30002862204600F076FF0028A1D09AE700BF74
:101E4000833200084333000810B5242008F0BCF9A1
:101E500004462422002116F07DFC204610BD70B5FA
:101E6000044638B3006800F06BFD606800F068FD60
:101E7000A06800F065FDE068FFF73FFD206900F015
:101E8000BFFF606900F0BCFFA06901F013F8E569CD
:101E900045B12E4630686D6800F052FD304608F0BE
:101EA0007DF9F5E7206A01F030FA2046BDE8704080
:101EB00008F074B970BD2DE9F8430446FFF7C4FF7C
:101EC0000546204600F033FF702806D00123E3606A
:101ED0002846FFF7C4FF002550E0204600F002FF2F
:101EE0000928F3D1204600F038FD2860204600F094
:101EF00019FF0028ECD1204600F02FFD6860204635
:101F000000F010FF0028E3D1204600F026FDA86075
:101F1000204600F007FF0028DAD12046FFF7C7FC73
:101F2000E860204600F0FEFE0028D1D1204600F0F7
:101F300076FF2861204600F0F5FE0028C8D1204633
:101F400000F06DFF6861204600F0ECFE0028BFD174
:101F5000204600F0CAFFA861204600F0E3FE0028FA
:101F6000B6D1204600F0F5FE58B1204601F074FAD3
:101F70002862204600F0D6FE0028A9D12846BDE8F8
:101F8000F883204600F0D3FE70289FD1204600F051
:101F9000A9FE4FF000080746C146002FE5DD0820E6
:101FA00008F012F90646C0F80090C0F804902046E8
:101FB00000F0D3FC3060204600F0B4FE002887D14A
:101FC000EB691BB9EE61B046013FE6E7C8F8046073
:101FD000F9E710B5044668B1006800F0B1FC60682C
:101FE00000F093FCA06800F090FC2046BDE8104093
:101FF00008F0D4B810BD10B5044680B1006800F0F8
:10200000FFFE606800F081FCA06800F07FF9E068E6
:1020100000F096FC2046BDE8104008F0BFB810BDA7
:1020200010B5044650B1006801F069FA606800F02C
:1020300087FC2046BDE8104008F0B0B810BD10B5D0
:10204000202008F0C1F804462022002116F082FB6F
:10205000204610BD10B50446E0B1006800F070FCE9
:10206000606800F0CDFEA06800F04FFCE06800F072
:1020700021FF206900F04AF9606900F047F9A06982
:1020800000F05EFCE06900F05BFC2046BDE810401B
:1020900008F084B810BD000038B50446FFF7CFFF44
:1020A0000546204600F043FE702807D0012328464D
:1020B000E360FFF7CFFF0025284638BD204600F03B
:1020C00011FE0828F2D1204600F047FC2860204687
:1020D00000F028FE0028E9D1204600F0A0FE68604C
:1020E000204600F01FFE0028E0D104226021204697
:1020F00000F0C4FBA860204600F014FE0028D5D1F3
:10210000204600F0F2FEE860204600F00BFE0028BA
:10211000CCD12046134A144900F021F92861204609
:1021200000F000FE0028C1D12046104A104900F0FE
:1021300016F96861204600F0F5FD0028B6D120466A
:1021400000F00BFCA861204600F0ECFD0028ADD1AA
:10215000204600F002FCE861204600F0E3FD002884
:10216000AAD0A3E7D31F000887210008F71F0008A3
:102170000D22000808B50C2008F026F800220260A5
:102180004260826008BD38B50446FFF7F3FF05469C
:10219000204600F0CCFD702807D001232846E360DC
:1021A000FFF717FF0025284638BD204600F09AFDAE
:1021B0000328F2D1204600F0D0FB2860204600F032
:1021C000B1FD0028E9D101226021204600F056FB34
:1021D0006860204600F0A6FD0028DED101225021D3
:1021E000204600F04BFBA860204600F09BFD002835
:1021F000D9D0D2E710B5102007F0E6FF0446102230
:10220000002116F0A7FA204610BD000038B504469C
:10221000FFF7F0FF0546204600F089FD702807D043
:1022200001232846E360FFF7E6FE0025284638BD77
:10223000204600F057FD0428F2D1204600F0EFFDC3
:102240002860204600F06EFD0028E9D108226021B8
:10225000204600F013FB6860204600F063FD002874
:10226000DED12046094A0A4900F079F8A8602046E4
:1022700000F058FD0028D3D1204600F06EFBE86046
:10228000204600F04FFD0028D0D0C9E721200008EB
:10229000A522000808B5082007F096FF002202607A
:1022A000426008BD38B50446FFF7F4FF05462046F6
:1022B00000F03DFD702807D001232846E360FFF7BA
:1022C000AFFE0025284638BD204600F00BFD022851
:1022D000F2D1204601F029F92860204600F022FDC5
:1022E0000028E9D1204600F038FB6860204600F065
:1022F00019FD0028E6D0DFE710B504460C2007F0F2
:1023000063FF002202604260846010BD38B504465D
:1023100088B938BD50F82500A36898470135D4E93D
:1023200000039D42F6DB08B107F038FF2046BDE808
:10233000384007F033BF0025F1E738B5436804465D
:10234000013343600D460068990017F0CFF86368C9
:10235000206003F18043013B40F8235038BD2DE954
:10236000F84305468846164600F0E1FC70281AD16D
:102370003046FFF7C1FF0446284600F0B3FC0027B3
:102380000646B74202DB2046BDE8F8832846C04730
:102390008146284600F0C6FC28B949462046FFF78A
:1023A000CCFF0137EDE701232046EB60FFF7AEFFDE
:1023B0000024E8E710B5202007F006FF044620229D
:1023C000002116F0C7F9204610BD38B5044600F0CC
:1023D000AEFC702804D001230025E360284638BDF8
:1023E000204600F07FFC0728F5D1FFF7E3FF054604
:1023F000204600F0B2FA2860204600F093FC002846
:10240000E9D1204600F0C3FC6860204600F08AFC59
:102410000028E0D1204600F002FDA860204600F030
:1024200081FC0028D7D101226021204600F026FA45
:10243000E860204600F076FC0028CCD10122502133
:10244000204600F01BFA2861204600F06BFC0028B3
:10245000C1D1204601F069F86861204600F062FCB5
:102460000028B8D1204600F078FAA861204600F094
:1024700059FC0028B2D0AEE710B50446C8B10068D8
:1024800000F05EFA606800F076FCA06800F0B8FC2E
:10249000E06800F03AFA206900F037FA606901F06C
:1024A0002EF8A06900F04CFA2046BDE8104007F075
:1024B00075BE10BD10B530B1C469FFF7DDFF14B1B2
:1024C0002046E469F9E710BDF8B5054600F041FC87
:1024D000044608B1002406E0284600F028FC7028D5
:1024E00003D00123EB602046F8BD284600F0FAFB3C
:1024F000061EEFDD2846FFF768FF0446284600F079
:1025000011FC70B92746013E002EECD02846FFF79B
:102510005CFFF861284600F005FC10B9FF69013E38
:10252000F2E701232046EB60FFF7C4FFD2E700008B
:1025300038B50546082007F047FE0023044603602F
:102540004360284600F0F3FB702806D00123EB60BF
:10255000204607F023FE002459E0284600F0C2FB85
:102560000228F3D104226021284600F087F9206078
:10257000284600F0D7FB0028EAD12368196840F20A
:102580000143994255D020D840F20123994248D0C6
:102590000DD840F2011399423BD0B1F5007F3CD0F9
:1025A000B1F5807F2FD02D4816F01CFF2FE040F2B0
:1025B0000133994239D0B1F5806F02D0B1F5407F37
:1025C000F1D12846FFF777FC20E0B1F5E06F3CD071
:1025D0000DD840F2015399422FD0B1F5C06F30D0E1
:1025E000B1F5A06FDFD12846FFF7F8FA0EE040F210
:1025F000017399422DD04FF601739942D3D12846E9
:10260000FFF712F902E0284600F035FA6060204634
:1026100038BD284600F0AEFAF8E72846FFF784F9FF
:10262000F4E72846FFF7B4F9F0E72846FFF734FD52
:10263000ECE72846FFF794FBE8E72846FFF72EFB78
:10264000E4E7284600F009FBE0E72846FFF7D9F960
:10265000DCE72846FFF748FAD8E700BF7EB9010853
:1026600010B50446002875D003681A6840F201438B
:102670009A425BD021D840F201239A424ED00ED824
:1026800040F201139A4241D0B2F5007F42D0B2F538
:10269000807F30D03049314816F0A4FE2EE040F261
:1026A00001339A423ED0B2F5806F02D0B2F5407F3E
:1026B000F0D16068FFF7D3FB20E0B2F5E06F41D0C6
:1026C0000DD840F201539A4234D0B2F5C06F35D0E4
:1026D000B2F5A06FDED14068FFF768FA0EE040F275
:1026E00001739A4232D04FF601739A42D2D14068B8
:1026F000FFF785F802E0406800F09FF9206800F0DD
:1027000004F92046BDE8104007F048BD406800F0DD
:1027100016FAF3E74068FFF7FBF8EFE74068FFF7CA
:102720002BF9EBE74068FFF795FCE7E74068FFF718
:10273000F3FAE3E74068FFF79FFADFE7406800F04D
:1027400074FADBE74068FFF744F9D7E74068FFF722
:10275000ADF9D3E710BD00BFCBB90108ACB9010892
:1027600010B5044698B1006800F0EAF8606800F01F
:10277000CCF8A06800F0C9F8E068FFF771FF2069A5
:1027800000F0C3F82046BDE8104007F007BD10BDBB
:1027900038B50446142007F017FD14220021054621
:1027A00015F0D8FF204600F0C2FA702806D00123A9
:1027B000E3602846FFF7D4FF00253FE0204600F005
:1027C00091FA0628F3D1204600F0C7F82860204689
:1027D00000F0A8FA0028ECD101226021204600F088
:1027E0004DF86860204600F09DFA0028E1D10122F2
:1027F0006021204600F042F8A860204600F092FADE
:102800000028D6D12046FFF793FEE860204600F06E
:1028100089FA0028CDD102226021204600F02EF84E
:102820002861204600F07EFA0028C2D1204600F040
:1028300084FA18B90121204600F087FA284638BDED
:10284000B0B504460D46CB1D23F0070300AFADEB3A
:10285000030D0A460146684615F054FF631E0DEB52
:102860000502C4F10104E1188D4202F1FF3201DCDE
:10287000BD46B0BD117803F8011FF4E72DE9F0471C
:1028800005460C46904600F064FA064638B92846DC
:1028900000F04DFAA042814603D00123EB600024F2
:1028A00030E0284600F01EFA071EF6DB4745F4DC50
:1028B000404607F089FC31464246044615F04AFF7F
:1028C000284600F03AFAB9F1500F08BFC0F3C0161D
:1028D000284600F036FAA8EB070904EB090A01467E
:1028E0003A46504615F00EFF26B14A46FF212046D3
:1028F00015F030FF41462046FFF7A2FF3946284633
:1029000000F023FA2046BDE8F08708B107F046BC86
:10291000704770B5064608200D4607F055FC0023A9
:102920009D4204460360436008DD284607F04CFCE6
:102930002A463146206015F0E5FE6560204670BDF0
:1029400010B5044640B1006808B107F027FC2046E6
:10295000BDE8104007F022BC10BD70B5044600F081
:10296000F8F928B9204600F0E2F918B10123E36034
:1029700000250FE0204600F0B5F9061EF6DB2046E4
:1029800000F0DFF93146FFF7C4FF31460546204627
:1029900000F0DBF9284670BD03463038C0B2092884
:1029A0000DD9A3F16102052A02D8573BD8B270476E
:1029B000A3F14102052A01D8373BF7E70020704711
:1029C00010B501460078FFF7E7FF04464878FFF7A7
:1029D000E3FF40EA0410C0B210BD2DE9F84300AF98
:1029E000044616F0D7FEC3071AD44510EB1D23F09A
:1029F0000703ADEB030DE8460DF1FF3604EB450987
:102A00004C4506D129464046FFF783FFBD46BDE849
:102A1000F8832046FFF7D4FF023406F8010FEFE7F2
:102A20000020F3E710B51C2007F0CEFB04461C2263
:102A3000002115F08FFE204610BD10B50446C8B128
:102A40000068FFF77DFF6068FFF77AFFA068FFF777
:102A500077FFE068FFF774FF2069FFF771FF606997
:102A6000FFF76EFFA069FFF750FF2046BDE810405A
:102A700007F094BB10BD38B50446FFF7D3FF0546F9
:102A8000204600F054F9702806D00123E360284660
:102A9000FFF7D3FF002545E0204600F023F9072883
:102AA000F3D12046FFF759FF2860204600F03AF99D
:102AB0000028ECD12046FFF750FF6860204600F068
:102AC00031F90028E3D12046FFF747FFA8602046F0
:102AD00000F028F90028DAD12046FFF73EFFE86031
:102AE000204600F01FF90028D1D12046FFF735FF1E
:102AF0002861204600F016F90028C8D12046FFF7CB
:102B00002CFF6861204600F00DF90028BFD101229A
:102B100060212046FFF7B2FEA861204600F002F9CE
:102B20000028B4D1284638BD10B5182007F04CFB5A
:102B300004461822002115F00DFE204610BD10B5E8
:102B40000446B0B10068FFF7FBFE6068FFF7F8FECF
:102B5000A068FFF7F5FEE068FFF7F2FE206900F0DD
:102B60004FF96069FFF7D1FE2046BDE8104007F03D
:102B700015BB10BD38B50446FFF7D6FF0546204605
:102B800000F0D5F8702806D00123E3602846FFF74F
:102B9000D6FF00253CE0204600F0A4F80628F3D13B
:102BA0002046FFF7DAFE2860204600F0BBF8002838
:102BB000ECD12046FFF7D1FE6860204600F0B2F865
:102BC0000028E3D12046FFF7C8FEA860204600F0A9
:102BD000A9F80028DAD12046FFF7BFFEE8602046BA
:102BE00000F0A0F80028D1D1204600F018F92861A3
:102BF000204600F097F80028C8D101226021204625
:102C0000FFF73CFE6861204600F08CF80028BDD13B
:102C1000284638BD10B5142007F0D6FA0446142211
:102C2000002115F097FD204610BD10B5044698B15F
:102C30000068FFF785FE6068FFF782FEA068FFF777
:102C40007FFEE06800F036F9206900F05EFB204668
:102C5000BDE8104007F0A2BA10BD38B50446FFF732
:102C6000D9FF0546204600F062F8702806D00123FF
:102C7000E3602846FFF7D9FF002531E0204600F049
:102C800031F80528F3D12046FFF767FE286020467B
:102C900000F048F80028ECD12046FFF75EFE68609F
:102CA000204600F03FF80028E3D12046FFF755FE0C
:102CB000A860204600F036F80028DAD1204600F05F
:102CC00014F9E860204600F02DF80028D1D1204604
:102CD00000F0C2FB2861204600F024F80028C8D18B
:102CE000284638BDF0B5836805680022EB5C46686D
:102CF00003F07003703B18BF4FF0FF338168B1429F
:102D000001F1010402D38460D018F0BD695C01F0C8
:102D10000F07090647EA0212F5D58460002BEDD0B3
:102D2000013BEBE7C068003818BF0120704702681C
:102D30008368D05C00F07000704702688368D05CE4
:102D40007047026880681044704783680B44836052
:102D50007047034682680168885C01280ABF013217
:102D600000209A60704708B5082007F02DFA00226D
:102D70000260426008BD10B5044638B14068FFF7F4
:102D8000C4FD2046BDE8104007F008BA10BDF8B5F4
:102D90000646FFF7DEFF30BB3046FFF7C8FF0546AB
:102DA0003046FFF7CAFF0746FFF7DDFF602D0570CD
:102DB00004464FF0010519D107F00F07013F00E06D
:102DC0006D00AF42FCDC2A4660213046FFF756FD1D
:102DD000237860602B4323703046FFF7A3FF18B1C0
:102DE0002046FFF7C8FF00242046F8BDF560F3E752
:102DF00008B5082007F0E8F900220260426008BD2B
:102E000010B5044650B10068FFF77FFD6068FFF71A
:102E10007CFD2046BDE8104007F0C0B910BD38B5B4
:102E20000446FFF796FF60B9FFF7E2FF054620462C
:102E3000FFF77DFF702806D00123E3602846FFF7E7
:102E4000DFFF00251AE02046FFF74CFF0228F3D1F0
:102E5000012260212046FFF711FD28602046FFF780
:102E600061FF0028EAD1042260212046FFF706FD19
:102E700068602046FFF756FF0028DFD1284638BD9E
:102E800008B5082007F0A0F900220260426008BDE2
:102E900038B503680446013303600D464068990065
:102EA00016F024FB2368606003F18043013B40F887
:102EB000235038BD38B50446B0B143687BB10368D0
:102EC000002B0CDD0025636853F82500FFF738FD63
:102ED00023680135AB42F6DC606807F05FF92046F5
:102EE000BDE8384007F05AB938BDF8B50546FFF7D8
:102EF00030FF48B9FFF7C4FF04462846FFF717FF25
:102F0000702803D00123EB60002405E02846FFF77A
:102F1000E9FE0646002E01DC2046F8BD2846FFF7F4
:102F20001CFD07462846FFF7FDFE28B10123204679
:102F3000EB60FFF7BFFFE7E71FB139462046FFF719
:102F4000A7FF013EE6E710B5102007F03DF9044663
:102F50001022002115F0FEFB204610BD38B5C368D5
:102F600004460133C3600D468068990016F0BEFA2E
:102F7000E368A06003F18043013B40F8235038BD73
:102F800010B55C2007F020F904465C22002115F002
:102F9000E1FB204610BD10B50446002849D000686A
:102FA000FFF7CEFC6068FFF72BFFA068FFF7ADFCD2
:102FB000E068FFF7AAFC2069FFF7A7FC6069FFF74C
:102FC000A4FCA069FFF7A1FCE069FFF79EFC206A62
:102FD000FFF79BFC606AFFF798FCA06AFFF795FC7F
:102FE000E06AFFF792FC206BFFF7AAFC606BFFF72B
:102FF0008CFCA06BFFF789FCE06BFFF786FC206C74
:10300000FFF783FC606CFFF780FCA06CFFF77DFC92
:10301000E06CFFF77AFC206DFFF777FC606DFFF73F
:1030200074FCA06DFFF78CFC2046BDE8104007F053
:10303000B5B810BD38B50446FFF78BFE60B9FFF791
:103040009FFF05462046FFF772FE702806D0012339
:10305000E3602846FFF79FFF002505E12046FFF7C4
:1030600041FE1728F3D12046FFF777FC2860204661
:10307000FFF758FE0028ECD12046FFF7D0FE68602D
:103080002046FFF74FFE0028E3D1082260212046AA
:10309000FFF7F4FBA8602046FFF744FE0028D8D1D4
:1030A000012260212046FFF7E9FBE8602046FFF798
:1030B00039FE0028CDD1012250212046FFF7DEFB4A
:1030C00028612046FFF72EFE0028C2D10822502199
:1030D0002046FFF7D3FB68612046FFF723FE002858
:1030E000B7D1012260212046FFF7C8FBA861204626
:1030F000FFF718FE0028ACD1012250212046FFF72F
:10310000BDFBE8612046FFF70DFE0028A1D1082293
:1031100050212046FFF7B2FB28622046FFF702FE4F
:10312000002896D1012260212046FFF7A7FB6862A4
:103130002046FFF7F7FD00288BD1012250212046C1
:10314000FFF79CFBA8622046FFF7ECFD002880D12A
:10315000082250212046FFF791FBE8622046FFF746
:10316000E1FD00287FF475AF2046FFF7F6FB2863EA
:103170002046FFF7D7FD00287FF46BAF01226021C6
:103180002046FFF77BFB68632046FFF7CBFD002856
:103190007FF45FAF012250212046FFF76FFBA86349
:1031A0002046FFF7BFFD00287FF453AF08225021CF
:1031B0002046FFF763FBE8632046FFF7B3FD0028D6
:1031C0007FF447AF012260212046FFF757FB2864B8
:1031D0002046FFF7A7FD00287FF43BAF01225021D6
:1031E0002046FFF74BFB68642046FFF79BFD002855
:1031F0007FF42FAF082250212046FFF73FFBA86441
:103200002046FFF78FFD00287FF423AF01226021C5
:103210002046FFF733FBE8642046FFF783FD0028D4
:103220007FF417AF012250212046FFF727FB2865C6
:103230002046FFF777FD00287FF40BAF08225021CE
:103240002046FFF71BFB68652046FFF76BFD002853
:103250007FF4FFAE2046FFF780FBA8652046FFF70E
:1032600061FD00287FF4F5AE284638BD10B5142066
:1032700006F0AAFF04461422002115F06BFA20463E
:1032800010BD10B5044698B10068FFF759FB60689F
:10329000FFF73BFBA068FFF738FBE06800F02FF971
:1032A0002069FFF74DFB2046BDE8104006F076BFD1
:1032B00010BD10B5044638B3D0E90030FBB11B781F
:1032C000013B032B16D8DFE803F0020C0F1200F0CD
:1032D00016F92068FFF719FB2046BDE8104006F0FC
:1032E0005DBFFFF7CEFFF4E7FFF755FEF1E7FFF70D
:1032F00087FDEEE70028ECD006F050FFE9E7002854
:10330000EAD006F04BFFE7E710BD38B50446B8B188
:103310000068FFF715FB6068FFF7CBFF0025D4E9D5
:1033200002039D4206DB06F039FF2046BDE8384027
:1033300006F034BF50F82500FFF7E7FF0135EEE750
:1033400038BD38B50446FFF704FD60B9FFF78EFFBE
:1033500005462046FFF7EBFC702806D00123E3600A
:103360002846FFF78EFF002535E02046FFF7BAFC20
:103370000528F3D12046FFF7F0FA28602046FFF732
:10338000D1FC0028ECD1012260212046FFF776FA1B
:1033900068602046FFF7C6FC0028E1D101225021D9
:1033A0002046FFF76BFAA8602046FFF7BBFC002819
:1033B000D6D1204600F0B9F8E8602046FFF7B2FC0D
:1033C0000028CDD12046FFF7C8FA28612046FFF734
:1033D000A9FC0028C4D1284638BD38B50546FFF7FA
:1033E000B8FC60B9FFF74CFD04462846FFF79FFC88
:1033F000702806D00123EB602046FFF75AFF002417
:103400001CE02846FFF76EFC0228F3D10122602160
:103410002846FFF733FA20602846FFF783FC002890
:10342000EAD123681B78013B032BE3D8DFE803F0E4
:1034300002080C10284600F078F86060204638BD7D
:103440002846FFF77EFFF8E72846FFF7F3FDF4E78D
:103450002846FFF7E4FCF0E7F8B50446FFF779FCEF
:1034600060B9FFF770FD05462046FFF760FC702845
:1034700006D00123E3602846FFF747FF002525E03B
:103480002046FFF72FFC0328F3D12046FFF765FA0B
:1034900028602046FFF746FC0028ECD12046FFF7C5
:1034A0009CFF68602046FFF73DFC0028E3D12046E2
:1034B000FFF74FFC50B92046FFF739FC7028D8D1F0
:1034C0002046FFF70FFC0646002E01DC2846F8BD1B
:1034D0002046FFF7C1FF07462046FFF723FC0028E0
:1034E000C9D11FB139462846FFF738FD013EEBE749
:1034F00008B5082006F068FE0023036008BD10B57B
:10350000044688B10378406823B1402B09D0FFF707
:10351000FCF901E0FFF714FA2046BDE8104006F080
:103520003DBEFEF7EAF9F7E710BDF8B50546FFF72F
:1035300010FC38BB2846FFF7FAFB07462846FFF782
:10354000FCFB0646FFF7D4FFF9B2402F044601709A
:103550001BD003DC5FB10123EB600CE0502F01D0E6
:10356000602FF8D106F00F060127013E12E0284631
:10357000FFF7F3F960602846FFF7D4FB18B1204647
:10358000FFF7BDFF00242046F8BD2846FEF78FF95F
:10359000F0E77F00BE42FCDC3A462846FFF76EF9B2
:1035A000237860603B432370E5E7000038B50A4CA0
:1035B00005460121204603F0C7FD002320461A4698
:1035C000012103F0FBFC204685F001020121BDE84A
:1035D000384003F0C3BD00BF0000024008B5012021
:1035E000FFF7E4FFBDE80840032004F0E1BC084613
:1035F000FFF7DCBF10B50446024B036013F00AFB73
:10360000204610BDD4BD010810B50446054B50300E
:1036100040F8503C044B40F8083CFFF7EBFF2046D5
:1036200010BD00BFE8BD010834C0010810B5044654
:10363000FFF7E0FF2046082112F010FD204610BDE4
:1036400010B50446FFF7E0FF20467C2112F006FD8E
:10365000204610BD04F05CBD10B50C460AF098FD84
:10366000022808D14FF47A704443B4FBF0F0BDE86F
:1036700010400AF0F5BA2046BDE8104003F0BABA8F
:1036800010B5094C094806F003FD20460B2103F054
:103690005BFD002320461A460B2103F08FFCBDE89A
:1036A000104003F08DBA00BF00000240E1B90108EC
:1036B00008B5034806F0ECFCBDE8084004F028BD5E
:1036C000FDB90108021E18BF01220321014803F0C1
:1036D00045BD00BF000402400321014803F047BD7F
:1036E00000040240024B0121186803681B68184758
:1036F000140D002008B5022003F0C6F903F028FAE3
:1037000000F092FC03F04EFA00F078FE03F0AEFFFA
:103710000C4802F0F7FE4FF4E13004F0BFFA0A4B18
:103720001A680AB9094A1A60094B1A680AB9074A9D
:103730001A60084806F0ACFCBDE80840064806F0F0
:10374000A7BC00BFDD350008081000204D7B000835
:103750000C1000201BBA010833BA01082DE9F3410F
:10376000044626464FF01B0813F0ECF9264B04F1F3
:10377000210746F8113B10220021304614F0EAFFE1
:1037800042460021384614F0E5FF002521461F4B34
:10379000C4E90F5504F1480041F8443F01F022F814
:1037A0001B4BC4E91B55A3651A4B84F85C50C4E954
:1037B0001835194B84F87450A567184DA36618483E
:1037C00006F066FC6B6E174A01936B6D41460093E1
:1037D0002B6D384615F0FCFE296D304606F063FD72
:1037E000696D04F1150006F05EFD696E04F11900C3
:1037F00006F059FD296D04F11D0006F054FD204628
:1038000002B0BDE8F08100BFE8BD010894BE010828
:10381000A4BE0108FCBE0108C0BE01080000F81FDC
:1038200049BA01085EBA010810B5094CFFF762FFFA
:103830002368DB0709D40748FFF790FF0123064AF6
:1038400006490448236013F03BFA024810BD00BF4C
:103850000C0D0020180D0020000000200936000883
:1038600038B5064D064C2B6813F0010F04D1FFF755
:10387000DBFF012320602B60206838BD100D002085
:10388000940D002010B5FFF7EBFF836F11203BB1C3
:1038900004F02CFCFFF7E4FFBDE81040836F1847ED
:1038A000BDE8104004F02FBC08B50B21054803F01B
:1038B00065FC28B1BDE808400B21024803F074BC48
:1038C00008BD00BF0000024008B519B1BDE80840BE
:1038D000FFF7D6BE044806F0DBFBBDE80840022235
:1038E0000B21024803F0AABB70BA01080000024095
:1038F00070B504462E4804F1440506F0C9FB28467D
:10390000002100F097FD0021284600F0A9FD204687
:1039100013F048F90CF04EFB20460021FFF7D4FFCE
:103920000BF046FA01220C21224803F087FB03F03A
:10393000CDFF04F1480000F037FF23682046DB6824
:1039400004F16805002198471B4E0021284600F02D
:1039500013FE03F085FC194806F09AFB04F09CF86E
:1039600003F020F9304601220D2103F067FB01220C
:1039700030460E2103F062FB0021084603F052FF9F
:1039800004F1580000F082FD0121284600F0F4FD0A
:103990004FF4E13004F082F9094806F079FB0BF0AE
:1039A0002DF903F091FF2046BDE8704013F007B9F0
:1039B00088BA01080004024000000240ACBA0108C5
:1039C00096C3010838B50546FFF76EFF044628B1D7
:1039D00000212846FFF778FF03F0F2F802F0C0FF5D
:1039E00005460CB1FFF74CFE284638BD70B50C46B5
:1039F00006461549204614F03FFA20B9002120461A
:103A000014F01CFA70B11149204614F079F814F042
:103A10003DFA01460E4806F03BFB4FF4C0710D48DD
:103A200002F0AAFD3046FFF73FFF054648B9304691
:103A3000FFF7C8FF0146204614F01EFA08B1FFF751
:103A40001FFE284670BD00BF3333534000007A4448
:103A5000BABA01088AE5010870B52D4A054613680F
:103A6000D6B0DB0705D42B4900F168030B600123B6
:103A7000136029492846FFF7B9FF0646274806F094
:103A800007FB002105F1440000F0EAFC244C254B23
:103A9000E360254B2361254BA360254B6360254BD9
:103AA0002360254B6361254BA361254BE36104F142
:103AB00010030FCB8DE80F0094E80F0012F098FD73
:103AC000002305A8EB632B6412F01AFD9DF8143057
:103AD00005F13C04012B14D1DDF8153005A8EB638A
:103AE000DDF819302B6412F0DBFC164806F0D0FA32
:103AF0000821204606F032FBBDF91611124806F0E7
:103B0000C7FA31462846FFF7DFFE56B070BD00BF4A
:103B1000080D0020140D002000004040E9BA010803
:103B2000F41D0020F56B00087D6B0008E5360008E9
:103B3000D9360008C536000891A0000845C3000822
:103B400081C300080ABB010830BB01087FB5F82318
:103B500000F15805064628468DF80F3000F09CFC11
:103B600002230DF10F0100930122A123284600F04A
:103B700097FC4FF400430822009306F16C01A12347
:103B80000446284600F0B8FC0440E4B2284600F0A1
:103B900085FC204604B070BD30B58BB0044604F0FF
:103BA00035FA01465A4806F073FA04F089FA0146DC
:103BB000584806F06DFA584806F06AFA204600F0B8
:103BC000D3FB04F1580500F009FB00F0B5FA5348A7
:103BD000534906F05DFA284600F058FC38B95148C0
:103BE00006F056FA40F23B114F4802F0C5FC02F0D5
:103BF000E7FF2046FFF7AAFF20B94FF4A0714A481B
:103C000002F0BAFC94F8733094F86D20049394F8A1
:103C1000723094F86C10039394F871304348029317
:103C200094F87030019394F86F30009394F86E30EC
:103C300006F02EFA284600F081FA284600F0E0FA55
:103C400004F14405002184F87400284600F0F2FBDA
:103C5000012000F0D5FD0021284600F001FC0120E4
:103C600000F0ECFD2046FFF7F7FE204600F014FBC5
:103C70002F4806F00DFA4FF4FA7014F015FD0546C2
:103C800000283ED12B4806F003FA2B4806F000FA34
:103C90002A4806F0FDF92A4806F0FAF9294806F004
:103CA000F7F9294806F0F4F9284806F0F1F9284810
:103CB00006F0EEF9274806F0EBF9274A274928488D
:103CC00006F0E6F92749284806F0E2F9274806F009
:103CD000DFF904F12101264806F0DAF925492648E2
:103CE00006F0D6F907A803F063FC07A806F02AF946
:103CF0000146224806F0CCF9104806F0C9F90BB08D
:103D000030BD1F4806F0C4F9284614F0D5FCBCE7C6
:103D100050BB010866BB01087CBB010893BB0108CE
:103D2000A0860100AEBB01088AE50108C4BB0108FA
:103D3000F9BB01082CBC010888E501086ABC010830
:103D40009BBC0108AABC0108CCBC0108EFBC01085F
:103D500013BD010889E5010836BD01083CBD010815
:103D60004BBD01085ABD010861BD01086CBD0108C9
:103D70008CBD010897BD01089DBD0108B7BD0108B4
:103D800060BC01082DE9FF4100F15805284600F00C
:103D900083FB04240226DFF8A080013C14F0FF041A
:103DA00031D0A123012241462846009600F078FB3D
:103DB0004FF40043074600930422A123284602A99A
:103DC00000F09AFB002FE8D00028E6D09DF80830DC
:103DD000442B1FD19DF809306E2B1BD10DF10A0029
:103DE00006F045FA441CA4B221460DF109008DF8F5
:103DF000086006F061FA002303220093A0232846FE
:103E000002A900F04DFB284600F048FB204604B014
:103E1000BDE8F081442300248DF809306E2321464B
:103E20000DF10B008DF80A308DF8084006F044FAC9
:103E3000A02305220094E2E7DCBD010838B50D4659
:103E4000044611310BF078FFEB6E204623602B6F98
:103E5000636038BD30B50D469DB0044601466846E6
:103E6000FFF7ECFF694628460BF018FE04F111033A
:103E700021346B632C631DB030BD000030B50846A3
:103E80008DB014460F4B104A104911F0A9F90022C9
:103E90000F490A9207910F49069208910E4A0F495D
:103EA0000F4D09910494059204A901AC07C90B9523
:103EB00084E8070007AB00950FCB11F0A5FB0DB010
:103EC00030BD00BF5536000844B3010868B301088F
:103ED000B16C0008396C000800000808B136000811
:103EE0008538000810B50446FFF7BAFC2146BDE846
:103EF0001040FFF747BF0000024B186803689B683B
:103F0000184700BFA00D0020024B186803685B68CB
:103F1000184700BFA00D0020024B186803681B68FB
:103F2000184700BFA00D002037B5022405461346F0
:103F3000044A106802680094D4680A462946A047DB
:103F400003B030BDA00D002037B500240546134650
:103F5000044A106802680094D4680A462946A047BB
:103F600003B030BDA00D002037B54FF40044054626
:103F70001346054A10680268009414690A462946E7
:103F8000A04703B030BD00BFA00D00204FF47A73EE
:103F90005843B0FBF3F009F063BE00001FB58DF885
:103FA0000C1000218DF80D20054A034610680268A8
:103FB0000091D46803A90222A04704B010BD00BF3D
:103FC000A40D00200023F0B513701446022205460C
:103FD0000C4E85B030688DF80F1003680092DF68D2
:103FE00001222B460DF10F01B84748B14FF40042B2
:103FF00030682146036800921E6901222B46B047B3
:1040000005B0F0BDA40D0020024B186803689B6842
:10401000184700BFA40D0020024B186803685B68B6
:10402000184700BFA40D002010B5424C0AF012FF43
:1040300020460222002103F001F801222046114609
:1040400002F0FCFF20460122022102F0F7FF204689
:104050000222032102F0F2FF20460022042102F096
:10406000EDFF20460222082102F0E8FF204601224F
:10407000092102F0E3FF204601220A2102F0DEFFBF
:10408000204602220B2102F0D9FF02F08BFD002313
:1040900020461A460C2102F091FF204600220C21F6
:1040A00003F05CF82046002204F580640F2102F042
:1040B000C5FF20460122002102F0C0FF2046002259
:1040C000022102F0BBFF20460022032102F0B6FFCE
:1040D00020460222062102F0B1FF204600220821DC
:1040E00002F0ACFF20460022092102F0A7FF204683
:1040F00001220C2102F0A2FF204602220D2102F033
:104100009DFF204602220E2102F098FF2046022247
:104110000F2102F093FF002304F5806420461A4625
:104120000D2102F04BFF2046BDE8104000220D217A
:1041300003F014B80000024003F098BA1C4B00B51D
:104140001A6889B0D2075FBF1A4A106001221A604C
:10415000194B0493194B0593194B0393194B029375
:10416000194B0793194B069308AB13E903008DE82D
:10417000030002AB0FCB12F0E7F890B1144805F042
:1041800087FF00221348114602F058FF0F23022236
:104190000021104802F0F0FD09B05DF804EB12F0C8
:1041A0006DB86A210C4809B05DF804EB02F0E4B97F
:1041B0009C0D0020A40D00201940000809400008B3
:1041C000C53F00089D3F000891A000088D3F0008F2
:1041D000FCBD0108000002408AE50108002307B584
:1041E000ADF8043001238DF8063001980AF08EFDF9
:1041F00002F0D8FC03B05DF804EB0AF0D9BD000072
:10420000194B10B51A688CB0D2075FBF174A1060FF
:1042100001221A60164B0793164B0593164B069313
:10422000164B0893164B0993164B0A93164B0B9398
:104230000CAB13E907008DE8070005AB0FCB11F0BD
:10424000A5FF044601220F21104802F0F7FE3CB101
:104250000F4805F01DFF11F077FF20460CB010BD90
:104260000C4805F015FFF8E7980D0020A00D002080
:10427000693F0008493F0008293F0008193F00082E
:10428000093F0008F93E000891A000080000024024
:104290000DBE010840BE01082DE9F0479AB00BF0B1
:1042A00065F9DFF89CA0274C274FDFF8A08012ADFE
:1042B00050B9CDE91544CDE91387CDF848A0009455
:1042C00095E80F000BF06CF9214B00261393214B5E
:1042D0004FF001091293204B06A914931F4B284657
:1042E00015931F4BCDE91887CDE916340423CDE98A
:1042F00006368DF81D9006F0E7FB06F0D9FB06F0B8
:1043000021F8184ACDE9096611920322CDE90C443F
:104310000B9608928DF8269008AB02AC0FCBCDE936
:104320000F87CDF838A084E80F00DDE910018DE893
:1043300003000CAB0FCB0BF041FD1AB0BDE8F087CA
:104340005976000891A000089DA10008C9A10008A5
:1043500035ED0008FDEB00080DEB0008A5EA0008AC
:10436000B9EA0008E53E00082DE9F047044602F0EE
:10437000F7FA1E49054613F0C3FB13F087FD01460B
:104380001B4805F085FE4FF08041284613F056FD8E
:1043900048B30025DFF85C90DFF85080164F02F03C
:1043A000DFFA4946064613F05DFDA8B9414630469E
:1043B00013F0A6FB13F06AFD0146384605F068FECF
:1043C000236885F0010520462946DB6898474FF4AD
:1043D0007A7002F00FFCE2E723682046BDE8F04760
:1043E0000021DB681847BDE8F08700BF00007A4471
:1043F0005EBE01080000204070BE010808B5012023
:10440000084902F091FF0B20074902F08DFF0A20B6
:10441000064902F089FFBDE808400720044902F080
:1044200083BF00BFF9BD000899C10008B9BF0008EB
:1044300011C20008002310B50C461A460D2107488A
:1044400002F0BCFD14B1012C00D010BD2246BDE825
:1044500010400D21014802F081BE00BF000802405B
:10446000002310B50C461A460C21074802F0A6FDA1
:1044700014B1012C00D010BD2246BDE810400C2123
:10448000014802F06BBE00BF00000240014802F08C
:10449000D5BE00BFA086010002F0A0BE02F0BABEE9
:1044A0002DE9F041DDF818801E4608F00303032BC8
:1044B00007460C46154603D12F210E4802F05CF842
:1044C00018F0020F32462946204609D002F0F0FECD
:1044D00010B10120BDE8F081012300203B71F9E714
:1044E00018F0010F02D002F0F1FEF1E702F0D2FE67
:1044F000EEE700BF8AE501082DE9F041DDF81880FC
:10450000074618F0010F0C4615461E4603D04C21F5
:104510000E4802F031F818F0020F03D04F210B487B
:1045200002F02AF818F4004F32462946204609D0F6
:1045300002F0DAFE10B10120BDE8F0810123002075
:104540003B71F9E702F098FEF4E700BF8AE5010845
:10455000032108B5034802F00AFE003818BF012005
:1045600008BD00BF000402400A460248032102F0D1
:10457000F5BD00BF0004024008B581B1012303214D
:104580001A460A4802F01AFD0321084802F0DCFD31
:10459000BDE8084003220548114602F0EFBC0122A5
:1045A000BDE808400321014802F048BD0004024074
:1045B00003F052B81FB501A805F087FC01A803F06D
:1045C0002BF905B05DF804FB03F094B803F0ACB828
:1045D000084602F029BF7FB50023CDE90133ADF8CD
:1045E0000C3001238DF807308DF808306FF01D0373
:1045F0008DF809300723044601A88DF80A3005F02C
:1046000089FC236806461B6820460D46984786426B
:1046100075EB0103B4BF0120002004B070BD70B57C
:104620000646194610461C4615460BF003F87368FB
:1046300023B128462146BDE87040184770BD0000F0
:104640002DE9FF4714461D46804603F005F806464F
:104650000F46B4EB000A22462B4601A865EB010980
:1046600005F033FC3046394605F096FC29460646EF
:10467000204605F091FC49460446504605F0A2FC50
:10468000224603463146074805F002FD01A802F024
:104690007FFF20B152464B464046FFF7C0FF04B0B3
:1046A000BDE8F087CCBE0108704770477FB500F1C8
:1046B0000806054630460C4612F0D6FA60BB324872
:1046C00005F0E6FCA27C617C304805F0E1FC637CEF
:1046D0003BB16868002103681B689847022000F01E
:1046E0008FF8A37C3BB16868002103685B6898473A
:1046F000022000F0A3F861684E2918D04F2916D087
:10470000452914D01621224801F036FF1721214BEC
:10471000214A224813F0BCFD6421304612F090FA81
:104720000028CFD143211A4801F026FFCAE7A2682A
:10473000D31F022B14D8E368D2B20F2B19D00BDC95
:10474000052B16D00A2B13D03421114801F014FF89
:104750003521104B124ADCE7142BF5D1022308E077
:1047600024210B4801F008FF25210A4B0D4AD0E710
:104770000123A07C0290607C0190207C0090206846
:1047800003F0C6FA04B070BD18BF010831BF0108BC
:104790008AE5010840B401084EBF01087EBF010848
:1047A000F6BF0108BEBF010810B5044603F082FA47
:1047B00004F10800BDE8104012F059BA084603F0B1
:1047C0007BBB38B50C468D18AC4204D014F8010BF5
:1047D00003F072FBF8E738BD03F092BA084603F025
:1047E00099BB000010B50446044BC0E9003101211B
:1047F000083012F047FA204610BD00BF34C001084F
:10480000042817D8DFE800F00309100E1200002377
:1048100003211A46084802F0D1BB002203210648B2
:1048200002F00CBC0222F9E70122F7E7032102485B
:1048300002F02ABC704700BF00000240042817D8CD
:10484000DFE800F00309100E1200002302211A46CF
:10485000084802F0B3BB00220221064802F0EEBB7A
:104860000222F9E70122F7E70221024802F00CBC1C
:10487000704700BF0000024010B50446C06908B18F
:1048800005F08CFC206908B105F088FC606808B16F
:1048900005F084FC204610BD10B50446006808F001
:1048A0005BFB204610BD00001FB5536802931378D0
:1048B00001934B6800930B6842680178024805F049
:1048C000E7FB05B05DF804FB54C00108FE2307B503
:1048D0008DF80430054B01A91868002300681A46BA
:1048E00008F02CF803B05DF804FB00BFB40D002005
:1048F000814203D0CB21024801F03EBE704700BF89
:104900008AE5010870B51D467423C0E90031002313
:10491000044683600820164611F080FBC0E900655C
:10492000A060204670BD000037B504460D46006803
:104930006321FFF7DDFF00232846A16801AA019348
:1049400005F090F9019B1BB13821024801F014FEDB
:1049500003B030BD8AE50108F8B563230027C0E93C
:104960000031044687601A20154611F057FB0646B1
:104970001A22394613F0EEFE20462946A660FFF7BC
:10498000D3FF2046F8BD81647047C16470470000C2
:104990002DE9F843D0E90174884600264FF00C0950
:1049A0000A4BE41BA4105C43F5B2A5420BD209FBF1
:1049B00005734146586814F0DBFE01360028F3D138
:1049C0002846BDE8F8834FF0FF30FAE7ABAAAAAA61
:1049D0002DE9F843D0E90474884600264FF00C090D
:1049E0000A4BE41BA4105C43F5B2A5420BD209FBB1
:1049F00005734146586814F0BBFE01360028F3D118
:104A00002846BDE8F8834FF0FF30FAE7ABAAAAAA20
:104A1000F8B50E4649680446FFF7BAFFC0B2FF2852
:104A200003D07C21204801F0A7FDD4E901239B1A83
:104A3000B3F5BD6F03D97F211B4801F09DFDD4E97B
:104A40000153E0685A1B194902F10C071B1A921016
:104A50004A439B104B4301329A420DD83D44A56016
:104A6000D4E9013496E80700E31A04E907000F4887
:104A70009B1058430138F8BD384605F0A5FB0546A4
:104A800018B96921084801F077FDD4E901128A427A
:104A900003D02846521A13F043FE606805F07EFBEF
:104AA00065603D44E560DAE78AE50108ABAAAAAA99
:104AB0001FB56E23CDE90131002301A90393FFF750
:104AC000A7FF05B05DF804FBFF22F8B500230446FC
:104AD0000526002780F828204FF0FF356FF07F4231
:104AE000C0E90033C0E90233C0E90433C0E906334A
:104AF000C0E908334FF000410020C4E91467234E99
:104B0000C4E910523268C4E90C0112F00102C4E990
:104B10000E01C4E91233C4E91801A36513D10121C0
:104B20001B4D08462A60696007F02CFE286018B902
:104B30005121184801F020FD0123174A1749144854
:104B4000336012F0BDF8164B1A680AB9104A1A60A1
:104B500020461449FFF7ACFF134B14491870204648
:104B6000FFF7A6FF124B134918702046FFF7A0FF6E
:104B7000114B124918702046FFF79AFFFE22104B86
:104B80001870104B20461A70F8BD00BFB00D002001
:104B9000380E00208AE5010800000020994800082E
:104BA000B40D002072C00108BC0D00207AC00108BD
:104BB000BA0D002082C00108B80D002087C001088E
:104BC000BB0D0020B90D002010B5084C2368DB0791
:104BD00009D40748FFF778FF0123064A064904482D
:104BE000236012F06DF8024810BD00BFAC0D00202C
:104BF000D00D00200000002079480008F8B50E46CE
:104C000049680446FFF7E4FEC0B2FF2803D08721BD
:104C1000204801F0B1FCD4E904239B1AB3F5BD6F21
:104C200003D98A211B4801F0A7FCD4E90453A069E9
:104C30005A1B194902F10C071B1A92104A439B1088
:104C40004B4301329A420DD83D446561D4E90434A6
:104C500096E80700E31A04E907000F489B10584341
:104C60000138F8BD384605F0AFFA054618B9692194
:104C7000084801F081FCD4E904128A4203D0284696
:104C8000521A13F04DFD206905F088FA25613D4464
:104C9000A561DAE78AE50108ABAAAAAA38B5D0E986
:104CA00001239B1A074A9B105343CDB29D420446F1
:104CB00003D3A621044801F05FFC0C20636800FBCD
:104CC000053038BDABAAAAAA8AE5010838B5CCB22E
:104CD000114905460B6813F0010307D170200F4AF4
:104CE00010600F48C2E9010301230B60FF2C10D0B4
:104CF000D5E904239B1A0B4A9B1053439C4203D3D0
:104D0000B221094801F038FC0C21286901FB04009C
:104D100038BD0248FCE700BFA80D0020C00D0020F0
:104D20008FC00108ABAAAAAA8AE5010810B5D0E98C
:104D30000730C9B2D2B2834209D01C788C4204D168
:104D40005C78944201D1987810BD0333F3E74FF0BB
:104D5000FF30F9E72DE9F0410D460A78D0E9041358
:104D60005B1A49499B104B439A42044603D3932153
:104D7000464801F001FCD4E901135B1A42499B103B
:104D80004B436A789A4203D39421404801F0F4FBE4
:104D9000D4E904135B1A3C499B104B43AA789A420E
:104DA00005D3FE2A03D09521384801F0E5FB2F7882
:104DB000204639466A78FFF7B9FFC3B2FF2B064693
:104DC00029D039462046FFF781FF697807462046FB
:104DD000FFF764FF314680462046FFF777FF4146E4
:104DE00002463846FFF760FD29782046FFF76EFF40
:104DF000697806462046FFF751FFA9780746204606
:104E0000FFF764FF394602463046FFF74DFD9C210F
:104E10001E4801F0B1FBD4E907239B1AB3F5BD7F0F
:104E200003D99F21194801F0A7FBD4E9076316496C
:104E3000606A9A1BD71C1B1A4A434B4301329A42A1
:104E40000AD83E4426622A88236A23F8032CAA78CB
:104E500003F8012CBDE8F081384605F0B5F90646A7
:104E600018B96921094801F087FBD4E907128A4281
:104E700003D03046521A13F053FCE06905F08EF966
:104E8000E6613E446662DDE7ABAAAAAA8AE50108AC
:104E900038B58168006814461D4605F045FA01469C
:104EA000001945EBE17138BD2DE9F0470F680E465A
:104EB000722F9046994633D0742F08D0632F1ED09E
:104EC00000254FF0004428462146BDE8F0873946CA
:104ED0003846FFF70DFDB368D3E90054B4F1004F35
:104EE00008BF002DEFD039463068FFF701FDB368E9
:104EF000D3E9005418EB050549EB0404E3E7394610
:104F00003846FFF7F5FC42464B46B06804F06CFFAC
:104F10000C1E0546D7DADD21074801F02DFBD2E74C
:104F200038463946FFF7E4FC42464B46B068BDE8D8
:104F3000F047FFF7ADBF00BF8AE501082DE9F84350
:104F40000F4606460024FFB2FFF7C0FED6E9075918
:104F5000A94516D02B78BB4211D169783046FFF7AE
:104F60009DFE01688046692909D10846FFF7C0FC0B
:104F7000D8F808301B6803B198470134E4B2033510
:104F8000E6E72046BDE8F8832DE9F74306460F46DD
:104F90000025FFF79BFEF469336A033403F103092C
:104FA000FFB24C4520D014F8013C34F8032C8DF8A6
:104FB000063014F8033CADF804209F4212D19DF84E
:104FC00005103046FFF76AFE01688046692909D15D
:104FD0000846FFF78DFCD8F808305B6803B19847A6
:104FE0000135EDB20334DCE7284603B0BDE8F083B9
:104FF000836C73B504460D46164623B94FF48E7183
:105000000B4801F0B9FA23462A46CDE90064094964
:10501000094808F095FA012807D04FF49171044827
:1050200002B0BDE8704001F0A7BA02B070BD00BF89
:105030008AE501089DC001080D57000838B590F8B1
:1050400047300446032B0D4604D940F2351106487B
:1050500001F092FA94F84700431C84F84730044466
:1050600084F8425038BD00BF8AE5010810B590F8B9
:105070004730044623B94FF49D71064801F07CFA8D
:1050800094F847000138C0B284F84700044494F80B
:10509000420010BD8AE50108CBB2FE2B10B50446D4
:1050A0000AD0FFF713FE03686D2B05D1017A204665
:1050B000BDE81040FFF70ABE10BD00002DE9F8431F
:1050C00004460026114FD4E904239B1A9B107B430E
:1050D0005FFA86F8984516D241462046FFF7DCFF76
:1050E000D4E90759A9450CD02B78434507D16978F5
:1050F0002046FFF7D3FD2046A978FFF7CDFF033503
:10510000F0E70136DFE7BDE8F88300BFABAAAAAA43
:1051100070B56FF04106044600F14205361A94F866
:10512000472073199A4205DD204615F8011BFFF749
:10513000CDFDF4E770BD2DE9F74F4FF00009DDE933
:105140000CBA04468846C0E90899D8E907734FF0BD
:1051500000410020C4E90001C4E90201C4E90401DE
:10516000C4E90601FF210093D3B284F82010019313
:10517000009BD4E900569F4222D03A78019B9A4284
:105180001CD179784046FFF789FD5A4601465346BF
:105190004046FFF789FEB1F1004F08BF48450DD0EA
:1051A000B6F1004F08BF4D4503D0A84271EB06038E
:1051B00004DA7A78C4E9000184F820200337D7E7BD
:1051C000B6F1004F08BF002D05D0B5EB0B0566EB1F
:1051D0000A03C4E90453204603B0BDE8F08F70B55C
:1051E00015461C46FFF75AFD866874210068FFF7D4
:1051F0007FFBC6E9005470BD836C10B5044623B92B
:1052000040F29D21024801F0B7F9A06C10BD00BF2B
:105210008AE50108036870B504460D4616461BB9B9
:105220002921064801F0A8F932462946206807F0EE
:1052300029FC431E5842584170BD00BF8AE5010851
:1052400013B5FF24074B0A46186801A98DF80440DE
:10525000FFF7E0FF18B19DF8040002B010BD204632
:10526000FBE700BFB40D0020F8B50D460B4B896974
:10527000064659434FF47A73B1FBF3F1FFF7E0FFB1
:105280000446C7B2B06C03681B689847FF2FC6E995
:105290000E0114BF204695F82000F8BD40420F00D3
:1052A00038B5C36C04460D461BB9BDE83840FFF75E
:1052B000DBBF806C174903685B699847A06C036883
:1052C000DB689847D5E9020104F066FE0146124802
:1052D00004F0DEFEA06C03689968D5E902238847D4
:1052E000A06C03681B699847E36C9847A06C03683F
:1052F000DB689847A06C03681B689847C4E90E01F7
:1053000000212046FFF79CFFC0B2FE2808BF95F899
:10531000200038BDCD480008A8C00108F8B5D1E983
:105320000663B3F1004F08BF002E05460C4608D1B6
:105330001AB1BDE8F840FFF797BFBDE8F840FFF7A6
:10534000AFBF012E73F1000702DA91F82000F8BD1B
:1053500092B121462846FFF787FF94F82030C0B26B
:105360008342F4D1D5E90E62D4E900138E4272EB88
:105370000303B8BFFF20EAE7D0E91472BE429341AD
:10538000E7DBFFF78DFFE8E72DE9F0478CB0044637
:105390000D46FFF79BFC03680646702B04D04FF4C4
:1053A000A071694801F0E8F8A06C03681B68984791
:1053B0002A46C4E90C01CDE90001214602A8FFF705
:1053C000BAFE29462046FFF7B9FD9DF8283007466A
:1053D000FF2B05D120B940F24B115B4801F0CCF80E
:1053E000D4E90C0104F0D8FD0146584804F050FE01
:1053F0003946574804F04CFE9DF82810FF297CD10F
:1054000000224FF00043CDE90623DDE90223CDE978
:105410000423DDE90623CDE90823A36D13B39847E0
:10542000DDE90223D4E91801B3F1004F08BF002AD7
:1054300009D0069B10F10B0741F100029F42079B28
:1054400072EB03030EDAD4E90C321B1842EB0102B3
:10545000CDE90801CDE9043204F0B4FD01463D4830
:1054600004F016FE4FF00009DFF8EC80394F2046BB
:10547000327A02A9FFF752FFA36D824603B1984723
:105480005FFA8AF3FF2B57D1DDE90232D4E90E012E
:10549000181A62EB0101CDE90432CDE90601CDE92C
:1054A000080104F08FFD0146404604F0F1FDA36DB4
:1054B000002BDCD0DDE90223D4E91801B3F1004F61
:1054C00008BF4A4509D0069B10F10B0C41F10002C0
:1054D0009C45079B72EB0303C9DAD4E90E321B1813
:1054E00041EB0202CDE90801CDE9043204F06AFD86
:1054F0000146384604F0CCFDB9E72046FFF7CEFB65
:10550000D0E90078DDE9020104F046FD4246034699
:105510003946124804F0BCFDD4E90C3202980399D4
:10552000C01A61EB0201CDE9060104F04BFD014612
:105530000B4804F0ADFD68E729462046FFF724FD3F
:1055400050460CB0BDE8F0878AE50108BBC00108F1
:10555000DAC0010837C101084FC10108F5C00108D0
:1055600019C1010870B504460D46FFF7AFFB03688B
:105570006D2B0FD0702B07D0836894F8411094F8EE
:105580004000BDE87040184729462046BDE87040FD
:10559000FFF7FABE40F22F11024800F0EDFF4FF086
:1055A000FF3070BD8AE501082DE9F04790F82830FA
:1055B0000446FF2B04D14FF4E5714D4800F0DCFFA9
:1055C00094F828102046FFF781FB4268017849488B
:1055D00004F05EFD94F82830DFF81C8184F8463032
:1055E00094F846102046FFF771FB036805466D2BC3
:1055F000204694F846100BD1FFF720FD297A20466B
:1056000084F84610FFF762FB2046FFF781FDE7E7CD
:10561000FFF7A8FFC3B2FF2B07460BD140F2DF1103
:10562000334800F0A9FF40F2DF11344B344A3548CB
:1056300012F02EFE94F84650024629462046FFF707
:1056400075FBC6B2FF2E14D139462046FFF726FB64
:1056500041682D4804F01CFD4FF4F371244800F01C
:105660008BFF4FF4F371254B254AE0E72046FFF707
:105670004FFDFE2E294620461CD1FFF7F7FC0546BC
:1056800001462046FFF722FB3A4629462046FFF70F
:105690004DFBC6B2FF2EE9D139462046FFF7FEFA90
:1056A0004FF4F971124800F067FF4FF4F971134B92
:1056B000134ABCE7FFF70AFB394605462046FFF7C9
:1056C000EDFA314681462046FFF700FB8246404610
:1056D00004F0DEFC524649462846FFF7E5F894F808
:1056E000463084F8417084F8403084F8466077E7AB
:1056F0008AE5010877C1010804C2010840B4010825
:1057000095C10108BAC10108FCC1010808B504F03F
:1057100023FEFFF759FAFFF747FF0000FF23054A72
:105720001370054A1370054A1370054A1370054A31
:1057300013707047BC0D0020BA0D0020B80D00207A
:10574000BB0D0020B90D002010B50446006807F01D
:1057500003FC204610BD000073B50AF071FC4FF643
:10576000FF71334A334D13888B421CBF01331380C2
:10577000FFF72AFAFFF740FD03681B6898476E7829
:10578000DEB92D4B1C89C4B12C4AD2E90032B2F1EA
:10579000004F08BFB3420ED0834272EB01060CDA11
:1057A000274EC31A06FB04F461EB0202E617A3427C
:1057B00072EB060301DB01236B700023ADF80430AC
:1057C0008DF806306B782BB101238DF804301B4B1C
:1057D000C3E900012A781B4B8AB101228DF805200C
:1057E0001A70194A19491A48019B127809780068F9
:1057F0000AF092FCD0B1174B187802B070BD1A7045
:105800000D4B9B89002BECD04AF6C0025343124C3F
:10581000DD17D4E90024801A61EB0401984271EB92
:105820000503A4BF01238DF80530DAE70B4BE3E74E
:10583000820E0020600E00206C0E0020400200202E
:1058400080510100690E0020630E0020620E0020CE
:105850005C0E0020B80D002030020020BA0D0020A0
:10586000104B1B8913B9104B1878704700220F4B4F
:10587000D3E90013B3F1004F08BF9142F3D10C49B3
:105880000B780133DBB2012B0B70ECD8094B1A708B
:10589000094B1A70094B1A60094B1A7001225A7091
:1058A000084BE1E76C0E0020B80D00203802002004
:1058B000940E0020630E0020620E00205C0E00207B
:1058C000600E0020BB0D00201FB57023CDE9013113
:1058D000002301A90393FFF791F905B05DF804FBDC
:1058E0002DE9F04F4B4B04461A7885B0002A40F062
:1058F0008E80012648491E70FFF7DAF8474B484969
:1059000018702046FFF7D4F8DFF818A146498AF846
:1059100000002046FFF7CCF8DFF810910A220023A0
:10592000434989F8000001A8FEF7ECFF01A92046D1
:10593000FFF76EF8DFF8FC803F4988F8000020464A
:10594000FFF7B6F83D4B3E4918702046FFF7B0F818
:105950003C4B3D4918702046FFF7AAF83B4B3C49A9
:1059600018702046FFF7A4F83A4B3B4A18703B49A1
:105970002046FBF70EF8DFF8E8B03A4A3A498BF8D0
:1059800000002046FBF705F8384905462046FFF79A
:105990009BFF70230193364B074601A92046CDE9B2
:1059A0000236FFF72BF90646324A2B46204612787C
:1059B0009BF80010FAF7F8FF3B46294620469AF874
:1059C0000020FAF7F1FF33462946204699F80020D7
:1059D000FAF7EAFF2B463946204698F80020FAF7F6
:1059E000E3FF2B463146204698F80020FAF7DCFF0B
:1059F000214A2B46294620461278FAF7D5FF1F4B3D
:105A00001F4A294620461B781278FAF7CDFF05B0C9
:105A1000BDE8F08F950E002014C20108640E00202E
:105A20001EC20108680E002029C20108480E00208D
:105A300035C20108490E002042C20108810E002033
:105A400050C20108800E00205CC20108840E0020B4
:105A500069C20108850E00205957000877C2010865
:105A6000660E00206161000881C2010895C201082C
:105A7000A8C20108B80D0020BB0D0020B90D002000
:105A8000BC0D002030B5044685B00D46FFF728FF59
:105A90006D22064B20461B7801A9CDE901258DF822
:105AA0000C30FFF7ABF805B030BD00BF660E00202C
:105AB0002DE9F84F434B04461A68434D12F0010F8D
:105AC00079D1FF222A7001221A602046FFF708FFD1
:105AD00020463E4A3E49FAF75CFF3E4A28703E495E
:105AE0002046FAF756FF3D4F3D4A38703D49204663
:105AF000FAF74FFF3C4E3D4930702046FFF7C2FF9A
:105B00003B4980462046FFF7DFFE3A498246204661
:105B1000FFF7DAFE8146384A20463B78297812782A
:105B2000FAF742FF354ADFF8D8B0204633782978B3
:105B30001278FAF739FF204633789BF8002039783D
:105B4000FAF732FF20462B789BF800203178FAF7DD
:105B50002BFF2C4A5346204639781278FAF724FF57
:105B6000294920463B780A785146FAF71DFF274A13
:105B70004B46204639781278FAF716FF224920461C
:105B80003B780A784946FAF70FFF1C4A43462046FD
:105B900031781278FAF708FF4146204633789BF8AF
:105BA0000020FAF701FF1A4A20462B781278317844
:105BB000FAF7FAFE02E02B78FF2B86D02878BDE8B2
:105BC000F88F00BF440E0020970E0020F55E0008FD
:105BD000BCC20108355C0008C6C20108650E002081
:105BE00061580008D0C20108670E0020DAC201081F
:105BF000E6C20108F4C20108640E0020BB0D0020BB
:105C0000BC0D0020680E0020490E0020BA0D0020B7
:105C1000B80D002070B50C460546FEF7D5FF0449C7
:105C20002A462346BDE870400978FFF7D8BA00BF7E
:105C3000490E002070B5484E3368013333600AF0D6
:105C4000FFF90AF02BFA44F620600AF00FFA4178C7
:105C50000446042908D0414804F01AFA204604F00A
:105C60009DFA0120002147E00578446804F096FA87
:105C7000012D4DD133683A4C042B0BD90FF05AFB50
:105C800003783BB1A36803B1984740F28B113548C4
:105C900000F072FC23690BB10020984734681E2184
:105CA000013CE4B21E2C28BF1E24A4F12005C4F13F
:105CB000200321FA03F301FA05F51D4347F281039E
:105CC00001FA04F49C4275F1000319D2B4F5616F36
:105CD00075F1000317D2B4F5167F75F1000315DADC
:105CE0003C2C75F1000300DA0A21002004F01CFBB3
:105CF0000146001945EBE171FFF78CFF1A4B0EE0EE
:105D00004FF4E14400254FF41671EEE73C21ECE737
:105D1000032D06D120460021FFF77CFF134B187896
:105D200070BD9DB935600AF045F9FEF74DFFFFF7EC
:105D300063FA03681B6898470D4BC3E90001084BE1
:105D40001B690BB1012098470A4BE8E70A4829462E
:105D500004F09EF90A2085E7900E002003C3010895
:105D6000980E00208AE50108BA0D0020680E002078
:105D700030020020BC0D002024C30108054B187020
:105D8000054B1A700022054B1960054B1A705A70AA
:105D9000704700BF630E0020620E00205C0E0020E2
:105DA000600E002008B50AF067FAC0B2F22828BFDA
:105DB000F22008BD002337B54FF47A7201930B4BE4
:105DC00002FB00F41D68B4FBF2F42B681BB9292117
:105DD000074800F0D1FB2246286801A906F052FED0
:105DE000012814BF0020019803B030BD4C0E0020E4
:105DF0008AE50108022818BF00200AF035BB000020
:105E0000F0B5304B05461E7885B0002E57D10122E3
:105E10008DF80F601A7009F077FC07230C222A4CCA
:105E2000CDE9003228460DF10F022849231D0EF05E
:105E300059FF0E23264928464FF47A776371A371E0
:105E400026610EF013FF2349607004F10803284611
:105E50000DF10F02CDE900670EF064FF42F21073FE
:105E60000DF10F022846CDE900631B4904F10A0336
:105E70000EF058FF194928460EF0F8FE04F10C0305
:105E80001749A0700DF10F022846CDE900670EF00A
:105E900049FF284613490EF0E9FE9DF80F30E070E7
:105EA00053B1114804F0F4F8104B1B6803B1984744
:105EB00060210F4800F060FB2069FFF79BFF05B0F1
:105EC000F0BD00BF960E00206C0E002049C30108F3
:105ED0004CC3010850C3010859C3010862E401081A
:105EE00062C301086DC3010872C30108980E002047
:105EF0008AE5010870B5294BC0B21B78984206D1DB
:105F00000FF018FA0EF0DEFE254B187870BD254C08
:105F10000FF010FAFFF774FF94F905000BF0FCFF87
:105F20000AF0BEF920790BF0C6FF0AF0AFF91E4E59
:105F3000A0790AF0BDF960780AF090FA326812F0A0
:105F4000010213D10421194D08462A60696006F048
:105F500019FC286018B95121154800F00DFB0123E8
:105F6000144A15491148336010F0AAFE134B1A6801
:105F70000AB90E4A1A60FEF727FEFFF73DF90368DB
:105F80001B68984701220E4BC3E900010D4B5A7262
:105F9000E3780BB10C4BB8E70C4BB6E7670E00206B
:105FA000BC0D00206C0E0020400E0020880E00204A
:105FB0008AE5010800000020495700084C0E002027
:105FC00030020020500E0020640E0020BB0D002087
:105FD000034B93F82F30022B0CBF02200020704798
:105FE000D0020020F8B51D4600234171BDF81810FD
:105FF000044617460360C18002B115B923712046DB
:10600000F8BD2846064910F025F8064610B920715B
:106010002660F4E72A46394612F074FB2571F7E74B
:1060200074ED010810B50446006808B110F014F8CA
:10603000204610BD7FB5304E0446336823B940F288
:10604000C1112E4800F098FA002C52D000222C4B9F
:106050001A80D4E91C23134317D02A4B1D6807F07C
:10606000A7FC01462848A847FEF7AEFDFFF7C4F895
:1060700003685968D4E91C238847D4E91C232349C1
:10608000C1E900232249C1E90023FEF79DFDFFF786
:10609000B3F803681B6898471E4B1F4AC3E9000109
:1060A000237AC3F3C0031370637F13B3237F03B357
:1060B00008201A490FF0C4FF054630B163890093E8
:1060C000237FA26E617FFFF78DFF03958DB10023C3
:1060D00030681A46006803A906F078FB012808D04A
:1060E000039C34B12046FFF79DFF082120460FF0A6
:1060F000B5FF04B070BD00BF4C0E00208AE501085A
:10610000820E0020D002002085C301083802002042
:106110004002002030020020860E002074ED0108AD
:1061200038B542F2107009F0A1FF0446A0B105781D
:10613000032D03D100214068FFF76CFDD4F8A000C7
:10614000FFF778FF237A13B10022044B1A70204620
:106150000BF0A6FC284638BD0125FBE7690E0020A0
:10616000002310B5114C84F8343009F047FF08B112
:1061700009F066FFFFF7D4FF012809D903280AD0E8
:106180000B484FF42C7100F0F7F94FF0FF3001E0AD
:10619000084B187810BDFFF71BFF022809BF012329
:1061A000054B84F83430054BF3E700BFD0020020E4
:1061B0008AE50108BC0D0020680E0020480E002072
:1061C000FF2300210D4A13700D4A13700D4A1370FE
:1061D0000D4A13700D4A13700D4A13700D4A137057
:1061E0000D4A13700D4A13700D4A13700D4A137047
:1061F0000D4AC2E900111372704700BF660E0020FD
:10620000650E0020670E0020810E0020800E002009
:10621000850E0020840E0020640E0020680E0020F1
:10622000480E0020490E0020500E0020034AC0E90D
:106230000021002202818272704700BF4849F8F9AC
:10624000437A10B504461BB92121094800F094F99E
:10625000207A08B9002010BDA37A002BFBD060681B
:1062600003681B6898470028F4D00023A372F2E764
:106270008AE5010830B5044685B08DF80F10FFF7A8
:10628000DFFF9DF80F30606803F00F038DF80F30CB
:1062900003685B68984768B1002260680DF10F01E0
:1062A00003680092DD6801222378A84760680368CC
:1062B0009B68984705B030BD30B50446002585B0D1
:1062C000FFF7BEFF60688DF80F5003685B68984762
:1062D00060B160680122036800951D690DF10F012E
:1062E0006378A847606803689B6898479DF80F002B
:1062F00000F00F0005B030BD7FB505460E46FFF734
:106300009FFF686803685B689847044620B30222D1
:106310006B7868688DF80C30EB7803A98DF80D3038
:1063200003680092DC680122AB78A04704466868E5
:1063300014B90123AB720CE04FF4004203680092E1
:106340001C6903223146AB78A04704466868002CDC
:10635000EFD003689B689847204604B070BD13B522
:1063600001A90446FFF7C8FF70B19DF80530082B5E
:1063700007D19DF804209DF80630134301D1012375
:106380002372207A02B010BD2072FAE7002310B504
:10639000038183720446406803681B68984730B1E4
:1063A000012320466372BDE81040FFF7D8BF10BD3F
:1063B00070B5164605460C46FFF77EFF3EB140EA33
:1063C00004012846BDE87040C9B2FFF753BF20EA78
:1063D0000401F6E72DE9F04340488BB003F058FE86
:1063E00007F0F4FA2425079007993D4803F050FE82
:1063F0000798684303F0E8FE04463A4803F048FE75
:106400008CB1204607990DEB050207F05BFE0023D7
:10641000354E364F07900893089A079B9A421DD332
:10642000204603F0BBFE06F0CDF8044606F0D8F88F
:10643000214602462E4803F02BFE2E4B2E4819888B
:106440009A888B1A03F024FE2C4B1B6803B19847E3
:106450002B480BB0BDE8F04303F01ABE089B05FBC8
:1064600003431B7B042B98BFF25C099B88BF3F2230
:10647000642B83BF6420B3FBF0F30899002382BF31
:1064800005FB01418969B1FBF3F308990898DDF830
:1064900020C0DDF820E0DDF82080DDF8209005FB4D
:1064A000004005FB0949D9F81C9005FB0141CDE9E5
:1064B000033905FB08439B69029305FB0E439B6868
:1064C000019305FB0C431B8C009303694968384614
:1064D00003F0DEFD089B013308939DE792C301089A
:1064E0009EC30108A9C301089AC40108DEC30108BC
:1064F000DCB501089410002010C40108240F00200E
:1065000072B90108014B1860704700BF400F0020AE
:1065100073B5134E054632780C46124B1AB91A78E9
:106520000AB172B6FEE7012200211A700E486422F9
:1065300012F010F9234664210C4A0B48009513F021
:1065400047F80B4B1B6803B198470124064D2846BA
:1065500003F0E2FD72B6074B3470013BFDD1F6E764
:106560001D0F0020B10E0020B20E002034C401081F
:10657000400F0020FFFF0F00F7B5184E0546327898
:106580000C46174B1AB91A780AB172B6FEE7012207
:1065900000211A701348642212F0DCF823466421AB
:1065A000114A1048009513F013F8104B1B680BB1FB
:1065B0000C4898470E4B1B6803B198470124094DBE
:1065C0000C4F284603F0A8FD384603F0A5FD72B62F
:1065D000094B347000BF013BFCD1F2E71C0F0020D7
:1065E000B00E0020B20E00205CC40108AC0E0020EA
:1065F000400F00206BC40108FFFF0F00F8B5DFF863
:1066000070C003681B4FCCF8003043681A4E3B60E3
:1066100083681A4D3360C36819492B600369194AAE
:106620000B604369184C13608369C0692360174B82
:106630001860DCF80000386830682868144E096873
:10664000144D126822681B6864220021284612F04B
:1066500081F8236832466421284612F0B9FF2846A3
:1066600003F05AFD0C4B00BF013BFCD1ECE700BF2F
:106670002C0F0020300F0020380F00203C0F00208E
:10668000340F0020180F0020200F0020280F0020BA
:1066900087C40108B20E0020FFFF0F00074B1B68E4
:1066A00003B198471EF0040F0CBFEFF30880EFF31F
:1066B00009808169004A1047FD650008400F0020ED
:1066C000002103E00A4B5B584350043109480A4B50
:1066D00042189A42F6D3094A02E0002342F8043BEA
:1066E000074B9A42F9D300F00DF8FBF72DF87047ED
:1066F0000CF2010800000020100600201006002007
:10670000741E0020314B82B01A6842F480721A6005
:1067100099682F4A0A409A601A6822F0885222F03B
:1067200001121A601A6822F480221A609A6822F410
:106730007D029A600022DA6001921B6813F40073F4
:1067400018BF01230193019B012B37D14FF48051D6
:10675000204B1A68A3F5806322F00102C3F80024DD
:10676000D3F8002422F00202C3F80024D3F8002456
:1067700022F00402C3F800245A6A42F080525A629E
:10678000154A11605168C906FCD49A689A609A68E3
:106790009A609A689A605A6822F460425A605A680D
:1067A00042F440425A609A6822F003029A609A6862
:1067B0009A60064A936813F00C0FFBD14FF0006209
:1067C000064B9A60064ADA6002B070470038024011
:1067D0000CC0FF88003C02400070004000ED00E06B
:1067E0000003FA0570B5064688B02D4801F0B8FCE4
:1067F0002C4B1A680092009A91073AD501214FF468
:10680000007001F0F9FE012001F0F8FC264A5368FF
:1068100043F400335360A2F5374253681B07FCD59D
:106820000024012502A801F0D5FC1D4802A9069408
:106830008DF81C50ADF80C4001F0A6FC2A4606234A
:106840003146174801F0E6FC2946154801F0CDFC19
:106850000221134801F06EFD114801F05DFD134D5A
:1068600001940F4C0221204601F05EFD58B108B0A2
:1068700070BD1A6842F001021A60009A9207BDD4F6
:106880001A680092F9E7019B01330193019BB3F56C
:10689000805FE7DB38212846FFF76EFEE2E700BFA6
:1068A0000024014000380240002701408AE5010829
:1068B00008B5002001F0A2FC0021074801F095FC7A
:1068C00000214FF4007001F097FE044A136823F092
:1068D0000103136008BD00BF0024014000380240DE
:1068E00013B5072301460122114801F093FC022150
:1068F0000F4801F01FFD0E4801F00EFD00230D4C66
:10690000019302210A4801F00FFD28B1084802B0A6
:10691000BDE8104001F005BD019B01330193019BCF
:10692000B3F5805FEDDB4C212046FFF725FEE8E75D
:10693000002401408AE5010870B506460825FFF7E6
:1069400051FF00243046FFF7CBFF013D0444F9D14D
:10695000FFF7AEFFC4F3CF0070BD000000000000E1
:1069600008B51120FFF7E8FF11F072F8014608485A
:1069700011F07AF910F054FC03A3D3E9002310F0CE
:10698000A7FC10F05FFF08BD2FDD24068195F33FC3
:1069900000F07F450F4A536A43F080535362A2F5DB
:1069A000E4325368D906FCD41368022823F4C05398
:1069B00006D143F4C05313605368DB06FCD4704720
:1069C000012802D143F48053F5E70028F3D143F4C2
:1069D0000063F0E70038024010B50C4B5A68D2064D
:1069E000FCD41C6814F4C05F0BD114F480500AD19D
:1069F00014F4006404D106482A21FFF7BDFD2046A7
:106A000010BD0220FCE70120FAE700BF0070004043
:106A10008AE5010838B50546012001F09BFC022DEE
:106A200001BF154A136843F001031360134B1A6842
:106A300042F480321A601A689203FCD542F69052F2
:106A40009A6099689142FCD19A6842F002029A6079
:106A50000A4A946814F00804FBD14FF480331360A1
:106A6000074B084A28461A60FFF794FF2046BDE806
:106A7000384001F063BC00BF003C024000380240D7
:106A80004802002000093D0038B50546012001F00C
:106A900061FC022D01BF144A136843F00103136027
:106AA000124B1A6842F480721A601A689205FCD57B
:106AB0005A6822F4604242F440425A6000229A60CE
:106AC0000A4A946814F00C04FBD14FF480731360ED
:106AD000074B084A28461A60FFF75CFF2046BDE8CE
:106AE000384001F02BBC00BF003C0240003802409F
:106AF00048020020D0FE3F000C4B5A6B900513D487
:106B00005A6A42F080525A62094A116841F480710F
:106B10001160596B41F480715963596B8905FCD53B
:106B2000136823F480731360704700BF003802407D
:106B300000700040054B5A6B910706D45A6B42F027
:106B400001025A635A6B9207FCD570470038024025
:106B5000094B5A6A42F020025A629A6942F02002B6
:106B60009A619A6922F020029A610022A3F5093302
:106B70001A801A855A62704700380240152102387F
:106B8000002248430121064B1A85D86299825A6235
:106B90001A8219801A8AD207FCD500221A807047FF
:106BA00000140040002349F6FE7282B00193019B5D
:106BB000934201DD02B07047019B01330193F6E778
:106BC000002340F6FE7282B00193019B934201DDE7
:106BD00002B07047019B01330193F6E7002382B0B6
:106BE0000193019BB3F5CC7F01DD02B07047019B9F
:106BF0000133F5E7D0B1012801D1FFF7EFBF0C4B0E
:106C000000211A684FF47A73B2FBF3F2094B013A90
:106C100092B21A8501220138D8629A825962198289
:106C20001A801A8AD207FCD500221A80704700BF4A
:106C3000480200200014004000F1774303F5780378
:106C4000B3F5804F2DE9F04105460C4616462DD28E
:106C500002F1F73303F608030344B3F5804F25D25E
:106C6000FFF7BAFE804610B10020FFF793FE01F057
:106C700089FB012726442D1BA6420AD101F092FB75
:106C8000B8F1000F02D04046FFF784FE3846BDE859
:106C9000F08141F6027001F08DFB281914F8011BF8
:106CA00001F0E4FB042818BF0027E5E70027EDE723
:106CB00010B50446084604F1774101F57801B1F5B5
:106CC000804F0CD202F1F73303F608032344B3F5E7
:106CD000804F04D2214611F015FD012010BD002087
:106CE000FCE7000008B5114B984215D003F580630E
:106CF000984213D003F58063984211D003F5806366
:106D000098420FD003F5006398420DD01421084B30
:106D1000084A094811F0BCFA002008BD0120FCE730
:106D20000220FAE70320F8E70520F6E7000002401A
:106D30009FC4010819C50108B8C401080F2808B587
:106D400005D93B21084B094A094811F0A1FA012253
:106D5000084B02FA00F0596821EA000159601A68EC
:106D600022EA0000186008BD01C5010844C50108F9
:106D7000B8C40108000401400F292DE9F84F8146ED
:106D80000C4692461E4605D954215A4B5A4A5B4836
:106D900011F07EFA4FF00108594F00F0B9F87B6806
:106DA00008FA04F823EA08037B603B68554A23EAA3
:106DB00008033B60136A032C43F00103524D136236
:106DC00030D80F22AB684FEA840B02FA0BF223EAA9
:106DD0000203AB604846FFF785FFAB6800FA0BF093
:106DE0001843A8601AF0020F18BFBB684FEA0612DA
:106DF0001CBF43EA0803BB601AF0040F18BFFB680E
:106E0000D2B21CBF43EA0803FB603B6843EA0803B5
:106E10003B603E4B002C44D183F8062340221A608D
:106E2000BDE8F88F072C12D80F22201FEB684FEA1D
:106E3000800B02FA0BF223EA0203EB604846FFF7ED
:106E400051FFEB6800FA0BF01843E860CAE70B2C1F
:106E500013D80F22A4F108002B694FEA800B02FA25
:106E60000BF223EA02032B614846FFF73BFF2B6935
:106E700000FA0BF018432861B4E70F22A4F10C00CC
:106E80006B694FEA800B02FA0BF223EA02036B6193
:106E90004846FFF727FF6B6900FA0BF0184368615B
:106EA000A0E7012C03D183F807238022B7E7022C47
:106EB00004D183F808234FF48072B0E7032C04D187
:106EC00083F809234FF40072A9E7042C04D183F856
:106ED0000A234FF48062A2E7092C04D883F8172311
:106EE0004FF400029BE783F828234FF480725A6026
:106EF00096E700BF0DC5010823C50108B8C4010805
:106F000000040140003802400000014000E100E0C0
:106F1000144B984205D1144AD36943F00103D3615D
:106F20007047124B984204D10F4AD36943F00203D1
:106F3000F5E70F4B984204D10B4AD36943F00403A1
:106F4000EDE70C4B984204D1074AD36943F008039C
:106F5000E5E7094B9842E3D1034AD36943F02003A4
:106F6000DDE700BF0000024000380240000402409C
:106F700000080240000C02400014024003234900B4
:106F800010B584688B4024EA030484600124022A3B
:106F900004FA01F407D0032A0DD0012A07D183682F
:106FA0002343836003E083688A401A4382608368D6
:106FB0001C43846010BD82681343F2E70F292DE95A
:106FC000F0410446884615461F4603D94B211A480E
:106FD000FFF7D2FA2046FFF79BFF03230120216829
:106FE0004FEA480293406FEA030C21EA030323604F
:106FF000236800FA02F63343236000FA08F1A388FD
:1070000009B267B1194389B2A180E368012D0CEA86
:107010000303E36007D0022D09D0BDE8F0819BB2E5
:1070200023EA0101F0E7E3681E43E660F5E7E36861
:1070300095401D43E560F0E78AE501080F2970B52A
:1070400005460C46164603D96B210E48FFF794FA05
:107050002846FFF75DFF0323E86861008B40DA43B1
:10706000012E20EA0303EB6005D0022E03D02B682B
:1070700013402B6070BDEB6806FA01F11943E9601B
:10708000F5E700BF8AE501080F2910B505D9812170
:10709000074B084A084811F0FBF8FFF739FF0323B4
:1070A0000268490003FA01F11143016010BD00BFFD
:1070B00001C50108D7C501085FC501080F2938B50A
:1070C0000446154605D987211B4B1C4A1C4811F064
:1070D000DFF80F2A03D988211A4B184AF6E7FFF781
:1070E00017FF07294FF00F0318D8006A8A00934052
:1070F00020EA03032362236A05FA02F21A4322629A
:107100000322236849008A4023EA02032360022302
:10711000226803FA01F11143216038BDA1F1080290
:10712000406A9200934020EA03036362636A9540D9
:107130001D436562E4E700BF01C50108B9C5010848
:107140005FC50108A6C5010801238B409BB20383DC
:10715000704701238B409BB243837047012303FA9E
:1071600001F189B20AB10183704741837047008AF7
:1071700080B2084100F00100704700000F2938B5C7
:1071800005460C4603D9B4210648FFF7F5F92868EF
:10719000640020FA04F404F00300431E58425841EE
:1071A00038BD00BF8AE50108808A80B2084100F03E
:1071B0000100704710B5074C236853B9012005F052
:1071C000ABFB206028B9BDE8104036210248FFF72C
:1071D000D3B910BD440F00208AE5010810B50B4C4F
:1071E00023681BB93C210A48FFF7C6F9206842F220
:1071F000107105F0D9FC01280CBF0124002403D034
:1072000040210348FFF7B8F9204610BD440F002085
:107210008AE5010810B5074C23681BB951210648BF
:10722000FFF7AAF9002320681A46BDE81040194666
:1072300005F0CCBA440F00208AE5010810B50446D9
:10724000FFF7B8FFFFF7CAFF21461022034801F0FD
:10725000D9FE0446FFF7DEFF204610BD0054004073
:1072600010B5FFF7A7FFFFF7B9FF01F083FE044653
:10727000FFF7D0FF204610BD08B513460A46014669
:10728000034801F0B1FA003818BF012008BD00BF63
:107290000054004008B513460A460146034801F071
:1072A000A3FB003818BF012008BD00BF00540040F8
:1072B00008B513460A460146034801F073FC00383E
:1072C00018BF012008BD00BF0054004008B5134698
:1072D0000A460146034801F0F7FC003818BF0120B8
:1072E00008BD00BF0054004008B513460A460146D9
:1072F000034801F043FD003818BF012008BD00BF5E
:10730000005400400123064A83405169194205D0C8
:107310005361044B53F8203003B11847704700BF46
:1073200000040140480F00200F2838B504460D46E0
:1073300003D926210348FFF71FF9034B43F82450D4
:1073400038BD00BF8AE50108480F00200020FFF784
:10735000D9BF0120FFF7D6BF0220FFF7D3BF03201C
:10736000FFF7D0BF0420FFF7CDBF08B50920FFF716
:10737000C9FF0820FFF7C6FF0720FFF7C3FF06205D
:10738000FFF7C0FFBDE808400520FFF7BBBF08B509
:107390000F20FFF7B7FF0E20FFF7B4FF0D20FFF718
:1073A000B1FF0C20FFF7AEFF0B20FFF7ABFFBDE8EE
:1073B00008400A20FFF7A6BFFEE7FEE7FEE7FEE76C
:1073C000FEE7FEE7FEE7FEE7FEE7FEE7FEE7FEE795
:1073D000FEE7FEE7FEE7FEE7FEE7FEE7FEE7FEE785
:1073E000FEE7FEE7FEE7FEE7FEE7FEE7FEE7FEE775
:1073F000FEE7FEE7FEE7FEE7FEE7FEE7FEE7FEE765
:10740000FEE7FEE7FEE70A22B0FBF2F302FB130001
:1074100040EA0310C0B27047CA22024B5A6253229C
:107420005A62704700280040014B1860704700BF47
:10743000880F00204FF400320F4B10B50F4C5A61EB
:10744000E368DB0503D430210D48FFF795F8FFF71B
:10745000E3FF4FF40072A36823F48853A360094B41
:10746000C3F88420FF236362074B1B6813B1BDE898
:107470001040184710BD00BF000401400028004024
:107480008AE5010800E100E0880F00202DE9F04FB7
:107490009046394A87B014781F4681469DF840309F
:1074A0009DF844B02CB98C21344B354A354810F046
:1074B000EFFE421E1E2A5DD80C295BD8A8F5FA62A1
:1074C000632A57D8172F55D83B2B019352D8BBF1BD
:1074D0003B0F4FD808F13000C0B2FFF794FF82464F
:1074E0000846FFF790FF05024846FFF78CFF45EA84
:1074F0000A4A40EA0A0A3846FFF785FF019B06461A
:107500001846FFF780FF05025846FFF77CFF45EA63
:10751000064528431C4DFFF77FFFEA68019B42F0B8
:1075200080024AF4005AEA60EA685606FCD5C5F8BB
:1075300004A02860EA6822F08002EA60124AD0685B
:107540008006FCD5FF20506203A88DF80D308DF821
:107550000F908DF81010ADF811808DF80E708DF829
:107560000CB002F0D7FC094BC3E90001204607B07C
:10757000BDE8F08F0024F9E78C0F0020EAC5010870
:1075800060C60108F3C5010800280040900F0020E4
:1075900007B503780193437800938378B0F805200A
:1075A0000179C078FFF772FF03B05DF804FB0000BB
:1075B000264B10B51B7804461BB9E4212448FEF77E
:1075C000DBFF244AD36823F02003D360D3689B06F3
:1075D000FCD513685268C2F3035101EB8100C2F37A
:1075E000034101EB4001C9B201F5FA61A4F80510AD
:1075F000C2F30031C2F3032001EB810100EB410132
:107600002171C2F3011101EB810102F00F0202EBC3
:107610004102E270C3F30152C3F3034102EB820261
:1076200001EB4202A270C3F30232C3F3032102EB67
:10763000820201EB42026270C3F3021202EB820289
:1076400003F00F0303EB4203237010BD8C0F0020E7
:107650008AE50108002800401FB501A8FFF7A8FF30
:1076600001A802F057FC05B05DF804FB08B5FFF770
:1076700043FA1B4A136843F480731360FFF7CCFE90
:10768000184A536B23F4403343F482035363164B7D
:10769000DA6842F08002DA60DA685106FCD5FF222F
:1076A0001A611A6942F4FE021A619A6822F04002D5
:1076B0009A609A6822F44C529A60DA6822F080024A
:1076C000DA60094BDA689206FCD5FF225A62012281
:1076D000064B1A70FFF7C0FF054BC3E9000108BD58
:1076E0000070004000380240002800408C0F00204D
:1076F000900F002008B5094B1B7823B940F21F11E9
:107700000748FEF739FFFFF787FE064B9A6822F419
:1077100080729A60FF225A6208BD00BF8C0F002061
:107720008AE501080028004008B5144B1B7833B9DE
:1077300040F22711124B134A134810F0A9FDFFF72E
:107740006BFE124BDA6822F48072DA60104A91689C
:1077500041F400319160116841F400311160F02171
:107760000C4A82F829134FF4007151609A6842F470
:1077700088529A60FF225A6208BD00BF8C0F002019
:10778000EAC501084BC60108F3C5010800280040FE
:107790000004014000E100E0F8B51E46194B154613
:1077A0001B7833B94FF4A571174B184A184810F0DD
:1077B0006FFD184CFFF730FEA36823F48073A360BD
:1077C000E36823F48073E360FFF71DFE0746084675
:1077D000FFF719FE01042846FFF715FE054630465F
:1077E000FFF711FE41EA0761014341EA0521E36821
:1077F000DB07FCD5FF23E1616362BDE8F840FFF7DA
:1078000093BF00BF8C0F0020EAC5010839C60108EC
:10781000F3C5010800280040037842788178C078D9
:10782000FFF7BABF38B50D46044604F08BFD4FF0A4
:10783000E022136923F00103136104F0A1FD25B1D7
:107840001B4A536843F00603536072B6BFF34F8F71
:10785000BFF36F8F174A0120136823F0030343F42B
:10786000007343F00103136000F080FD124B1A69AE
:1078700042F004021A6130BF1A6922F004021A6150
:107880000E4B0F4A1B6893420BD10220FFF7FCF806
:107890004FF0E022136943F00103136104B162B6B3
:1078A00038BD084A9342F3D10220FFF7B3F8EFE75F
:1078B000002004E00070004000ED00E048020020DD
:1078C000D0FE3F0000093D0062B6704700220E4B1B
:1078D00010B51A700D4A0E4C1388204623F0400351
:1078E0001B041B0C13800D210222FFF7A7FB20466F
:1078F00002220E21FFF7A2FB2046BDE81040022223
:107900000F21FFF79BBB00BF980F002000380040FD
:1079100000040240294A38B5136A054643F48053EF
:107920001362052226480C461146FFF7C7FB0522C5
:1079300006212348FFF7C2FB052207212048FFF755
:10794000BDFBC5B1022205211D48FFF717FB02222E
:1079500006211B48FFF712FB022207211848FFF7F8
:107960000DFB012C1BD144F451740122154B1C80DA
:10797000154B1A7038BD2A4605211148FFF7FEFA4B
:107980002A4606210E48FFF7F9FA2A4607210C4835
:10799000FFF7F4FA012C09D144F45974E5E7022CFD
:1079A000E1D0032C0CBF03240024DCE7022CF3D02D
:1079B000032C14BF00240324EEE700BF003802406C
:1079C0000000024000300140990F002000220E4BC1
:1079D00010B51A700D4A0E4C1388204623F0400350
:1079E0001B041B0C138005210222FFF727FB2046F6
:1079F00002220621FFF722FB2046BDE810400222AA
:107A00000721FFF71BBB00BF990F0020003001408A
:107A100000000240054A064B127898811989C9076F
:107A200001D4002AFAD19889C0B27047990F00207A
:107A30000030014004480121038823F001031B04A6
:107A40001B0C038000F03FBE0004004010B5012174
:107A5000084800F02DFE60B1074C23684BB10121AE
:107A6000044800F030FEFFF7E5FF2368BDE8104052
:107A7000184710BD000400409C0F0020054AD36841
:107A800023F4E0631B041B0C43F0BF6343F4003397
:107A9000D360704700ED00E020220021114B10B5AB
:107AA000C3F88420104B114C1A6A204642F48042DD
:107AB0001A625A6942F480425A615A6922F4804239
:107AC0005A610B4A91811A6A092122F480421A6292
:107AD0000222FFF7B3FA2046BDE8104002220A2135
:107AE000FFF7ACBA00E100E00038024000000240BD
:107AF00000380140074B1A88920605D5064A1268DD
:107B000032B19888C0B210479B88044ADBB2137028
:107B1000704700BF00380140A40F0020A00F0020D4
:107B200010B504468021084800F050FE0028F9D026
:107B30002146054800F02AFE034C4021204600F073
:107B400045FE0028F9D010BD0038014010B5441E94
:107B500014F8010F00B910BDFFF7E2FFF8E70000CD
:107B600008B5024800F016FEC0B208BD003801405A
:107B70002DE9F0410E4601214FF4C068074688B058
:107B8000084614461D4600F02BFD01214FF48040AD
:107B900000F032FD3C4B3D4802A9CDE9028300F0E4
:107BA0008BFC07220921394800F0C2FC07220A2178
:107BB000364800F0BDFC452E04973CD14FF480635D
:107BC000ADF81830072C42D10023ADF81430052D44
:107BD0004ED14FF48053ADF816300023ADF81C3071
:107BE0000C232B4804A9ADF81A3000F071FD294B85
:107BF0001A6802B1012240F22551254800F0CEFD5D
:107C00000121234800F0B6FDFFF7AAFF25238DF8D8
:107C100004309DF8383001A88DF8053000238DF828
:107C2000063001238DF80730FFF728FF00F07CFABB
:107C300008B0BDE8F0814F2E02D1ADF81880C1E741
:107C40000023072CADF818300DD1592107E0082C7E
:107C500002D14FF48053B8E7092CB8D154210E4813
:107C6000FEF78AFCB3E7082CAED0092CAFD1F0E7C1
:107C70000F2D02D14FF44053ADE7022D0CBF4FF44E
:107C800000530023A7E700BF0202000100000240EA
:107C900000380140A40F00208AE501080E2307B533
:107CA000082200934E210123FFF762FF03B05DF825
:107CB00004FB0000402200210D4B0E48C3F8842035
:107CC0000D4B5A6A42F400325A629A6942F4003209
:107CD0009A619A6922F400329A61084A91815A6A3B
:107CE000032122F400325A620222FFF7A7B900BF33
:107CF00000E100E000000240003802400044004083
:107D000008B5024800F046FDC0B208BD004400407E
:107D10002DE9F0471D46262388B08DF80430002356
:107D20009DF84080824601A814468DF806308DF8F3
:107D300007300E469DF844709DF848908DF80580F8
:107D4000FFF79CFE00F0F0F90121084600F048FC26
:107D500001214FF4003000F05BFC67B10821514B6A
:107D60005148CDE9021302A900F0A6FB0722032126
:107D70004D4800F0DDFBB9F1000F0CD00422494B57
:107D8000494802A9CDE9022300F096FB072202210F
:107D9000454800F0CDFB452ECDF810A044D14FF45E
:107DA0008063072CADF818304BD10023ADF81430A8
:107DB000052D57D14FF480530024ADF81630ADF89F
:107DC0001C40B9F1000F58D1ADF81A9077B1BDF849
:107DD0001A3043F00403ADF81A30344B1A6802B17C
:107DE000012240F22551324800F0D8FC304804A965
:107DF00000F06EFC01212E4800F0BCFC0FB1FFF733
:107E00007FFF26238DF8043000238DF806300123F0
:107E100001A88DF807308DF80580FFF72FFE00F0E0
:107E200083F908B0BDE8F0874F2E02D14FF4C0634C
:107E3000B7E70023072CADF818300ED140F203113C
:107E400007E0082C02D14FF48053AFE7092CAFD1E3
:107E5000FE211848FEF790FBAAE7082CA5D0092CB4
:107E6000A6D1F0E70F2D02D14FF44053A4E7022D25
:107E70000CBF4FF4005300239EE70823224640F234
:107E800027710B48ADF81A3000F088FC40F22661EB
:107E9000074800F0A1FC224640F22661044800F0A9
:107EA0007DFC93E70203000100000240A80F0020C0
:107EB000004400408AE5010870B504460025134ED1
:107EC0008021134800F082FC60B12146104800F088
:107ED0005DFC00240E4D0D4E4021284600F076FC3E
:107EE00050B170BD0135B5F5801FE9D340F24F1197
:107EF0003046FEF741FBE3E70134B4F5801FEBD3D6
:107F00004FF4AC713046FEF737FBE5E78AE5010830
:107F10000044004008B5064B0246186000B101223B
:107F200040F22551034800F039FC012008BD00BF94
:107F3000A80F002000440040114810B5038899069E
:107F400008D5104B1B682BB10288D20710D480884B
:107F5000C0B298470A4803885B060FD540F22661F5
:107F600000F03AFC084B1B6843B1BDE810401847CD
:107F700000F010FC054BC0B21870EBE710BD00BF5D
:107F800000440040A80F0020AC0F0020A00F0020EC
:107F9000BFF34F8F0449054BCA6802F4E0621343F4
:107FA000CB60BFF34F8FFEE700ED00E00400FA0561
:107FB00010B5441EE3B2052B03D917211148FEF773
:107FC000DBFAFEF7B7FD45F255520F4B1A60DA683F
:107FD000D207FCD4052C06D8DFE804F0030A0C0E07
:107FE000101201225A604CF6CC42074B1A6010BDA9
:107FF0000222F7E70322F5E70422F3E70522F1E77F
:108000000622EFE78AE501080030004038B5224C2F
:10801000236853B95F2000F013FB204D38B1204B8B
:10802000236001232B7000F01BFB206838BD5E200D
:1080300000F006FB18B11B4B23600223F2E75D2022
:1080400000F0FEFA18B1184B23600323EAE75C2026
:1080500000F0F6FA18B1154B23600423E2E75B2029
:1080600000F0EEFA18B1124B23600523DAE75A202C
:1080700000F0E6FA18B10F4B23600623D2E759202F
:1080800000F0DEFA18B10C4B23600723CAE70B4B54
:108090002360FF23C6E700BFB40F0020B80F002005
:1080A0006CC601087CC6010892C60108ADC601086D
:1080B000BCC60108CBC60108E4C60108FBCE010816
:1080C00038B5084B084D1A7852B9012420461C7067
:1080D00000F0DEFA287020F0FF01204600F0C8FA18
:1080E000287838BDB00F0020B10F002010B504462D
:1080F000012000F0CDFA20F0FF0121430120BDE86E
:10810000104000F0B5BA08B5FFF7F0FFFFF740FFE9
:10811000012008B500F0BCFAC0B210B90120FFF789
:10812000F2FFFFF735FF000030B5012403780A4D58
:1081300003F01F029440C278590952B1074A2B44F8
:10814000D26842781201D2B283F8002345F8214068
:1081500030BD2031FAE700BF00E100E000ED00E0B3
:1081600008B5084B98420BD101214FF4007000F084
:108170005BFABDE8084000214FF4007000F054BAEB
:1081800008BD00BF0024014043680A7923F0407312
:1081900023F4807343EA02230A6810B51343436053
:1081A000D1E9032313438A6884681343084A2240B1
:1081B00013434A7943EA420383600A7D036B013A21
:1081C00023F0F873D2B243EA0253036310BD00BF39
:1081D000FDF7FFC000234FF040720360C0E90323A6
:1081E00083808360012303757047836819B143F06E
:1081F00001038360704723F00103FAE7044B5A68D8
:1082000018B142F400025A60704722F40002FAE703
:10821000002701401D2970B51AD90726A1F11E04B7
:10822000C56D04EB4404A64025EA0605A3402B4394
:10823000C365062A35D81F24013A036C02EB82027B
:10824000944023EA040301FA02F21A43026470BD67
:1082500013290CD90726A1F11404C56804EB4404C2
:10826000A64025EA0605A3402B43C360E1E70929A0
:108270000CD90726A1F10A04056904EB4404A640C1
:1082800025EA0605A3402B430361D2E7072544698D
:1082900001EB4106B54024EA0504B34023434361A2
:1082A000C7E70C2A0CD8D41F1F22C36B04EB84042D
:1082B000A24023EA020301FA04F21A43C263C6E7AA
:1082C000122A0DD8A2F10D031F22846B03EB830346
:1082D0009A4024EA020401FA03F222438263B6E7D9
:1082E000182A0CD81F24133A436B02EB82029440E5
:1082F00023EA040301FA02F21A434263A7E71F24A8
:10830000193A036B02EB8202944023EA040301FA58
:1083100002F21A4302639AE7836843F08043836062
:108320007047806D80B270470368194214BF012006
:1083300000207047C943016070470000044B1A6871
:1083400018B142F002021A60704722F00202FAE706
:10835000003C0240044B1A6818B142F004021A6053
:10836000704722F00402FAE7003C0240044B1A680E
:1083700018B142F008021A60704722F00802FAE7CA
:10838000003C0240044B5A68D20741BF034ADA60FE
:10839000034ADA60704700BF003C0240EFCDAB8972
:1083A00005040302024A536843F001035360704717
:1083B000003C0240014B9861704700BF003C024006
:1083C000084B9A69D10709D49A69D20508D49B69E8
:1083D00013F4F05F14BF032004207047012070479E
:1083E00002207047003C0240042313B504468DF878
:1083F0000730FFF7E5FF8DF807009DF80730012BE8
:108400000AD11CB905238DF8073007E0FFF7D8FF24
:10841000013C8DF80700F0E7002CF3D09DF8070031
:1084200002B010BD10B504464FF40040FFF7DCFF6A
:10843000042804BF0023236010BD000038B50446A3
:108440004FF400400D46FFF7CFFF04280BD1064A3A
:108450004FF40040536823F4807353602560BDE8F7
:108460003840FFF7C1BF38BD003C024038B5044674
:108470004FF400400D46FFF7B7FF04281BD135B17C
:1084800025704FF40040BDE83840FFF7ADBFFF2333
:1084900024F0030504F003042968E40003FA04F45B
:1084A00021EA04042846FFF7BDFF21462846BDE81F
:1084B0003840FFF7C3BF38BD2DE9F0410022012746
:1084C00003260B6807FA02FE3EEA03032BD103687A
:1084D00091F804C0540006FA04F86FEA080523EA8C
:1084E00008080CFA04F30CF1FF3C43EA0803BCF162
:1084F000010F03600ED883682B404D79A5401D43C2
:10850000856083889BB223EA0E058B7993409BB2EA
:108510002B438380C36806FA04F523EA0505CB796B
:10852000A3402B43C3600132102ACAD1BDE8F081B9
:1085300010B50F2401F00703C90800EB8100016AA0
:108540009B009C4021EA04010162016A9A400A43AF
:10855000026210BD1E4B10B59A6802F00C02082A88
:108560001DD00BD80AB1042A19D04FF400425B6821
:10857000C3F34233013302FA03F311E00C2AF4D1BE
:108580009A68144CC2F383429968A25C9B68124BB0
:108590005343C1F381520132B3FBF2F300E00E4BBF
:1085A0000B4A036093680D49C3F30313CC5C036863
:1085B000E34043609468C4F302240C5D23FA04F49E
:1085C00084609268C2F3C2228A5CD340C36010BD4B
:1085D000003802405C0200200024F4004C0200201D
:1085E000044BDA6911B11043D861704722EA0000E8
:1085F000FAE700BF00380240044B1A6A11B1104379
:108600001862704722EA0000FAE700BF0038024013
:10861000044B5A6A11B110435862704722EA0000B5
:10862000FAE700BF00380240044B5A6911B1104309
:108630005861704722EA0000FAE700BF00380240A4
:108640004309012B054B00F01F000CBF1B685B6B3F
:1086500023FA00F000F00100704700BF003802402C
:10866000024A536B43F080735363704700380240F3
:10867000002382B00193054B0193019B03EB800320
:108680000193019B196002B0704700BF5028004061
:10869000002382B00193054B0193019B03EB800300
:1086A0000193019B186802B0704700BF502800403A
:1086B000038A828911EA030092B203D00A4214BFEE
:1086C000012000207047C94389B201827047000031
:1086D00030B50D460446038AEA889BB223F4405322
:1086E0001343898903828389288923F4B052AB8894
:1086F00022F00C020343688912040343120C9BB25C
:108700001343A381A38A85B09BB223F440730B4328
:108710006846A382FFF71EFFDDE9023214498C424E
:1087200008BF13461922A18953432A680D044CBF80
:10873000520092006421B3FBF2F3B3FBF1F001FBB2
:1087400010330201A08900044BBFDB001B01323350
:1087500032334BBFB3FBF1F3B3FBF1F303F0070389
:1087600003F00F0313439BB2238105B030BD00BF5C
:1087700000380140838921B19BB243F400538381C7
:10878000704723F400531B041B0CF8E7C1F30801E6
:10879000818070478088C0F308007047012310B5BE
:1087A000C1F342149C4201F01F0103FA01F105D10B
:1087B0000C3003683AB11943016010BD022C0CBFA4
:1087C00010301430F5E723EA0101F5E70388194278
:1087D00014BF0120002070470123090A8B40DB43AE
:1087E0009BB20380704700002DE9F3411F46002330
:1087F00004460D46164601931AB9012002B0BDE8A1
:10880000F08140F6FF7301934FF40031204600F0F1
:108810005DFD002852D10121204600F023FD4FF2DA
:10882000FF71204600F038FD0121204600F002FDD6
:1088300040F6FF73DFF89C8101934146204600F02B
:1088400039FD002841D039460122204600F016FDAE
:1088500040F6FF73604F01933946204600F036FD25
:10886000002838D0012E42D10021204600F0FAFC29
:1088700003F068FD31462046238B00F0E7FC03F04F
:108880007FFD40F6FF73554E01933146204600F0C0
:108890001DFD30B3204600F0FCFC287040F6FF734D
:1088A0004F4D01932946204600F010FD0028A4D02A
:1088B000019B5A1E0192002BF4D104E0019B5A1E29
:1088C0000192002BA0D1002098E7019B5A1E019233
:1088D000002BB2D1F7E7019B5A1E0192002BBBD1AE
:1088E000F1E7019B5A1E0192002BCED1EBE7022E3D
:1088F00025D103F027FD4FF40061204600F0CCFCA9
:108900000021204600F0AEFC238B03F039FD40F639
:10891000FF73344E01933146204600F0D7FC40B13E
:108920000121204600F092FC238A2B70238A6B7071
:10893000B4E7019B5A1E0192002BECD1C3E740F62D
:10894000FF77033E238BDFF89C802E44B5420197CE
:1089500028D1244E3146204600F0B8FC70B30021E7
:10896000204600F07FFC204600F093FC40F6FF73A9
:108970001C4E287001933146204600F0A7FC18B326
:108980000121204600F062FC204600F082FC687065
:10899000204600F07EFCA87080E7019B5A1E0192E1
:1089A000002B90D04146204600F090FC0028F4D0E7
:1089B000204600F06EFC05F8010BC7E7019B5A1E2C
:1089C0000192002BC6D17EE7019B5A1E0192002B1B
:1089D000D1D178E701000300020000104000001030
:1089E00010000010040000102DE9F3411E46002382
:1089F000019340F6FF7304460D4617460193002A83
:108A000000F082804FF40031204600F05FFC002827
:108A100043D10121204600F00DFC40F6FF73DFF842
:108A2000708101934146204600F044FC00283DD06F
:108A300031460022204600F021FC40F6FF73554EDF
:108A400001933146204600F035FC002834D02E46F4
:108A5000204616F8011B3D4400F019FC40F6FF7754
:108A6000DFF83481AE42019731D14B4D2946204683
:108A700000F02CFC002836D02046012100F0E6FB57
:108A800040F6FF73454D464C01932946204600F0C1
:108A90001DFC00282DD1012005E0019B5A1E0192EA
:108AA000002BAFD1002002B0BDE8F081019B5A1E1F
:108AB0000192002BB6D1F5E7019B5A1E0192002BC3
:108AC000BFD1EFE7019B5A1E0192002BEAD041462D
:108AD000204600F0FBFB0028F4D0204616F8011BCE
:108AE00000F0D5FBBEE7019B5A1E0192002BBDD1C1
:108AF000D8E7019B5A1E0192002BC6D1D2E7019BF9
:108B00005A1E0192002BCDD04FF40031204600F0C8
:108B1000DDFB0028F3D10121204600F08BFB40F65D
:108B2000FF731B4D01932946204600F0C3FB10B391
:108B300000223146204600F0A1FB40F6FF73154DA0
:108B400001932946204600F0B5FBD0B12046012113
:108B500000F07CFB40F6FF73104D114C0193294649
:108B6000204600F0B3FB002895D0019B5A1E0192CD
:108B7000002BF4D196E7019B5A1E0192002BD2D113
:108B800090E7019B5A1E0192002BDAD18AE700BFC1
:108B90000100030082000700040000101000001014
:108BA000005400402DE9F3411E46002304460D46C3
:108BB000174601931AB9012002B0BDE8F08140F6D2
:108BC000FF7301934FF40031204600F07FFB002833
:108BD00038D10121204600F02DFB40F6FF73DFF86D
:108BE000D48001934146204600F064FB002843D026
:108BF00031460022204600F041FB40F6FF732E4E26
:108C000001933146204600F055FB00283AD02E460D
:108C1000204616F8011B3D4400F039FB40F6FF7773
:108C2000DFF89880AE42019737D1244D294620467F
:108C300000F04CFB0028BED1019B5A1E0192002B74
:108C4000F4D104E0019B5A1E0192002BBAD12046B8
:108C5000012100F0FBFA40F6FF73194D194C019306
:108C60002946204600F032FB20B1019B5A1E01929A
:108C7000002BF5D100209FE7019B5A1E0192002B8B
:108C8000B0D1E4E7019B5A1E0192002BB9D1DEE777
:108C9000019B5A1E0192002BD9D04146204600F07C
:108CA00015FB0028F4D0204616F8011B00F0EFFA5F
:108CB000B8E700BF010003008200070004000010B5
:108CC000100000100054004000232DE9F3410D4630
:108CD0004FF4003104461746019300F0F7FA18B933
:108CE000002002B0BDE8F0810FB90120F9E72E465F
:108CF000204616F8011B3D4400F0C9FA40F6FF7704
:108D0000DFF86C80AE4201971FD1194D29462046ED
:108D100000F0DCFA28B32046012100F097FA40F673
:108D2000FF73144D144C01932946204600F0CEFAEF
:108D30000028DAD0019B5A1E0192002BF4D1CFE714
:108D4000019B5A1E0192002BCAD04146204600F0DA
:108D5000BDFA0028F4D0204616F8011B00F097FA5F
:108D6000D0E7019B5A1E0192002BCFD1B8E700BF7C
:108D70000400001010000010005400402DE9F341E1
:108D80001F46002304460D46164601931AB90120DA
:108D900002B0BDE8F0814FF4003100F097FA08B955
:108DA0000020F5E70121204600F05CFA4FF2FF7148
:108DB000204600F071FA0121204600F03BFA40F60F
:108DC000FF73DFF89C8101934146204600F072FA60
:108DD00000283AD039460122204600F04FFA40F6EA
:108DE000FF73604F01933946204600F06FFA002868
:108DF00031D0012E3BD10021204600F033FA03F0A0
:108E0000A1FA31462046238B00F020FA03F0B8FA8D
:108E100040F6FF73544E01933146204600F056FA57
:108E2000F8B1204600F035FA287040F6FF734F4D38
:108E300001932946204600F049FA0028A7D0019B5B
:108E40005A1E0192002BF4D1AAE7019B5A1E0192EF
:108E5000002BB9D1A4E7019B5A1E0192002BC2D16D
:108E60009EE7019B5A1E0192002BD5D198E7022E56
:108E700029D14FF40061204600F00EFA03F062FAA7
:108E800000212046238B00F0EDF903F079FA40F63B
:108E9000FF73374E01933146204600F017FA60B158
:108EA00003F050FA0121204600F0D0F9238A2B70FC
:108EB000238A6B7003F064FAB7E7019B5A1E019294
:108EC000002BE8D16CE740F6FF77033E238BDFF8F9
:108ED000A0802E44B542019729D1254E3146204627
:108EE00000F0F4F978B30021204600F0BBF92046E9
:108EF00000F0CFF940F6FF731D4E28700193314604
:108F0000204600F0E3F920B30121204600F09EF94D
:108F1000204600F0BEF96870204600F0BAF9A8704B
:108F200083E7019B5A1E0192002B3FF439AF414663
:108F3000204600F0CBF90028F3D0204600F0A9F934
:108F400005F8010BC6E7019B5A1E0192002BC5D103
:108F500026E7019B5A1E0192002BD0D120E700BFCB
:108F6000010003000200001040000010100000107B
:108F70000400001038B5204B08219A691F4842F4BC
:108F800000129A619A6922F400129A615A6A22F4D4
:108F900000125A62FEF7D8F8012308211A46174832
:108FA000FEF70CF8092115480122FEF747F80921C0
:108FB0001248FEF7DCF8D8B1012038BD0821284658
:108FC000FEF7C2F8FDF70AFE08212846FEF7C1F8B1
:108FD000FDF704FE013CF1D109210848FEF7C7F86E
:108FE00020B940F27D110648FDF7C6FA2046E4E7B5
:108FF0003324024DEEE700BF003802400004024077
:109000008AE501082DE9FF41444B054698420E468A
:1090100017467CD103F5F2335A6A082142F4001254
:109020005A629A693E4842F400129A619A6922F49F
:1090300000129A61FEF788F8012308211A46384881
:10904000FDF7BCFF092136480122FDF7F7FF092192
:109050003348FEF78CF8002855D0012308211A4622
:109060002F48FDF7ABFF042208212D48FEF726F814
:10907000012309211A462A48FDF7A0FF04220921ED
:109080002748FEF71BF8274B9A6942F400129A61B1
:109090009A6922F400129A61684600F0B1F8224BF6
:1090A000694601934FF48063ADF80A304FF4804372
:1090B0002846ADF80C30ADF80870009600F038F88E
:1090C0002846012100F0AAF8012019E008214046B5
:1090D000FEF73AF8FDF782FD08214046FEF739F821
:1090E000FDF77CFD013CF1D109210D48FEF73FF869
:1090F0000028B2D10D4840F2A511FDF73DFA2046F7
:1091000004B0BDE8F0813324DFF81480EAE74FF4BF
:10911000DA710648FDF730FABEE700BF00540040A0
:1091200000040240003802400000FFBF8AE5010849
:109130007FB50446868868460D46FFF70BFA029A0B
:109140002D4926F03F06B2FBF1F13604360C88B209
:109150000643A6802388294E23F001031B041B0C21
:1091600023802B68B34223D85B00B2FBF3F39BB29E
:10917000042B38BF0423013080B22084A3832388CA
:10918000AA889BB243F0010323802388698923F4D2
:10919000816323F002031B040A431B0C13439BB29D
:1091A0002A892380AB8913439BB2238104B070BD0D
:1091B0004BF6FF70EE8886421BBF1920434303EB3A
:1091C0004303B2FBF3F30BBFB2FBF3F39BB29BB2CF
:1091D00043F48043C3F30B020AB943F001034FF495
:1091E000967251434FF47A72B1FBF2F1013189B2B8
:1091F00043F400432184C1E740420F00A0860100F0
:1092000041F28832044BC0E90023002383604FF40D
:1092100080438381704700BF0000FFBF038821B1F6
:109220009BB243F001030380704723F001031B044A
:109230001B0CF8E7038821B19BB243F480730380D1
:10924000704723F480731B041B0CF8E7038821B1DB
:109250009BB243F400730380704723F400731B0434
:109260001B0CF8E7038821B19BB243F480630380B1
:10927000704723F480631B041B0CF8E722B141F014
:10928000010189B20182704701F0FE01F9E7018214
:109290007047008AC0B270470388B1F5006F15BFF0
:1092A00023F400639BB21B0443F4006318BF1B0C40
:1092B00003807047838A008B9BB243EA00430B40D4
:1092C00023F07F435B1A584258417047002382B015
:1092D000009301930B0F01900093009B21F07F41BD
:1092E00053B1019B14330193019B1B680B4214BFC4
:1092F0000120002002B07047019B090C1833F2E7EF
:10930000F8B50E46054680B14F1C384600F05CFFAC
:10931000044640B13A4600210FF01CFA3246294675
:1093200020460FF0EFF92046F8BD0446FBE738B5BC
:109330000D46044628B110F02DFA234620448342FE
:1093400001D1002038BD13F8012BAA42F7D101202A
:10935000F8E773B505460E4600240EF0C5FF224619
:10936000046001A9284610F035FB05460EF0BCFF4D
:109370000368222B0BD0019B1B7843B9A542ADBFDC
:109380002846204601232346336002B070BD0123E6
:109390002046F9E72DE9F04F05464FF0010B002676
:1093A00087B0CDE9021206F10903122B8CBF03200E
:1093B000022000F009FF0746F0B13246374910F0AD
:1093C0003BF9029B53F826A0F5B90024384600F07B
:1093D000E5FEBBF1000F02D1284600F0DFFE8CB1A4
:1093E000039B0136B3424FF0000B03D1204607B078
:1093F000BDE8F08F2546D6E7BBF1000F02D1284625
:1094000000F0CCFE0024F1E7254B4FF00009BAF143
:10941000000F08BF9A46504610F0BCF9009038463D
:1094200010F0B8F901902846514610F0E2F9B8B9A9
:10943000284610F0AFF9DDE9002301309B1A09FB43
:10944000030000F0C1FE04460028BED00346A84633
:10945000B9F1010909D24146184610F093F9B5E770
:10946000009B09F101091844DEE751464046059387
:1094700010F0BFF9059BA0EB080241461846049284
:1094800010F0A4F9049A3946104410F07BF90099C1
:10949000049A019B0A44C3189044D9E7A3B3010876
:1094A0008AE5010830B580B10346021F00F11804B7
:1094B00052F8045F8D4208D0A242F9D11C301A46FE
:1094C00014680433013401D1116030BD8342F6D1F8
:1094D000FBE700000649431E13F8010F00B970476F
:1094E0000A5C02F00302022A08BF20381870F3E772
:1094F000B2ED010870B50E46044670B10025AE42CB
:1095000004D12046BDE8704000F048BE54F8250064
:1095100008B100F043FE0135F1E770BD2DE9F74FCA
:109520008A4604460092002839D00027E35D8BBBB1
:10953000A04622461E46384804EB070B5A4537D151
:1095400003B10136002E5FD00137384600F03CFEF3
:10955000044628B33A4600210FF0FCF8B00000F0B2
:1095600033FE0546002851D04FF000090021C345C5
:109570002CD131B12046FFF7C3FE002846D045F874
:109580002900204600F00AFE009B1E60284603B01A
:10959000BDE8F08F0137B7F5807FC7D1002426469C
:1095A000002531462046FFF7A5FF009B1D60EDE733
:1095B00012F8011B514504D1002BBFD00023013606
:1095C000BCE7095C090758BF0133B7E718F8013B4E
:1095D000534512D10029CAD02046FFF791FEA8B109
:1095E00009F1010345F829003A460021204601937C
:1095F0000FF0B0F8019B9946B8E7074A985C02075C
:109600005CBF63540131B2E73546BFE7204600F046
:10961000C5FD2C46C4E700BFB2ED01082DE9F743B4
:10962000002507460820884691461E46009500F012
:10963000CBFD0446002865D0C0E90055384610F03F
:10964000A9F801280FD13B782A2B0CD109F1FF335F
:10965000C4F80080636022684A4502D263684B45C3
:1096600040D3294B0DE02D213846FFF760FE05461B
:10967000B8B9019001A93846FFF76BFE019B63B1B1
:10968000224B336028460099FFF734FF002C35D079
:10969000204600F083FD002430E01D46C4E90000B0
:1096A000D9E76A462D213846FFF738FF009B05466B
:1096B000013B012B01D9164BE3E70023006801A908
:1096C0000193FFF746FE2060019B0BB1114BD8E7D9
:1096D000686801A9FFF73DFE6060019B002BBAD0CE
:1096E0000D4BCEE7424501D3434501D20B4BC8E7B2
:1096F00028460099FFF7FEFE00233360204603B0A2
:10970000BDE8F0830546BDE774C70108EEC6010851
:109710000DC7010836C7010855C7010894C70108DD
:1097200008B520B34A1C22D0062920D8DFE801F072
:10973000040D101316191C00002303600FF0EAF843
:109740000840431C5842584108BD00234360F5E7D8
:1097500000238360F2E700238361EFE70123C36006
:10976000ECE700230361E9E700234361E6E701201A
:10977000EAE770B5054688B181B10E1F01F1180402
:1097800056F8041F4B1C03D1A642F9D1002070BD2E
:109790002846FFF7C5FF0028F6D0F8E70120F6E7D6
:1097A00008B538B34A1C25D0062923D8DFE801F0D4
:1097B000040E1216161A1E000368013303600FF020
:1097C000A9F80840431C5842584108BD436801337A
:1097D0004360F4E7836801338360F0E7C3680133D3
:1097E000C360ECE7036901330361E8E743690133D0
:1097F0004361E4E70120E8E700290B46B8BFCB1D31
:109800004A4202F0070201F0070158BF514201220B
:10981000C3F3C703C9B202FA01F1C25C1143C154D8
:10982000704700290B46B8BFCB1D4A4202F0070221
:1098300001F0070158BF51420122C3F3C703C9B267
:109840008A40C15C21EA0201C15470470B460029DD
:10985000B8BFCB1DC3F3C703C05C4B4203F0070383
:1098600001F0070158BF5942C9B2084100F0010098
:1098700070472DE9F843089E8846174699460546E5
:1098800010B11446A0450BD848460999FFF788FF48
:1098900068B1012200240B9B1A602046BDE8F883C2
:1098A00021462846FFF7D2FFE8B90134EAE73146FE
:1098B0004846FFF735FF04460028EAD1B5B12146F6
:1098C0002846FFF7C3FF70B90134A045F7D104461D
:1098D000B9F1000FDDD0711E042909D8DFE801F0CD
:1098E0001A1D20232600A742F2D1D6E72C46EFE727
:1098F000C9F8004048460FF00DF8B1F1FF3F08BF2E
:10990000B0F1FF3FC5D048460A99FFF732FF002863
:10991000C3D0BEE7C9F80440ECE7C9F80840E9E75E
:10992000C9F81840E6E7C9F80C40E3E7C9F8104069
:10993000E0E72DE9F04F4FF000098BB006461C2000
:109940000C469046CDF8249000F03EFC05460028D9
:1099500000F0EE801C2000F037FC0746002800F0E5
:10996000E78005F11B031B1A362B40F2A1801C2255
:10997000FF2128460EF0EEFE1C22FF2138460EF095
:10998000E9FE00230121D4F800A00DF12409CDE95E
:10999000003152463C2123463046CDE90279FFF79B
:1099A00068FF0999002940F09680824502D1284637
:1099B000FFF778FD02234FF0010AD4F804B0CDE997
:1099C00000A35A4623463C21CDE9025906F108007E
:1099D000FFF74FFF099B002B7DD1834573D1514683
:1099E0002846FFF75FFD03234FF0020AD4F808B0C2
:1099F000CDE900A35A4623461821CDE9025906F1C4
:109A00001000FFF736FF099B002B64D183456DD111
:109A100051462846FFF746FDE368D4F818B0049392
:109A200006F11403069306F11303079340F26F1334
:109A3000DDF810A0059351460698FFF707FF20B107
:109A400059460798FFF702FF68B9059B013B05934C
:109A500009D004212046FFF7A3FE00284FD00123A0
:109A60004FF0000A0993099BABBB049B53454FD1B0
:109A700004212846FFF716FD05230622D4F810A07E
:109A8000CDE900320C2123465246CDE9025906F1B8
:109A90001800FFF7EEFE099BEBB982451BD0636906
:109AA000A3EB0803042B3CD94FF0FF33099312E0DA
:109AB0004B464FF0FF3245F8232047F8232001336F
:109AC000072BF8D15DE7424621463046FFF731FFCC
:109AD0000990002887D0284600F060FB17B138466F
:109AE00000F05CFB09980BB0BDE8F08F42462146C0
:109AF0003046FFF71EFF099000288DD0EBE729467E
:109B00002046D4F80CA0D4F818B0FFF732FE92E744
:109B1000424621463046FFF70CFF09900028ABD0A3
:109B2000D9E7424621463046FFF703FF0990D2E7C6
:109B30004FF0FF330993002DD4D00027CBE700006E
:109B40002DE9F04F002487B0894692462C2103AAC4
:109B50009846109E0394FFF7E1FC074688B93E4BF8
:109B6000336038460399FFF7C5FC07B0BDE8F08FB6
:109B7000D0F800B06B685B451CD2284600F00EFBA5
:109B80000134039BA342ECD957F824502F212846D7
:109B9000FFF7CDFBA8B93346284642465146FFF7AA
:109BA0003DFD33680546002BE2D00028D9D000F0F7
:109BB000F5FAD6E759464846FFF71EFE0BF1010BB2
:109BC000D8E700232F21284604AA0493FFF7A6FC18
:109BD000049905464B1E012B04D9204B3360FFF737
:109BE00089FCBEE74246334651460068FFF716FD42
:109BF000326883462AB108B100F0D0FA28460499A9
:109C0000EDE72D212868FFF792FB18B908F1FF3224
:109C1000CBF80420002305A968680593FFF799FB9A
:109C20000599024619B10E4A58463260E4E7DBF85E
:109C30000010DBF80400884205D228460499FFF79B
:109C400059FC58469AE74846CDE90012FFF7D4FD83
:109C5000DDE900121144ECE7B9C70108CBC70108E0
:109C6000F0C701082DE9FF41002305460E461446C2
:109C7000039302B902AC236045B9574B23602846D1
:109C80000399FFF737FC04B0BDE8F0812846202196
:109C900003AAFFF743FC039B0546062B01D04F4B5D
:109CA000ECE71A22002130460EF054FD0094002209
:109CB0003C2331462868FFF743FF2268002ADED1A3
:109CC00000943C23686806F10801FFF739FF226819
:109CD000002AD4D100941823A86806F11001FFF7D8
:109CE0002FFF2368002BCAD1686908B1FFF7F2FB88
:109CF00007223B496869FFF74DFB07460FF04AFD15
:109D0000012806F1130804D13B783F2B04BF2A2316
:109D10003B7000220823414638460094FFF710FFAD
:109D2000384600F03BFA2268002AA8D107214046B5
:109D3000FFF78CFD30B111464046FFF75DFD07216E
:109D4000FFF76FFDEF6806F1140838460FF022FDAB
:109D5000012804D13B783F2B04BF2A233B702023EA
:109D60000022414638460094FFF7EAFE00214046B3
:109D7000FFF757FD2368002B81D12F69002F3FF497
:109D80007EAF3846FFF7A6FB00287FF478AF384651
:109D90000D221449FFF7FEFA074600283FF46FAF83
:109DA00018360D23012231460094FFF7C9FE3846CC
:109DB00000F0F4F9012421463046FFF747FD30B1A9
:109DC000611E3046FFF718FD2146FFF72AFD0134DA
:109DD0000D2CF0D153E700BF0FC8010827C80108B8
:109DE00068020020840200202DE9F0418CB0054675
:109DF000CDE9002328B94FF0FF3001460CB0BDE893
:109E0000F0812422002103A80EF0A4FC684603A9D7
:109E10000EF096FB04460028EDD00EF07BFDB1F16C
:109E2000FF3F08BFB0F1FF3F80460F46E3D0214619
:109E300028466269FFF77DFD06460028DBD12046F3
:109E40000EF068FDB1F1FF3F08BFB0F1FF3FD2D087
:109E50008F4208BF804503D020460EF05BFDCDE762
:109E600031462046FFF79CFC0028C4D121462846F5
:109E70006269FFF75EFD0028EED0BCE770B58AB0DE
:109E8000DDE90E4501953C2594FBF5F605FB1644EE
:109E90000294182493FBF4F505FB1433CDE9033049
:109EA0000C23013991FBF3F003FB10110023CDE9E2
:109EB00007339DF84030A2F26C7201A8059106921A
:109EC00009930EF027FD0AB070BDF7B50446684649
:109ED000CDE900230EF016FB0269037A551C426996
:109EE00090F804C0077B067E02F26C71C2690068BC
:109EF000A370003B18BF012320702046013284F874
:109F000001C0E7702571A4F80510E6712272637232
:109F100003B0F0BD1FB5437A0293037801934378F1
:109F200000938378B0F805200179C078FFF7A6FF89
:109F300005B05DF804FB904271EB0303B4BF012050
:109F400000207047032210B5104986B00B7801330A
:109F5000B3FBF2F202EB42029B1A0D4A0B7052F86D
:109F6000234003781A21049343780A4A03938378A1
:109F70000293C378019303790093B0F8053020462B
:109F80000FF026FB204606B010BD00BF07100020D2
:109F9000F0C80108B5C80108B1F1004F08BF00289A
:109FA0001FB502460B4608D001A8FFF78EFF01A897
:109FB000FFF7C8FF05B05DF804FB0148FAE700BFF2
:109FC000D3C801082DE9FF470322044629480D1E86
:109FD000037803F10103B3FBF2F202EB4202A3EBBD
:109FE0000203254A037052F823903DDA4FF0010A2C
:109FF000644265EB45050023204A204629460DF0C2
:10A000008BFF00230646294620461C4A0DF084FF9C
:10A01000104619464FF4616200230DF07DFF4FF4A6
:10A02000616207460023204629460DF075FF104661
:10A0300019463C2200230DF06FFF3C22804600238E
:10A04000204629460DF068FF3346CDE9018200978E
:10A05000BAF1000F0BD00A4A1A2148460FF0B8FA9D
:10A06000484604B0BDE8F0874FF0000AC3E7054A50
:10A07000F2E700BF07100020F0C80108805101007E
:10A08000DBC80108DCC801080FB404B07047000049
:10A090000FB437B51B4C256855B90322294601205A
:10A0A00002F070FB2B462A462946206002F08EFB08
:10A0B000154D2B68013B03331ED86421206802F044
:10A0C00073FD8022002111480EF044FB07AB802174
:10A0D000069A0E4801930FF0EBFE7F2803DD0C4932
:10A0E0000C480FF04FFB2B68084898470023206866
:10A0F0001A46194602F06AFB03B0BDE8304004B0CE
:10A10000704700BF901000200810002010100020A1
:10A110001BB601088B1000200FB410B50D4CA2B077
:10A120002368013B033310D825AB8021249A02A871
:10A1300001930FF0BDFE7F2804DD07490DF1830078
:10A140000FF020FB236802A8984722B0BDE810401A
:10A1500004B070470C1000201BB6010870B504460F
:10A16000054E4518AC4200D170BD304614F8011BB5
:10A17000FFF78EFFF6E700BFFCC8010838B50C46B4
:10A180001546FFF785FF20462946FFF7E7FFBDE8A4
:10A1900038400148FFF77CBF89E5010810B5044647
:10A1A00070B102F01FFA204602F00AFA02F0CAF873
:10A1B000BDE81040034A93880133938002F0E0B871
:10A1C00010BD00BF9410002070B5234D04462B68CD
:10A1D0008AB001332B6000283BD0632B1F4E0BDD70
:10A1E00003F0D0FF0523002201A903F0FDFE03F0D8
:10A1F000DFFB002330602B6003F0DAFB336803F5EC
:10A200007A73984204D903F0D3FB002330602B60AB
:10A21000134A144D13781BB92B606B600123137024
:10A2200002F0E0F9204602F0C9F9064668B122467C
:10A2300000210EF08FFA02F085F82B8801332B8075
:10A2400002F09EF830460AB070BD6B8801336B8017
:10A25000F8E70646F6E700BFA0100020A410002093
:10A260009C10002094100020006800BA70470088FD
:10A2700040BA80B2704700687047837842781B0408
:10A28000007843EA02231843704700887047FFF7BD
:10A29000F2BF0370130E4370130C8370130AC37064
:10A2A0000271052070470B0E03700B0C43700B0AF4
:10A2B0008370C170042070470B0A03704170022044
:10A2C00070470B0A017043700B0C090E8370C1704C
:10A2D00004207047A0F14103052B02D83738C0B2E3
:10A2E0007047A0F16103052B01D85738F7E73038E4
:10A2F000C0B20A2828BFFF207047002210B5441EB4
:10A3000021B114F8010F08B1002A01DA104610BD7E
:10A31000FFF7E0FF01390F28C9B202D840EA021264
:10A32000EEE74FF0FF32F1E738B505460C460FF087
:10A330009FF8611B013190FBF1F303FB11002844EE
:10A3400038BD000010B504460FF064F8014B1C60E6
:10A3500010BD00BFB8020020024B18680130186021
:10A360000FF058B8B80200200078013070470FB4E1
:10A3700004B070472DE9FF470D460021DFF8A4A087
:10A3800003AF06469146DAF800003A469846039134
:10A3900002F04AFD0128039B36D14BB14FF0E02378
:10A3A0004FF08052C3F8042DBFF34F8FBFF36F8F70
:10A3B000B5F5C87F88BF4FF4C87531462A461A489C
:10A3C0000EF0A0F9194C184B3946DAF80000A580B8
:10A3D0002360A4F8069084F8088002F009FB039B30
:10A3E0004BB14FF0E0234FF08052C3F8042DBFF380
:10A3F0004F8FBFF36F8F0E48009700230122042177
:10A40000006804F08DF8039B4BB14FF0E0234FF050
:10A410008052C3F8042DBFF34F8FBFF36F8F04B08A
:10A42000BDE8F087AC1200201011002004110020BC
:10A43000B81200200348002301220221006803F023
:10A44000FFBF00BFB81200201FB5002303AA0B48AE
:10A450000092102101220068039304F061F8039B2D
:10A460004BB14FF0E0234FF08052C3F8042DBFF3FF
:10A470004F8FBFF36F8F05B05DF804FBB81200205B
:10A480001FB5002303AA0B48009280210122006817
:10A49000039304F045F8039B4BB14FF0E0234FF0DA
:10A4A0008052C3F8042DBFF34F8FBFF36F8F05B0F9
:10A4B0005DF804FBB81200201FB50346104A10686F
:10A4C000B3B1002303AA009208210122039304F0F0
:10A4D00027F8039B4BB14FF0E0234FF08052C3F8B5
:10A4E000042DBFF34F8FBFF36F8F05B05DF804FBF2
:10A4F0000122082105B05DF804EB03F0A1BF00BF05
:10A50000B81200201FB503F059FA0D4B03AA1860CA
:10A510000092012200230B4811460068039303F0C8
:10A52000FFFF039B4BB14FF0E0234FF08052C3F885
:10A53000042DBFF34F8FBFF36F8F05B05DF804FBA1
:10A54000B4120020B81200201FB500230C4A40218D
:10A55000107003AA0B48009200680122039303F0D5
:10A56000DFFF039B4BB14FF0E0234FF08052C3F865
:10A57000042DBFF34F8FBFF36F8F05B05DF804FB61
:10A58000F4100020B812002000487047EC100020A2
:10A590001248002303224FF4807110B5006803F0C5
:10A5A0004FFF4FF0E0234FF08052C3F8042DBFF36C
:10A5B0004F8FBFF36F8F0A4C206802F081FC40B1CF
:10A5C000BDE81040002307481A461946006802F00B
:10A5D000FDB8012003F044FBEEE700BFB8120020F5
:10A5E000B0120020A8120020F8B5124B01461868DE
:10A5F00002F0DAFA0446D0B14FF0E0254FF0805671
:10A600000D4F002303224FF40071386803F018FF48
:10A61000C5F8046DBFF34F8FBFF36F8F386803F039
:10A6200033F9C5F8046DBFF34F8FBFF36F8F20462A
:10A63000F8BD00BFA8120020B8120020014B18601E
:10A64000704700BFA012002070B5044678B10378AF
:10A65000032B0CD1436853B10025054E1868F269ED
:10A6600090476068F369056098476560257070BD24
:10A67000C810002010B50E480E4C002305222146BC
:10A68000006802F0A3F8012807D1002363600A4B99
:10A690001B6863B1BDE810401847084B2178084893
:10A6A0005B6998472046BDE81040FFF7CDBF10BD5D
:10A6B000A4120020F8100020A0120020C8100020D2
:10A6C00002C901087FB50024094E0022306801A9A3
:10A6D00002F0D8F9651C30B9064B07485B69E1B256
:10A6E000984704B070BD01A8FFF7AEFF2C46ECE719
:10A6F000A4120020C810002029C90108014B1868C5
:10A70000704700BFA412002010B50446064B010A92
:10A71000A3F84A00202000F091FBE1B22120BDE81F
:10A72000104000F08BBB00BFE415002008B5FFF718
:10A73000EBFF0122014B83F8522008BDE4150020F5
:10A74000002238B50B4B05461D200C4683F84C20E3
:10A7500083F84E1000F0CCFB20F0060343EA4401DE
:10A760001D20C9B200F06AFB2946BDE8384023200D
:10A7700000F064BBE415002013B5164C0120A3685B
:10A780009847002341F6FE720093009B934218DD28
:10A79000A36802209847002341F6FE720193019BB3
:10A7A000934212DD0C4BB5211C6C4020A047A02128
:10A7B0004120A04700210120234602B0BDE81040FF
:10A7C0001847009B01330093DFE7019B013301939E
:10A7D000E5E700BFC81000201CCC0108094B07B5F5
:10A7E0001B6CC2213B209847002341F6FE72019367
:10A7F000019B934202DD03B05DF804FB019B013332
:10A800000193F5E71CCC01082DE987488D4B8E4854
:10A810008E4F03608E4B8F4C83608F4B8F4E436007
:10A820008F4BDFF84092C3608F4BDFF840820361AB
:10A830008F4BDFF840A283618F4BC3613B68984721
:10A8400063698E489847002330681A46194601F01C
:10A85000BDFF99F8040068B94FF0FF33194601AA0B
:10A8600003F0A4FD68B9656903F07CFC01468448E7
:10A87000A847EEE741F288334FF0FF31002001AAEC
:10A88000EEE7019BDA0516D500F098FA002000F0FB
:10A89000E9FDFB6A9847FFF715FF63697948984718
:10A8A0000023D8F800001A46194601F08FFF002057
:10A8B00003F054FACDE79B0510D500F07FFAFFF7BF
:10A8C0008DFFFB6A9847FFF7FDFE63696E48984766
:10A8D0006421D8F8000002F067F9BAE7D8F8000060
:10A8E00002F0EEFA012803D1636968489847B0E79F
:10A8F000DAF8003023B94FF4B5716548FBF73CFE38
:10A90000019B1D0604D50722624B1A70FFF7B2FEA9
:10A91000019B580750D50021306802F045F9012805
:10A920004AD10C20A3699847054688B90C21636970
:10A93000594898472B462A462946306801F046FF79
:10A94000002886D140F27F115148FBF715FE80E7C1
:10A95000524BA269988880B29047504B834698B971
:10A9600099884F4889B2636998472846E3699847B0
:10A970005B465A465946306801F028FF00287FF4AC
:10A9800068AF40F28711DFE71A1D03CAC5F800B0AF
:10A990006860A96019689A88584692B20DF0B2FEB4
:10A9A00003223C4B1A705D60FFF764FE00233068A1
:10A9B0001A46194601F00AFF019BD90709D5012261
:10A9C000344B1A7000225A60364A12689A60FFF7B8
:10A9D00051FE019BDB0606D505222E4B1A70002284
:10A9E0005A60FFF747FE019B1D0706D50422294B3D
:10A9F0001A7000225A60FFF73DFE019B980706D5AA
:10AA00000222244B1A7000225A60FFF733FE019B8A
:10AA1000990606D506221F4B1A70234A5A60FFF783
:10AA200029FE019B5B067FF514AF204B1B78002BA2
:10AA300014BF08220922174B1A7000225A60FFF730
:10AA400019FE06E705A50008A81000201CCC010887
:10AA500075A30008C810002035A40008AC1200201F
:10AA6000B9A40008EC10002049A40008B01200208E
:10AA700049A50008A412002081A400085AC90108B1
:10AA800070C901088EC90108B6C90108CDC90108FD
:10AA90008AE50108F8100020E3C90108041100202C
:10AAA00019CA0108B4120020F5100020F41000208B
:10AAB000044B10B55B6998470446FFF75DFE2046DE
:10AAC00010BD00BF1CCC0108F0B5724C05462646EF
:10AAD0000F460FCD0FC695E80F0086E80F0097E8E8
:10AAE000030063696C4E013B033388BF6B4B254603
:10AAF00088BF6361636886E80300013B033385B068
:10AB000007D96748636998474FF430716548FBF788
:10AB100033FD2368013B033307D9634863699847D2
:10AB20004FF431715F48FBF727FDA368013B033306
:10AB300007D95E48636998474FF432715948FBF76B
:10AB40001BFDE368013B033307D959486369984704
:10AB50004FF433715348FBF70FFD2369013B033377
:10AB600007D95448636998474FF434714D48FBF74F
:10AB700003FDE369013B033304D94FF435714948C0
:10AB8000FBF7FAFCA369013B033304D94FF4367198
:10AB90004448FBF7F1FC484B0FCB8DE80F0095E8DC
:10ABA0000F0000F0E1F823689847FFF7E5FD434BFD
:10ABB00042205B6C98472228014663693FD1404898
:10ABC000984703220021012001F0DCFD3D4B186075
:10ABD000012001F0A1FE3C4B186020B94FF43D71FB
:10ABE0003048FBF7C9FC03220021012001F0CAFD17
:10ABF000364D286020B94FF43E712A48FBF7BCFC63
:10AC0000002328681A46194601F0E0FD20B940F2F9
:10AC1000F9212448FBF7B0FC4FF0FF31286801F020
:10AC2000C3FF00220C21032001F0ACFD284B18606B
:10AC300078B963692748984740F2FF2103E0264826
:10AC4000984740F2EA211748FBF796FC002005B030
:10AC5000F0BD224B224A1A6033680BB904233360DB
:10AC6000204B1D680DB10120F1E701933368FA22F2
:10AC700000931D4901231D4802F062FC0128F2D017
:10AC800063691B489847074840F21131FBF774FC91
:10AC90002846DCE7C8100020EC1000206FA3000855
:10ACA00051CA01088AE5010892CA0108C9CA010807
:10ACB00001CB01083ACB0108D81000201CCC0108B8
:10ACC00076CB0108AC120020A8120020B0120020A0
:10ACD000A4120020A8CB01088DCB0108E8100020A9
:10ACE00069A30008B8120020DCCB010809A80008FD
:10ACF000E4CB010870B5084E044633680D4623B90D
:10AD000040F221310548FBF737FC294620463368DD
:10AD1000BDE87040184700BFE81000208AE5010830
:10AD200000F03CB80120704708B5FFF72DFC4379CF
:10AD3000002B0CBF8020002008BD0000094B002222
:10AD4000194610B51C68844202D89C68844205D814
:10AD50000132152A03F10803F4D1FEE701EBC20228
:10AD6000107910BDB0CC010884B030B503AC84E8D4
:10AD70000F00064C03AD0FCD0FC495E80F0084E81B
:10AD80000F00BDE8304004B0704700BF48160020F7
:10AD9000014B1878704700BFE4150020C82307B5A1
:10ADA0000093002304481A460321006803F0E6FCE0
:10ADB00003B05DF804FB00BFC012002013B5104CB7
:10ADC0000120A368984700230093009BB3F5CC7F34
:10ADD0000FDDA36800209847002342F6FE7201931E
:10ADE000019B934208DD0220A36802B0BDE8104039
:10ADF0001847009B0133E7E7019B01330193EFE71D
:10AE0000481600202DE9F04107460B4E0020F3685C
:10AE10000C4615469847336947F08000984725440B
:10AE2000AC4204D1F3680120BDE8F0411847336912
:10AE300014F8010B9847F3E74816002007B50122E4
:10AE40008DF807100DF10701FFF7DCFF03B05DF887
:10AE500004FB000000000000134A10B55060134AC4
:10AE6000904219D00CF0BAF90DA3D3E900230CF0ED
:10AE700059FB0CF0C7FC0446C4F307410620FFF75A
:10AE8000DDFFC4F307210720FFF7D8FFE1B2082058
:10AE9000BDE81040FFF7D2BF054CEDE7AFF30080EF
:10AEA0000000000080844E40E4150020F01FCB33EA
:10AEB000CD3CD9002DE9F04107460C4E0020F36847
:10AEC0000C4615469847336907F07F00984725449C
:10AED000AC4204D1F3680120BDE8F04118470020DE
:10AEE0003369984704F8010BF2E700BF48160020C9
:10AEF00007B501220DF10701FFF7DCFF9DF8070000
:10AF000003B05DF804FB000001282DE9F0478846F6
:10AF100004D0022854D00020BDE8F087704D2720CF
:10AF2000AC8BFFF7E5FFA4B220F0F8000134204419
:10AF30000CF054F9AB7F0022002B3CD1694B0CF094
:10AF400011F8064630200F46FFF7D2FF30F0F90324
:10AF50000CBF0023634B0022304639460CF002F848
:10AF6000064640460F460CF049F902460B4630466D
:10AF700039460BF0F7FF95F820300022EBB900239B
:10AF80000BF0F0FF0022584B0CF0A2F9AE6904461A
:10AF900030460D460CF022F902460B462046294663
:10AFA0000CF0C0FA0022514B0CF092F90BF088FF24
:10AFB0000CF028FCB0E70023C1E74FF08043DFE747
:10AFC000DFF81CA1DAF84020022A00F28280484B08
:10AFD00003EBC203D3E900450120DAF8443098407E
:10AFE0000CF00CF902460B46204629460CF09AFA62
:10AFF00002460B4600203B490CF094FA04460D46ED
:10B00000BAF84A0080B20CF0F9F80022394B0BF084
:10B01000A9FF22462B460CF05BF9DAF844300F46C4
:10B020009AF84E109AF84C200646002A14BF1420B5
:10B0300000209B00C3F11C0303EB011303EBC803C7
:10B04000181A0CF0CBF88046DAF844009AF8483029
:10B050008946002B14BF02230023C3EB80000CF0B1
:10B06000BDF802460B46404649460CF05BFA0BF031
:10B070002FFE804689469AF8490004300CF0BEF84D
:10B0800042464B460CF024F90022002380468946B4
:10B090000CF0AEFB18B94FF000084FF00009002289
:10B0A00040464946104B0BF05DFF22462B460CF004
:10B0B0000FF932463B460BF055FF00220B4B0CF0CC
:10B0C00007F905A3D3E900230BF04CFF0BF07CFE3E
:10B0D0006EE7002400257FE72B8716D9CEF7EF3FD8
:10B0E000E41500200000F03F0000204000408F40A9
:10B0F00098CC010800001140012808B504D00228AE
:10B100000AD04FF0FF3008BD1120FFF7F1FEC0F369
:10B110004700404200B2F6E71B20FFF7E9FE8B38FC
:10B12000F8E700000B4B10B55B68044660B90220DD
:10B1300098470120FFF7DCFE00F0F80121430120D1
:10B14000BDE81040FFF77ABE03280CBF01200020A5
:10B15000EEE700BF4816002013B5C82400230B48B3
:10B1600000941A460321006803F008FB00230848F6
:10B1700000941A460321006803F000FB0020FFF74B
:10B18000D1FF0022034B1A7002B010BDC012002084
:10B1900044160020E415002013B5C82400230B48F2
:10B1A00000941A460321006803F0E8FA00230848D7
:10B1B00000941A460321006803F0E0FA0120FFF72B
:10B1C000B1FF0022034B1A7002B010BDC012002064
:10B1D00044160020E415002073B5594C06466378E8
:10B1E000012BDAB22FD0022A5DD000254FF4C872AD
:10B1F000002154480DF0AEFA01232370524B186819
:10B200004FF0FF33002E00F08D804FF47A7101FB78
:10B2100006F20093B2FBF1F20023042103F0AEFA30
:10B220006378012B40F083800520FFF77BFF0D2022
:10B23000FFF75EFE40F020010D20C9B202B0BDE86C
:10B240007040FFF7FBBD402094F82250FFF750FEFE
:10B250000C214020FFF7F2FD4120FFF749FE60F08E
:10B260000E01C9B24120FFF7E9FD3520FFF740FE8E
:10B2700000F03F00112184F83A003F20FFF7DEFD87
:10B2800000230D2084F82C3084F82D302387E386AA
:10B29000FFF72EFE00F04001EDB241F02E010D202F
:10B2A000FFF7CCFDA2E794F8513033201BB3FFF732
:10B2B0001FFE40F04101C9B23320FFF7BFFD192145
:10B2C0003B20FFF7BBFD94F8525094F84F30EDB29D
:10B2D000E3B11D211120FFF7B1FD4020FFF708FE6B
:10B2E00000F033014020FFF7A9FD00210F20FFF7F8
:10B2F000A5FD0021D3E7FFF7FBFD00F0BE0141F003
:10B3000001013320FFF79AFD1D21D9E70F211120FC
:10B31000FFF794FD4020FFF7EBFD00F03C0141F00A
:10B320000101DFE7009332463346032176E72DB172
:10B33000052002B0BDE87040FFF7F4BE0620F8E734
:10B34000E4150020C4120020C012002037B54FF4CD
:10B350007A72642350432B4DB0FBF2F20093042128
:10B360000023286803F00AFA0022274B274C1A70A2
:10B370006378012BDAB214D0022A26D0022323707C
:10B380002C6802F015FB05230246009301210023DF
:10B39000204603F0F3F9032003B0BDE83040FFF787
:10B3A000C1BE14214020FFF749FDB0214120FFF725
:10B3B00045FD8F213520FFF741FD3520FFF798FD32
:10B3C00000F03F0084F83A00D8E794F84F3073B1AA
:10B3D000F5211120FFF732FD4020FFF789FD00F035
:10B3E0003301402041F04001FFF728FDC6E7F72177
:10B3F0001120FFF723FD4020FFF77AFD00F03F0109
:10B40000EFE700BF4416002068160020E415002076
:10B4100010B5124C6378012BDAB204D0022A09D09D
:10B4200040F2164101E040F2FF31BDE810400C4807
:10B43000FBF7A2B8FA211120FFF700FD4020FFF72B
:10B4400057FD00F0FC014020FFF7F8FC0323072024
:10B450002370BDE81040FFF765BE00BFE415002073
:10B460008AE5010808B51A4B5A7882422ED05870E6
:10B470005B780020022B13D0FFF754FE0120FFF76A
:10B4800037FD00F07F010120FFF7D8FC00214020AC
:10B49000FFF7D4FC30214120BDE80840FFF7CEBCC7
:10B4A000FFF740FE0120FFF723FD60F07F01C9B2E6
:10B4B0000120FFF7C3FC00214020FFF7BFFC002163
:10B4C0004120FFF7BBFC43213120E5E708BD00BF69
:10B4D000E41500201D4B13B5186000231C4C1A46C0
:10B4E0004FF47A711B48009403F026F91A4B186048
:10B4F00020B94FF486711948FBF73EF800234FF44A
:10B500007A711A461648009403F016F9154B186024
:10B5100020B94FF487711148FBF72EF8FFF74EFC66
:10B520000020FFF79FFF0020FFF7FCFD4FF4C872DB
:10B5300000210D480DF00EF9002201210B4B83F87C
:10B54000282083F829101A7002B010BDBC12002008
:10B55000F5BA000870CC0108441600208AE50108FD
:10B5600073CC0108C0120020C4120020E415002092
:10B5700073B50E4614460546FFF774FF3046FFF7D5
:10B580006BFC0520FFF7CEFD00230193019BB3F573
:10B59000CC7F0BDD2846FFF7AFFD0546FFF7DCFD4E
:10B5A000A542CCBF0020012002B070BD019B013339
:10B5B000EBE773B500240220FFF754FFFF211120B1
:10B5C000FFF73CFC0520FFF7ADFD2546264601961A
:10B5D000019BB3F5CC7F0DDD2C20FFF789FC00F03B
:10B5E0000100A0400134202C45EA0005EFD1284697
:10B5F00002B070BD019B01330193E9E70000000038
:10B600002DE9F04F834687B00093109B0E460193BF
:10B610009DF85C309DF86010029315469DF86430EB
:10B620009DF8582004910393BDF84470BDF848403C
:10B630009DF84C809DF850909DF854A00592FFF71E
:10B6400011FFDDE90331BBF1010F06D0BBF1020FA1
:10B65000059A66D007B0BDE8F08F7D4C019A26614F
:10B660002846A561626184F81E8084F81F9084F8E2
:10B6700020A084F8211084F82230A7830BF0AEFDBF
:10B680000B46024670A1D1E900010BF04BFF0CF014
:10B69000B9F8C0F3072185B20220FFF7CFFBE9B26A
:10B6A0000320FFF7CBFB3046FFF748FB0146122093
:10B6B000FFF7C4FB0198FFF741FB01461320FFF79A
:10B6C000BDFB2520390AFFF7B9FB2620F9B2FFF7A9
:10B6D000B5FBE37FE3B9A37FD3B184F829B0494632
:10B6E0003220FFF7ABFB3020FFF702FCB8F1000F70
:10B6F00014BF0021802100F06F0040EA0A1A3020B8
:10B7000041EA0A01C9B207B0BDE8F04FFFF796BBA6
:10B7100000234FF4D2714F4884F82930FAF72CFFF8
:10B72000DDE7DFF82CB10098CBF84060CBF844504F
:10B730008BF84900ABF84A708BF84C808BF84D9031
:10B740008BF84EA08BF84F20029A062D8BF85020D4
:10B750002A4638BF06220C2A8BF8511028BF0C222B
:10B760008BF85230002E5CD1A2F10B03012B5CD878
:10B7700001238BF848301D200192FFF7B9FB9BF89D
:10B780004810009B41EA4A0141EA880141EAC301AD
:10B7900041EA8611C9B21D20FFF750FB1E20FFF7BA
:10B7A000A7FB019AC4F3012141EA021200F00C0048
:10B7B0000243D1B21E20FFF741FB1F20E1B2FFF789
:10B7C0003DFB2020390AFFF739FB2120F9B2FFF7B2
:10B7D00035FBB8F1000F03D049462220FFF72EFBBE
:10B7E0009BF84F306BB14B20FFF782FB60F07F017D
:10B7F000C9B24B20FFF722FB24209BF85010FFF723
:10B800001DFB062D4FF0310011D8FFF771FB00F042
:10B81000F80141F005013120FFF710FB0C21372022
:10B8200071E7012E01D10B2DA2D80023A1E7FFF76C
:10B830005FFB00F0F80141F003013120FFF7FEFA51
:10B840000A21ECE7AFF300800000000080847E4115
:10B85000E41500208AE501082DE9F04F89B01D4666
:10B860009DF84C30079101939DF85C30924604930B
:10B870009DF86030009005939DF86430129E02930D
:10B880001A9BBDF8507003939DF854809DF8589012
:10B89000FFF7E8FD0920FFF72BFB04465A20FFF7CE
:10B8A00027FB04F07F03924C834660680693FFF702
:10B8B0003BFA069B0799034313F0800F03F0F00C4B
:10B8C00029D011291DDD14290B46A8BF14234BF0E4
:10B8D00007025FFA82FB591F4CEA01010920C9B235
:10B8E0000693FFF7ABFA59465A20FFF7A7FA009BD9
:10B8F000012B069B17D0009A022A6AD009B0BDE836
:10B90000F08F02290B46B8BF02230BF0F80242F079
:10B91000040B991EE0E70E290B46A8BF0E2343EA4D
:10B92000E373591CD8E72372029BC4F80CA025616D
:10B93000A661A78384F81E8084F8209084F82130C3
:10B94000039B504663620BF049FC65A3D3E90023D7
:10B950000BF0E8FD0BF056FF84B2C0F30721042082
:10B96000FFF76CFAE1B20520FFF768FA30460BF0FA
:10B9700035FC02460B465CA1D1E900010BF0D2FD7B
:10B980000BF040FFC0F3072184B20220FFF756FA04
:10B990000320E1B2FFF752FA2520390AFFF74EFAE9
:10B9A000F9B22620FFF74AFA3020FFF7A1FAB8F1E2
:10B9B000000F14BF0021802100F06F0040EA091938
:10B9C000302041EA0901C9B209B0BDE8F04FFFF7E4
:10B9D00035BA062EB24638BF4FF0060A84F83C301E
:10B9E000019B2564666484F84930049BA4F84A707E
:10B9F00084F84C8084F84F30059BBAF10C0F84F822
:10BA00005030029B84F84E9084F85130039B28BF3D
:10BA10004FF00C0ADFF8D8B06365002D4CD1AAF1C5
:10BA20000B03012B4CD801238BF848309BF84F3087
:10BA30006BB14B20FFF75CFA60F07F01C9B24B207D
:10BA4000FFF7FCF924209BF85010FFF7F7F91D20B1
:10BA5000FFF74EFA94F84810019B41EA490141EA88
:10BA6000880141EAC30141EA8511C9B21D20FFF7EF
:10BA7000E5F91E20FFF73CFA00F00F0141EA0A1138
:10BA80001E20C9B2FFF7DAF92020390AFFF7D6F9EC
:10BA90002120F9B2FFF7D2F9062E4FF0310011D86C
:10BAA000FFF726FA00F0F80141F005013120FFF719
:10BAB000C5F90C21372087E7012D01D10B2EB2D813
:10BAC0000023B1E7FFF714FA00F0F80141F0030199
:10BAD0003120FFF7B3F90A21ECE700BFAFF3008094
:10BAE0000000000080844E400000000080847E4101
:10BAF000E415002010B5254C2378012BDAB202D0D2
:10BB0000022A34D010BD6378012B29D100230B21E8
:10BB10003E2084F82C3084F82D302387E386FFF70D
:10BB20008DF910213F20FFF789F994F8223003F0B6
:10BB3000FF029BB10D20FFF7DBF940F02001C9B2F5
:10BB40000D20FFF77BF9124B1B68002BDAD0DB6866
:10BB5000002BD7D0BDE81040002018472270F2E734
:10BB600094F85230002BEED0FFF716FBEBE70023E2
:10BB700001222370074B1A70054B1B68002BC1D0A4
:10BB80005B68002BBED0BDE810401847E4150020CC
:10BB9000BC1200206816002007B50022154B8DF856
:10BBA000072083F82C2083F82D201A87DA8683F863
:10BBB0002E2093F8223023B903B05DF804EBFFF791
:10BBC000CBBA3F20FFF794F98DF807009DF80730B6
:10BBD000DB0603D510213F20FFF730F90D20FFF7DA
:10BBE00087F940F040010D20C9B203B05DF804EBC5
:10BBF000FFF724B9E41500202DE9F04107460C4E6B
:10BC00000020F3680C4615469847336907F07F001B
:10BC100098472544AC4204D1F3680120BDE8F041C7
:10BC20001847002033699847C04304F8010BF1E737
:10BC3000481600200A4601460020FFF7E3B800003E
:10BC4000F7B5584C064663780D46012BDAB212D090
:10BC5000022A36D000252846FFF778FB6378012BAF
:10BC600040F09E80002D00F09B804F4E4F4D33786A
:10BC7000002B69D094E0002323878BB2E386A37F57
:10BC800013B13220FFF7DAF86B1E3F2B0FD884F880
:10BC90003B500025304694F83B10FFF7CBFF94F85B
:10BCA0003B30228F13449BB22387606AD4E72A4635
:10BCB00031463E480CF026FD3C23012584F83B30FC
:10BCC000E8E794F8513033202BB3FFF711F900F077
:10BCD000BE013320FFF7B2F819213B20FFF7AEF881
:10BCE0002946222084F85C50FFF7A8F800210E2096
:10BCF000FFF7A4F800210D20FFF7A0F80120FFF7BF
:10BD0000F7F830F0F80711D029463046FFF792FFD8
:10BD10000025606DA0E7FFF7EBF800F0BE0141F0F1
:10BD200001013320FFF78AF81D21D6E7FFF734FA27
:10BD30000197019BB3F5CC7FE6DC019B01330193B6
:10BD4000F7E7012001F08CFF3F20FFF7D1F88306D1
:10BD5000F7D4E38E228F9BB294F83B1092B2208FDF
:10BD60009B1A8B4280B20BDD94F83B102844FFF7FE
:10BD700061FF94F83B30228F13449BB2238776E710
:10BD8000E18E238F2844C91AC9B2FFF753FFE38E0F
:10BD9000218F228F9BB292B213445B1A9BB22387EE
:10BDA00003B0F0BDE415002068160020C412002086
:10BDB0000A4601460020FFF77DB80A4601460020EA
:10BDC000FFF71ABF38B505460C46FFF74BFB012DB0
:10BDD00002D0022D0AD038BD064B9B7F002BFAD132
:10BDE00021463220BDE83840FFF728B821462320FD
:10BDF000F8E700BFE41500207FB50022694C8DF8FC
:10BE00000B2023780392012BD9B204D0022900F031
:10BE1000A68004B070BD6378012BDAB236D0022A56
:10BE2000F7D140211220FFF709F81220FFF760F840
:10BE30008DF80B009DF80B305B4E13F0200F2BD0CC
:10BE400020211220FEF7FAFF94F8523003F0FF028F
:10BE500003B9227000225548009203AB0821006804
:10BE600002F08CFC039B4BB14FF0E0234FF080526B
:10BE7000C3F8042DBFF34F8FBFF36F8F3368002BD0
:10BE8000C7D01B69002BC4D09847C2E740F22151AC
:10BE90004748FAF771FBBCE71920FFF729F840B2D1
:10BEA00084F8580094F8583094F858501B0642BF54
:10BEB0006DB26D42C5F385054FF01A004CBF6D425F
:10BEC000AD08FFF715F8002DB8BF2D1840F30B1380
:10BED000B4BF8B3D8B389BB2ACBF1B185B191BB238
:10BEE0001320A4F85A30FFF703F884F85C00102000
:10BEF000FEF7FEFF01460D20FEF7A0FF94F85C1050
:10BF00002C48FFF755FF94F8523003F0FF029BB91D
:10BF10002648009203AB08210068227002F02EFC34
:10BF2000039B4BB14FF0E0234FF08052C3F8042D38
:10BF3000BFF34F8FBFF36F8F3368002B3FF469AFB0
:10BF40009D68002D3FF465AF94F85C10B4F85A205A
:10BF500094F8583017485BB212B2A84759E7134813
:10BF6000009203AB0821006802F008FC039B4BB170
:10BF70004FF0E0234FF08052C3F8042DBFF34F8FF2
:10BF8000BFF36F8F6378022B03D108211220FEF7D5
:10BF900055FF00232370044B1B68002B3FF439AF7F
:10BFA0001B686FE7E4150020BC120020C0120020BF
:10BFB0008AE50108C41200202DE9FF4100256C4CE0
:10BFC0008DF80B5023780395012BDAB205D0022AA5
:10BFD00000F0CC8004B0BDE8F0816378012BDAB2C8
:10BFE00025D0022AF6D16348009503AB2A460821E2
:10BFF000006802F0C3FB039B4BB14FF0E0234FF00E
:10C000008052C3F8042DBFF34F8FBFF36F8F802191
:10C010001220FEF713FF00232370574B1B68002BE1
:10C02000D8D0DB68002BD5D001209847D2E73F203D
:10C03000FEF75EFF8DF80B009DF80B309A06C9D510
:10C040009DF80B30DB0619D5E18E228F4B4892B25A
:10C0500089B2FEF761F84A4E4A4F94F83A30AB4243
:10C0600005DC4948FEF758F8FFF796FDB2E7384679
:10C0700016F8011BFEF750F80135EEE794F8293069
:10C0800023B940F2D5514148FAF776FA94F82830AE
:10C09000022B3CD1238F3A489BB294F83A101844B3
:10C0A000FFF78BFE238F9BB2002B4BD094F83A30D6
:10C0B000228F13449BB22387228FE38E92B29BB2CE
:10C0C0009A4287D32E4DE28E294692B230480CF028
:10C0D00019FBFF232B7011236B70DD23AB70EE2354
:10C0E000EB7094F82E50E48EFFF756FD224B6DB2A4
:10C0F0001B68A4B2002B3FF46DAF9E68002E3FF486
:10C1000069AF00232A4621462148B04762E7214F04
:10C110000020FB68984700203B6998470026DFF81D
:10C12000608094F83A30B34203DC0120FB68984702
:10C13000B8E700203B69258F9847ADB24544A85524
:10C140000136EEE794F82D30002B8DD094F83A109C
:10C150000B48FEF7CFFDE086E38E9BB2B3F5C87FB8
:10C1600082D2E38E9BB2002BA0D17DE7637831E7CA
:10C17000E4150020C0120020BC12002076CC01087B
:10C18000C41200208BCC010889E501088AE501086A
:10C19000541400204816002010B51B4C2378012BA6
:10C1A000DAB202D0022A2AD010BD6378012BD9B2AC
:10C1B00018D00229F8D194F84F30002BF4D0122077
:10C1C000FEF73CFE114B1B68002BEDD05C69002C88
:10C1D000EAD01C20FEF78CFE2346BDE8104000F09C
:10C1E0003F00184700231120238784F82D10FEF705
:10C1F0007FFE4008404240B284F82E00D4E76378C6
:10C20000D9B2022BD6E700BFE4150020BC120020F3
:10C2100070B51F4B5A78022A05D11B78012BDAB270
:10C2200002D0032A13D070BD1220FEF761FEC306B0
:10C23000F9D510211220FEF701FE164B1B68002BCA
:10C24000F1D0DB69002BEED0BDE87040184712201A
:10C25000FEF74EFE10F001040E4D0DD00521122008
:10C26000FEF7ECFD2B68002BDDD09B69002BDAD0AC
:10C270000120BDE87040184704211220FEF7DEFDC2
:10C280002B68002BCFD09B69002BCCD02046F0E749
:10C29000E4150020BC12002006480068006880F306
:10C2A000088862B661B6BFF34F8FBFF36F8F00DFB0
:10C2B00000BF000008ED00E0002307B501930B4B21
:10C2C0001B68013303D0CA210948FAF755F94FF02A
:10C2D000500383F31188BFF36F8FBFF34F8F019B20
:10C2E000002BFCD003B05DF804FB00BFBC020020B3
:10C2F0008AE501084FF0807340F8043C054B21F0BB
:10C30000010140F8081C40F80C3C40F8202C403853
:10C31000704700BFB9C20008000000000000000024
:10C32000074B19680868B0E8F00F80F30988BFF37D
:10C330006F8F4FF0000080F311884EF00D0E7047A4
:10C340009C1600204FF0500383F31188BFF36F8FCA
:10C35000BFF34F8F084A13680133012B13600AD1D2
:10C360004FF0E023D3F8043DDBB223B140F2751166
:10C370000248FAF701B97047BC0200208AE50108BB
:10C3800010B5074C236823B94FF4BE710548FAF77E
:10C39000F3F82368013B23600BB983F3118810BDC8
:10C3A000BC0200208AE50108000000000000000037
:10C3B000EFF30980BFF36F8F0D4B1A6820E9F00F80
:10C3C00010602DE908404FF0500080F3118801F013
:10C3D0006DFC4FF0000080F31188BDE8084019683B
:10C3E0000868B0E8F00F80F30988BFF36F8F7047DB
:10C3F0009C16002008B54FF0500383F31188BFF35B
:10C400006F8FBFF34F8F01F0E7FA28B14FF0E023B1
:10C410004FF08052C3F8042D002383F3118808BD28
:10C420004FF0E02300221A619A6141F267025A61DB
:10C4300007221A617047000013B5284B284C1A7860
:10C44000D2B20192FF221A701B78264ADBB28DF815
:10C4500003309DF8033003F05003137007230022CC
:10C4600023609DF80310581E09062DD412B1032B2A
:10C47000236004D04FF49B711B48FAF77DF82368C2
:10C48000164A1B0203F4E0632360019B0024DBB225
:10C4900013704FF0E023D3F8202D42F47002C3F85C
:10C4A000202DD3F8202D42F07042C3F8202DFFF745
:10C4B000B7FF0E4B1C60FFF7EFFE01F0F7FBFFF735
:10C4C000FBFE204602B010BD9DF8033001225B0048
:10C4D000DBB28DF803300346C3E700BF00E400E0A1
:10C4E0006C160020691600208AE50108BC020020B5
:10C4F00008B5EFF305830F2B0AD90E4A9B5C0E4A51
:10C5000012789A4204D940F2A5210C48FAF734F87F
:10C510004FF0E0230A4AD3F80C3D126803F4E063BD
:10C52000934206D9BDE8084040F2B5210348FAF726
:10C5300023B808BDF0E300E0691600208AE5010891
:10C540006C16002070B50C46064601F029FA0D4B1A
:10C550000D491D682A198A4207D90C23336001F05E
:10C56000CBFA4FF0FF35284670BD1A60074A1368B2
:10C570001B1B1360064B19682144196001F0BCFABB
:10C58000F1E700BFC0020020746E0020C40200204A
:10C590007016002008B5EFF305831BB1C2210348D4
:10C5A000F9F7EAFFBDE8084001F0FAB98AE50108A9
:10C5B00001F0A2BA01F0F4B901F09EBA0CF074B81F
:10C5C0000CF07AB800B58BB068460CF03DFB034B1D
:10C5D00008981B6818440BB05DF804FBC4020020E7
:10C5E000002070477047000000487047741E00200C
:10C5F00010B50446FFF7A6FEA46BFFF7C1FEB4FA20
:10C6000084F0400910BDF8B51546026C0446866BEF
:10C6100052B9076847BB806801F01CFE0546A76059
:10C6200001362846A663F8BD65B940680CF06AF883
:10C630006368226C1344A26863609342F0D323685A
:10C640006360EDE7C0680CF05DF8226CE36851426E
:10C650009B1A2268E36093423EBFA3685B18E360C5
:10C66000022D01D116B1013E0025D9E73546D7E7A5
:10C6700003461A6C084610B462B1DC689968144429
:10C680008C4228BF1968DC6028BFD960D96810BC0B
:10C690000CF038B810BC704770B50446FFF752FE76
:10C6A00094F8455004F124066DB2002D14DCFF23EC
:10C6B00084F84530FFF764FEFFF744FE94F84450D9
:10C6C00004F110066DB2002D12DCFF2384F8443013
:10C6D000BDE87040FFF754BE636A002BE7D03046D8
:10C6E00001F0E0FB08B101F079FC013D6DB2DCE73F
:10C6F0002369002BE9D0304601F0D4FB08B101F0EA
:10C700006DFC013D6DB2DEE738B50D46044620B93B
:10C7100040F203111A48F9F72FFFFFF713FED4E98F
:10C720000F314B432268D0185B1A1344A060E360BA
:10C730000020FF23A063626084F8443084F8453011
:10C74000A5B9236973B104F1100001F0ABFB48B146
:10C750004FF0E0234FF08052C3F8042DBFF34F8F0A
:10C76000BFF36F8FFFF70CFE012038BD04F11000FE
:10C7700002F056F904F1240002F052F9F2E700BF8A
:10C780008AE50108F8B50D461746064620B94FF46C
:10C79000BB710D48F9F7F0FE05FB06F05030FFF7CE
:10C7A0000DFF044658B165B100F150030121204648
:10C7B000C4E90F652360FFF7A7FF84F84C7020469B
:10C7C000F8BD0346F2E700BF8AE501082DE9F04312
:10C7D00085B00F461E460446019220B940F2F12171
:10C7E0004C48F9F7C9FE37B9236C23B140F2F22166
:10C7F0004848F9F7C1FE022E07D1E36B012B04D0A4
:10C8000040F2F3214348F9F7B7FE01F0C1FC30B91B
:10C81000019B23B140F2F6213E48F9F7ADFE4FF0FF
:10C820000008C146FFF78EFDA26BE36B9A4201D36D
:10C83000022E1BD1324639462046FFF7E4FE636ADA
:10C840001BB104F1240001F02DFB48B14FF0E023AF
:10C850004FF08052C3F8042DBFF34F8FBFF36F8F9B
:10C86000FFF78EFD012005B0BDE8F083019D1DB9E5
:10C87000FFF786FD0020F6E7B8F1000F02D102A80D
:10C8800001F06AFBFFF77CFD01F08AF8FFF75AFD23
:10C8900094F84430FF2B08BF84F8449094F8453056
:10C8A000FF2B08BF84F84590FFF76AFD01A902A895
:10C8B00001F05EFB40BBFFF745FDA26BE36B9A42C4
:10C8C0000FD1FFF75DFD019904F1100001F0B0FAFE
:10C8D0002046FFF7E1FE01F00FF950B14FF00108DB
:10C8E000A0E7FFF74DFD2046FFF7D6FE01F004F963
:10C8F000F4E74FF0E0234FF08052C3F8042DBFF36C
:10C900004F8FBFF36F8FE9E72046FFF7C5FE01F0B9
:10C91000F3F8AFE78AE50108024610B500210120CF
:10C92000FFF730FF044638B100231A4619468360EA
:10C930000360C360FFF74AFF204610BD2DE9F843AE
:10C94000894690461F46044620B940F2C331274825
:10C95000F9F712FEB9F1000F06D1236C23B14FF4A1
:10C9600071712248F9F708FE022F07D1E36B012B02
:10C9700004D040F2C5311D48F9F7FEFDFFF7B8FDC0
:10C98000EFF311864FF0500383F31188BFF36F8FDD
:10C99000BFF34F8FA26BE36B9A4201D3022F22D1D8
:10C9A00094F845503A46494620466DB2FFF72BFEB3
:10C9B0006B1C13D1636A0BB901200BE004F1240056
:10C9C00001F070FA0028F7D0B8F1000FF4D0012080
:10C9D000C8F8000086F31188BDE8F88301356DB210
:10C9E00084F84550E8E70020F4E700BF8AE5010835
:10C9F00070B50D46044620B94FF48C612048F9F714
:10CA0000BBFD236C23B140F264411D48F9F7B4FD2E
:10CA1000236833B9A36823B140F269411848F9F794
:10CA2000ABFDFFF765FDEFF311864FF0500383F385
:10CA30001188BFF36F8FBFF34F8FA26BE36B9342ED
:10CA40001CD994F845100132FF294BB2A26310D1D2
:10CA5000636A0BB9012009E004F1240001F022FA15
:10CA60000028F7D0002DF5D00120286086F311882A
:10CA700070BD01335BB284F84530EBE70020F5E789
:10CA80008AE501082DE9FF410E460446019220B9CE
:10CA90004FF4A0614348F9F76FFD36B9236C23B119
:10CAA00040F204513F48F9F767FD01F071FB30B9DE
:10CAB000019B23B140F209513A48F9F75DFD002787
:10CAC000B846FFF73FFCA56BE5B131462046013D76
:10CAD000FFF7CEFDA563236973B104F1100001F0E7
:10CAE000E1F948B14FF0E0234FF08052C3F8042D34
:10CAF000BFF34F8FBFF36F8FFFF742FC012004B0ED
:10CB0000BDE8F081019D1DB9FFF73AFC0020F6E772
:10CB100017B902A801F020FAFFF732FC00F040FF3D
:10CB2000FFF710FC94F84430FF2B08BF84F84480D2
:10CB300094F84530FF2B08BF84F84580FFF720FCB0
:10CB400001A902A801F014FA00BB2046FFF750FD2E
:10CB5000B0B1019904F1240001F06AF92046FFF711
:10CB60009BFD00F0C9FF48B94FF0E0234FF0805221
:10CB7000C3F8042DBFF34F8FBFF36F8F0127A0E7DA
:10CB80002046FFF789FD00F0B7FFF7E72046FFF7E3
:10CB900083FD00F0B1FF2046FFF72AFD0028EDD00D
:10CBA000B4E700BF8AE50108F0B585B004460191FD
:10CBB00020B940F291515248F9F7DEFC236C23B1C1
:10CBC00040F295514E48F9F7D7FC01F0E1FA30B93F
:10CBD000019B23B140F29A514948F9F7CDFC002559
:10CBE0002F462E46FFF7AEFBA36BEBB1013BA363D1
:10CBF000236813B901F0CEFBA060236973B104F17F
:10CC0000100001F04FF948B14FF0E0234FF080528F
:10CC1000C3F8042DBFF34F8FBFF36F8FFFF7B0FB47
:10CC20000125284605B0F0BD019B4BB925B140F266
:10CC3000E1513348F9F7A0FCFFF7A2FB0025F0E72C
:10CC400017B902A801F088F9FFF79AFB00F0A8FED7
:10CC5000FFF778FB94F84430FF2B08BF84F844605A
:10CC600094F84530FF2B08BF84F84560FFF788FB38
:10CC700001A902A801F07CF950BB2046FFF7B8FCDF
:10CC800000B323683BB9FFF75DFBA06801F090FAA1
:10CC90000546FFF775FB019904F1240001F0C8F87F
:10CCA0002046FFF7F9FC00F027FF48B94FF0E023DA
:10CCB0004FF08052C3F8042DBFF34F8FBFF36F8F37
:10CCC00001278FE72046FFF7E7FC00F015FFF7E7A5
:10CCD0002046FFF7E1FC00F00FFF2046FFF788FC3D
:10CCE0000028EDD0002D9CD0FFF72CFB616A19B114
:10CCF000236B1968C1F10501A06801F0F7FA9BE701
:10CD00008AE501082DE9FF410E460446019220B94B
:10CD10004FF4CD614348F9F72FFC36B9236C23B1AA
:10CD200040F26C613F48F9F727FC01F031FA30B965
:10CD3000019B23B140F271613A48F9F71DFC0027CD
:10CD4000B846FFF7FFFAA36BE3B131462046E5682A
:10CD5000FFF78EFC636AE56073B104F1240001F013
:10CD6000A1F848B14FF0E0234FF08052C3F8042DF2
:10CD7000BFF34F8FBFF36F8FFFF702FB012004B0AB
:10CD8000BDE8F081019D1DB9FFF7FAFA0020F6E732
:10CD900017B902A801F0E0F8FFF7F2FA00F000FE80
:10CDA000FFF7D0FA94F84430FF2B08BF84F8448092
:10CDB00094F84530FF2B08BF84F84580FFF7E0FA70
:10CDC00001A902A801F0D4F800BB2046FFF710FC2F
:10CDD000B0B1019904F1240001F02AF82046FFF7D0
:10CDE0005BFC00F089FE48B94FF0E0234FF0805221
:10CDF000C3F8042DBFF34F8FBFF36F8F0127A0E758
:10CE00002046FFF749FC00F077FEF7E72046FFF7E2
:10CE100043FC00F071FE2046FFF7EAFB0028EDD04E
:10CE2000B4E700BF8AE501082DE9F843894690463A
:10CE3000054620B940F2FB612048F9F79DFBB9F1A6
:10CE4000000F06D12B6C23B140F2FC611B48F9F7AF
:10CE500093FBFFF74DFBEFF311874FF0500383F384
:10CE60001188BFF36F8FBFF34F8FAC6B1CB395F876
:10CE700044604946284676B2FFF7FAFB013C731C32
:10CE8000AC6313D12B690BB901200BE005F1100045
:10CE900001F008F80028F7D0B8F1000FF4D0012015
:10CEA000C8F8000087F31188BDE8F883013676B230
:10CEB00085F84460E8E72046F4E700BF8AE501080A
:10CEC00010B5044620B940F28A710548F9F754FBC1
:10CED000FFF738FAA46BFFF753FA204610BD00BFE6
:10CEE0008AE5010810B5044620B940F2A47106484D
:10CEF000F9F742FBFFF726FAA06BE46B241AFFF761
:10CF00003FFA204610BD00BF8AE50108002310B596
:10CF1000064A52F833402CB942F8331002EBC303EF
:10CF2000586010BD0133052BF3D1FAE774160020C9
:10CF3000002310B5074A02EBC3014C68844204D1B8
:10CF4000002042F83300486010BD0133052BF2D1B8
:10CF5000FAE700BF7416002010B5044620B94FF45C
:10CF6000F8610548F9F708FB2046FFF7E1FF204686
:10CF7000BDE81040FFF724BB8AE5010870B5044600
:10CF80000D461646FFF7DEF994F84430FF2B04BF38
:10CF9000002384F8443094F84530FF2B04BF00236D
:10CFA00084F84530FFF7ECF9A36B2BB932462946DC
:10CFB00004F1240000F056FF2046BDE87040FFF762
:10CFC0006BBB8268436800681344181A824298BF9A
:10CFD000801A70472DE9F84304468846164622B960
:10CFE00040F244411848F9F7C7FA6568A3685F1B27
:10CFF000B74228BF3746EA19934204D240F24E4165
:10D000001148F9F7B9FAA0693A46414628440BF0AD
:10D0100079FBBE420FD9A368A6EB0709994504D94D
:10D0200040F256410848F9F7A7FA4A46A06908EBCA
:10D0300007010BF067FBA3683544AB4298BFED1ABC
:10D0400030466560BDE8F8838AE5010893422DE922
:10D05000F84328BF13460646894690461D4683B3CB
:10D0600007688468E41B9C4228BF1C46A24204D285
:10D070004FF490611448F9F77FFAB2683B19934274
:10D0800004D940F281411048F9F776FAB169224695
:10D09000484639440BF036FBA5420CD9A84504D2CA
:10D0A00040F289410848F9F767FAB1692A1B09EB90
:10D0B00004000BF027FBB3682F44BB4298BFFF1A54
:10D0C00037602846BDE8F8838AE50108012A2DE982
:10D0D000F04104460F46164630D1042803D8E82113
:10D0E0001A48F9F749FABC4203D2F0211748F9F778
:10D0F00043FA04F12500FFF761FA0546D8B100F1C3
:10D10000240801342246552140460BF023FB80457C
:10D1100004D04FF499610D48F9F72EFA242200212A
:10D1200028460BF017FB012F38BF0127C5F81880E0
:10D13000AC60EF602E772846BDE8F08118B9EE218B
:10D140000248F9F719FA0026CDE700BF8AE5010881
:10D150002DE9F843044620B940F291111748F9F738
:10D160000BFA276AFFF7EEF8206918BB63691BBB4F
:10D17000D4E90269A56932465521284694F81C80F5
:10D180000BF0E8FA854204D04FF499610B48F9F7A7
:10D19000F3F92046242200210BF0DCFAC4E90269ED
:10D1A000A56184F81C8027620124FFF7E9F8204676
:10D1B000BDE8F8830024F8E70446F6E78AE50108AD
:10D1C00010B5044620B940F2DB110648F9F7D4F94E
:10D1D000A3682068626818440138801A834298BFA7
:10D1E000C01A10BD8AE501082DE9F04786B0044653
:10D1F00016460F46019321B94FF401714148F9F7E2
:10D20000BBF924B940F205213E48F9F7B5F9237F6F
:10D21000DA0716D506F10408464504D34FF4047125
:10D220003848F9F7A9F9019B6BB92046FFF7C8FF09
:10D2300005460396002D38D10025284606B0BDE8E6
:10D24000F087B046EFE704A800F06CFE4FF000094D
:10D25000DFF8B0A0FFF776F82046FFF7B1FF804572
:10D2600005461FD9002001F0E1F9636923B140F2BE
:10D2700029215046F9F780F900F084FF6061FFF73B
:10D280007FF80022019B1146104601F08FF8C4F888
:10D29000149001A904A800F06BFE0028DAD0002D3C
:10D2A000C3D0C6E7FFF76CF8F9E7237FDB0720D48C
:10D2B000B54294BF0395039639462046039AFFF77B
:10D2C00089FE05460028B8D02046FFF77AFEE368BD
:10D2D0009842B2D300F064FB23693BB1002320697C
:10D2E0001A46194601F0ACF80023236100F004FC53
:10D2F000A3E74545A0D30422204603A9FFF76AFE11
:10D30000DAE700BF8AE501082DE9F743044616462F
:10D310009946884621B940F2D1213348F9F72CF9D2
:10D3200024B940F2D2213048F9F726F9237F13F0CF
:10D33000010F14BF04270027B9F1000F20D0FFF719
:10D3400001F82046FFF73DFE874205460CD300203A
:10D3500001F06CF9236923B140F2F5212248F9F775
:10D360000BF900F00FFF2061FFF70AF8AF4212D36C
:10D3700000224B461146104601F018F800232361A5
:10D380002046FFF71EFEB842054604D80025284671
:10D3900003B0BDE8F0837FB12B463A46204601A991
:10D3A000D4F80090FFF752FE019BED1B9E4236BF62
:10D3B00000261E46C4F800902B46324641462046C1
:10D3C000FFF744FE05460028E0D000F0E9FA636963
:10D3D0003BB1002360691A46194601F031F8002379
:10D3E000636100F089FBD2E78AE5010880B5174D3B
:10D3F000174F184E2B6873B9174B1B68012BF8D9C0
:10D400004FF0E0234FF08052C3F8042DBFF34F8F4D
:10D41000BFF36F8FEDE7FEF795FFFB68DC68201D1B
:10D4200001F02FFB3368013B33602B68013B2B601D
:10D43000FEF7A6FF04F154000CF06EF8206BFFF726
:10D44000BFF82046FFF7BCF8D4E700BF1017002054
:10D45000841700200C170020A8160020F8B51A4BDE
:10D460001A4D06461C6828680F46043001F009FB77
:10D4700040B92A681649D06A01220B68824023EA23
:10D4800002030B60731C07D137B1296811480431BE
:10D49000BDE8F84001F0D2BA2B68A4195C6007D34C
:10D4A0000D4B18682968BDE8F840043101F0D2BA84
:10D4B0000A4B18682968043101F0CCFA084B1A6845
:10D4C000A24288BF1C60F8BD981700209C1600205F
:10D4D0002017002070170020A4160020A01600209E
:10D4E00050170020064A13681968064B19B94FF007
:10D4F000FF321A6070471268D268D2685268F8E743
:10D50000A01600205017002010B5044620B940F2A4
:10D51000F2610848F9F730F86269074B9A4207D17F
:10D52000A06A064B984203D0B0FA80F0400910BDC3
:10D530000020FCE78AE5010870170020581700203A
:10D540002DE9F84F4FEA820A064650460D461F461F
:10D55000DDF82C90FFF732F88046002800F0B58007
:10D56000BC20FFF72BF80446002800F0AB80C0F881
:10D57000308025B94FF458715B48F8F7FDFF5246EB
:10D58000A521206B0BF0E6F8236BAAF1040A9A445C
:10D590002AF0070A6B1E04F134020F3513F8011F3D
:10D5A00002F8011B09B19D42F8D10A9D4FF0000B12
:10D5B000042D28BF042504F104084046C4E9135B88
:10D5C000E56284F843B001F036FAC5F1050504F1CF
:10D5D000180001F030FA60225946C4F8B4B0246152
:10D5E000A561646284F8B8B004F154000BF0B2F89D
:10D5F0003E4B3A46A3653E4B3146E3653D4B5046B4
:10D600002366FEF777FE2060B9F1000F01D0C9F85C
:10D610000040FEF797FE384B384E1A68384F0132FB
:10D620001A603568002D53D134601B68012B1FD15F
:10D63000B9464846013501F0F3F9052D09F1140901
:10D64000F7D1DFF8C090304D484601F0E9F928469F
:10D6500001F0E6F92D4801F0E3F92D4801F0E0F979
:10D660002C4801F0DDF92C4BC3F800902B4B1D60CA
:10D6700001252B4A2B491368086801331360E26ABD
:10D68000636405FA02F3034314200B6000FB02708D
:10D69000414601F0D3F9FEF773FE234B1B6873B1CB
:10D6A0003368DA6AE36A9A4209D24FF0E0234FF016
:10D6B0008052C3F8042DBFF34F8FBFF36F8F2846FE
:10D6C000BDE8F88F4046FEF77BFF4FF0FF35F6E7E9
:10D6D000154B1B68002BCBD13368DA6AE36A9A4298
:10D6E00098BF3460C4E700BF8AE50108D4EE0108A2
:10D6F000F4EE0108B4EE01080C1700209C1600207F
:10D70000A8160020241700203817002058170020E2
:10D710008417002070170020A0160020A4160020F7
:10D720001C170020201700206C170020F8B50446B5
:10D730002B4DFEF707FE04B92C68261D304601F07C
:10D74000A0F960B91420E76A264B78431B5833B917
:10D7500001222549BA400B6823EA02030B60A36A41
:10D760001BB104F1180001F08CF9204A1368013351
:10D7700013602B68A34222D131461D4801F05EF9A7
:10D780001C4A136801331360FEF7FAFD1A4B1B683D
:10D79000A3B12B68A34211D1184B1B6823B140F2EF
:10D7A000B6411748F8F7E8FE4FF0E0234FF08052FB
:10D7B000C3F8042DBFF34F8FBFF36F8FF8BD114A2D
:10D7C00004F154001368013B13600BF0A5FE206BBD
:10D7D000FEF7F6FE2046FEF7F3FEFFF783FED3E7E3
:10D7E0009C160020A8160020201700201C170020DF
:10D7F00084170020101700206C1700201817002035
:10D800008AE501080C170020F8B5044620B940F25B
:10D810004C511748F8F7B0FE164B1B68A34220D0B6
:10D82000FEF790FD144B65691F68144B1E68FEF7E8
:10D83000A7FDBD4217D0B54215D0114B9D4208D16E
:10D84000A36A83B994F8B830012B0CBF02200320DF
:10D85000F8BD0C4B9D4208D0002D0CBF04200120C8
:10D86000F6E70020F4E70220F2E70420F0E700BF2B
:10D870008AE501089C160020A0160020A4160020AE
:10D88000701700208417002070B5044620B940F2BC
:10D890001C711A48F8F770FE194D2B68A3422BD063
:10D8A00054B3FEF74FFD2046FFF72EFE00B3261DB2
:10D8B000304601F0E6F801231249E26A0868934015
:10D8C000034314200B60104B314600FB023001F083
:10D8D000B5F82B68E26ADB6A9A4209D34FF0E0237D
:10D8E0004FF08052C3F8042DBFF34F8FBFF36F8FFB
:10D8F000BDE87040FEF744BD70BD00BF8AE5010879
:10D900009C16002020170020A816002013B5002424
:10D910001A4B502201931A4923461A480094FFF7E4
:10D920000FFE01281DD100F0E1FE012819D14FF0B2
:10D93000500383F31188BFF36F8FBFF34F8F124BE8
:10D94000124A1B68543313604FF0FF32104B1A60B9
:10D95000104B1860104B1C6002B0BDE81040FEF781
:10D960006BBD013007D140F604010C4802B0BDE8A0
:10D970001040F8F701BE02B010BD00BF4C170020E8
:10D9800060CD0108EDD300089C1600203005002072
:10D99000501700206C170020981700208AE5010816
:10D9A000024A136801331360704700BF1817002044
:10D9B000014B1868704700BF9817002008B5FEF7A4
:10D9C00097FD014B186808BD98170020014B186897
:10D9D000704700BF0C1700202DE9F84F3A4B1B6829
:10D9E000002B6AD1394B1D6801351D609DB9384C3B
:10D9F00023681B6823B140F662213648F8F7BCFD66
:10DA0000354B2268196821601A60344A1368013363
:10DA10001360FFF767FD324E00243368314FAB428D
:10DA200010D91422304B1B68DB6A5343FB58022B7E
:10DA300028BF01242D4B1B68002B0CBF2046012062
:10DA4000BDE8F88FDFF888A0DFF8A490DAF800309E
:10DA50001B681BB94FF0FF333360E2E7DAF80030A0
:10DA6000DB68D3F80CB0DBF80420954201D23260B9
:10DA7000D7E70BF10408404601F003F8DBF8282053
:10DA80001AB10BF1180000F0FCFF0122DBF82C00AA
:10DA9000D9F8003082401A43C9F8002014224146C8
:10DAA00002FB007000F0CAFF0F4BDBF82C20196856
:10DAB000CB6A9A4228BF0124C8E70E4A00241368A3
:10DAC00001331360B6E700BF181700209817002035
:10DAD000A01600208AE50108A41600205417002093
:10DAE00050170020A81600209C1600209C1700202C
:10DAF00020170020141700202DE9F8432F4C23682D
:10DB000023B940F668012E48F8F736FDFEF71AFCF7
:10DB10002368013B236024682CB10024FEF730FC0D
:10DB20002046BDE8F883274B1B68002BF5D0264D17
:10DB3000264EDFF89C801FE0EB680127DC6804F1CB
:10DB4000040904F1180000F09CFF484600F099FF1A
:10DB50001420E26A316807FA02F30B4300FB0280EB
:10DB60004946336000F06AFF1A4BE26A1B68DB6AC1
:10DB70009A4201D3184B1F602B68002BDCD10CB1EB
:10DB8000FFF7B0FC154D2C6844B10127124EFFF78A
:10DB900023FF00B13760013CF9D12C600E4B1B68AC
:10DBA000002BBAD04FF0E0234FF08052C3F8042D81
:10DBB000BFF34F8FBFF36F8F0124AFE7181700201B
:10DBC0008AE501080C1700205817002020170020B4
:10DBD000A81600209C1600209C1700201417002077
:10DBE00038B50C46054620B940F2CA411948F8F745
:10DBF000C3FC24B940F2CB411648F8F7BDFC164BE4
:10DC00001B6823B140F2CC411248F8F7B5FCFFF78E
:10DC1000C7FE124B2A68186814192CBF0121002175
:10DC200082422C600ED971B9FFF766FF48B94FF0F8
:10DC3000E0234FF08052C3F8042DBFF34F8FBFF3A2
:10DC40006F8F38BD09B9A042EED20021201AFFF72C
:10DC500005FCE9E78AE5010818170020981700205D
:10DC600010B5044650B94FF0E0234FF08052C3F88E
:10DC7000042DBFF34F8FBFF36F8F10BD094B1B688F
:10DC800023B14FF4A4610848F8F776FC0021204640
:10DC9000FFF786FEFFF7E2FBFFF72EFF0028E2D03A
:10DCA000EBE700BF181700208AE50108244B70B588
:10DCB0001A68244B12B101221A6070BD224E1A60FC
:10DCC00033681B6B1A68B2F1A53F0BD15A68B2F1E9
:10DCD000A53F07D19A68B2F1A53F03D1DB68B3F144
:10DCE000A53F04D0306831683431F8F711FC174B88
:10DCF0001C68B4FA84F41423E4B2C4F11F0463432F
:10DD0000134DEB5823B940F688311248F8F734FC2C
:10DD1000142000FB04F3EA185168083349682B44C7
:10DD2000994200FB045408BF4B68516008BF536020
:10DD30006368094ADB683360336854331360BCE7B7
:10DD4000181700209C1700209C1600202017002088
:10DD5000A81600208AE5010830050020F8B5044621
:10DD60002B4DFEF7EFFA04B92C68261D304600F063
:10DD700088FE60B91420E76A264B78431B5833B9F4
:10DD800001222549BA400B6823EA02030B60A36A0B
:10DD90001BB104F1180000F074FE31461F4800F07A
:10DDA0004DFE94F8B8301E4E012B04BF002384F8BA
:10DDB000B830FEF7E5FA33682BB1FEF7C3FAFFF788
:10DDC00091FBFEF7DDFA2B68A34213D1336893B1C0
:10DDD000144B1B6823B14FF4D9611348F8F7CCFBFF
:10DDE0004FF0E0234FF08052C3F8042DBFF34F8F64
:10DDF000BFF36F8FF8BD094A11680C4A126891424F
:10DE000001D12B60F6E7BDE8F840FFF74FBF00BF38
:10DE10009C160020A8160020201700207017002054
:10DE20006C170020181700208AE501080C17002045
:10DE300038B50D46044620B940F69F310748F8F73B
:10DE40009BFB074B20461968183100F003FE28465B
:10DE5000BDE838400121FFF701BB00BF8AE501089A
:10DE60009C16002070B50E461446054620B940F6B3
:10DE7000CA310A48F8F780FB094B2846196818315F
:10DE800000F0DCFD002C214608BF3046BDE87040A4
:10DE900018BF4FF0FF30FFF7E1BA00BF8AE5010875
:10DEA0009C16002038B5C368DC6824B940F6FA3106
:10DEB0001548F8F761FB04F11805284600F0E1FD6C
:10DEC000124B1B68E3B9251D284600F0DAFD01233B
:10DED0000F49E26A08689340034314200B60294607
:10DEE0000C4B00FB023000F0A9FD0B4BE26A1B68F3
:10DEF000DB6A9A4285BF0120084B0020186038BDBC
:10DF000029460748EFE700BF8AE5010818170020F7
:10DF100020170020A81600209C1600209C17002027
:10DF20005817002010B5044620B940F64F41074865
:10DF3000F8F722FBFEF706FA054B1B682360054B3A
:10DF40001B686360BDE81040FEF71ABA8AE5010855
:10DF50005417002098170020034B1B680360034BE5
:10DF60001B684360704700BF5417002098170020BB
:10DF700070B50C46054620B940F665411448F8F7DF
:10DF8000FBFA24B940F666411148F8F7F5FAFEF7B6
:10DF9000D9F9104B196823685A1C10D00E482E6806
:10DFA00000686A68864201D08A420FD9881A834283
:10DFB0000AD95B1A134428462360FFF7CDFF0024DB
:10DFC000FEF7DEF9204670BD002323600124F7E749
:10DFD0008AE5010898170020541700200122014B00
:10DFE0001A6070479C17002070B50C46164605460F
:10DFF00008B91B4A156805F134026260EA6A052B0C
:10E0000022612A6B2560E2616A6CA260EA6C62613F
:10E010004FF00002A26119D011490968A94209D143
:10E020002273D6B10023296BCA5CA52A13D09B08A2
:10E03000238470BD032B2373F3D1FFF7B1FCAB6ACC
:10E040000BB102232373FFF757FDEAE72846FFF7DA
:10E05000DBFB2073E5E70133E6E72684E9E700BF51
:10E060009C1600202DE9F84F0D6806460C46174611
:10E070002DB300254FF0240B4B6801F108085B68B5
:10E0800043454B6004BFCB684B604B68D3F80CA092
:10E0900063680BFB05615B6801229845636008BFFC
:10E0A000D8F8043005F1010508BF63606368D3F850
:10E0B0000C903B464846FFF797FFCA45E8D12846F3
:10E0C000BDE8F88F2DE9F0471746FFF769FC1F4BB5
:10E0D00005461B688B4237D8052600244FF0140AEA
:10E0E0004FF02408DFF86890013E08FB045001223D
:10E0F0000AFB0691FFF7B6FF0444002EF4D1154B3E
:10E100000222196808FB0450FFF7ACFF124B0444CD
:10E110001968022208FB0450FFF7A4FF04440422FC
:10E1200008FB04500D49FFF79DFF044408FB045011
:10E1300003220B49FFF796FF044407B13E60FFF747
:10E14000DBFC2046BDE8F0870024F8E70C17002030
:10E15000A8160020A0160020A41600208417002076
:10E160007017002008B9064B1868026B0020135C7A
:10E17000A52B02D0C0F38F0070470130F7E700BF36
:10E180009C160020014B1868704700BF9C160020A9
:10E19000054B1B6833B1054B1B68002B0CBF0220DD
:10E1A00000207047012070476C17002018170020CE
:10E1B0002DE9F0410446002835D0234DC36A2A6872
:10E1C000D26A934237D214268269204F002AA8BF10
:10E1D0002A6806FB0373A2BFD26AC2F105028261FC
:10E1E00042699A4221D100F10408404600F049FCFE
:10E1F000174B48B9E06A4643BA592AB901211A684F
:10E20000814022EA01021A602A681968D26AE26231
:10E21000012404FA02F0084318601420414600FB70
:10E22000027000F00BFC204603E02B68DB6AC3623F
:10E230000120BDE8F0812B68C06CDC6AA0422CBFD5
:10E2400000200120F5E700BF9C160020A816002042
:10E2500020170020F8B5044608B90020F8BD1F4B70
:10E260001B68834204D040F67A711D48F8F784F9A0
:10E27000236D23B940F67B711948F8F77DF9236DBA
:10E28000E16AE26C013B91422365E6D0002BE4D1C8
:10E29000261D304600F0F5FB124F134A50B91421E9
:10E2A000E06A41437B582BB901251368854023EA76
:10E2B00005031360E36C1420C3F10501A161E3625F
:10E2C0000124116804FA03F500FB03700D43314685
:10E2D000156000F0B3FB2046C0E700BF9C1600208D
:10E2E0008AE50108A816002020170020F8B50D4681
:10E2F0000446002845D0036D23B940F6C971214872
:10E30000F8F73AF9E16CE36A8D4238BF0D46AB424B
:10E3100037D0236D012B34D11B4B1B68A34204D192
:10E3200040F6E4711748F8F727F9A269E36A002A72
:10E33000E562A4BFC5F10505A5611425134E626908
:10E3400005FB03639A421CD1271D384600F099FB58
:10E35000E26A0F4C40B9554373592BB90121236828
:10E36000914023EA01032360012314202168934094
:10E370000B4300FB026039462360BDE8F84000F023
:10E380005DBBF8BD8AE501089C160020A816002098
:10E3900020170020044B1A681AB119680A6D01325F
:10E3A0000A651868704700BF9C1600202DE9F041EF
:10E3B000224C1E4680460F461546FDF7C3FF2368D4
:10E3C00093F8B830022B18D001212268D2F8B4306B
:10E3D00023EA0803C2F8B430236883F8B81066B1A2
:10E3E0003046FFF73BF84FF0E0234FF08052C3F880
:10E3F000042DBFF34F8FBFF36F8FFDF7C1FFFDF704
:10E40000A1FF1DB12368D3F8B4302B60236893F8C3
:10E41000B830022B03BF22680125D2F8B4300025A2
:10E4200004BFBB43C2F8B4300022236883F8B8208D
:10E43000FDF7A6FF2846BDE8F08100BF9C1600202E
:10E44000F8B50E4617461D46044620B941F219217B
:10E450002F48F8F791F8FDF775FF15B1D4F8B430EF
:10E460002B60022394F8B85084F8B830EDB2042F32
:10E470001AD8DFE807F00E0309061500D4F8B41027
:10E480000E43C4F8B46004E0D4F8B4300133C4F8E7
:10E49000B430012D12D00124FDF772FF2046F8BDE3
:10E4A000022DEED10024F7E7D4F8B4300133F0D0D8
:10E4B00041F24A211648F8F75FF8EAE7261D304690
:10E4C00000F0DFFA1420134AE36A11689D400D43FF
:10E4D0001560114A314600FB032000F0AFFAA36A31
:10E4E00023B141F259210A48F8F746F80B4BE26A8A
:10E4F0001B68DB6A9A42CED94FF0E0234FF080527E
:10E50000C3F8042DBFF34F8FBFF36F8FC3E700BF76
:10E510008AE5010820170020A81600209C1600207C
:10E520002DE9F843089F0D4691461E46044620B942
:10E5300041F28C213648F8F71FF8FDF7D9FFEFF3C9
:10E5400011884FF0500383F31188BFF36F8FBFF32F
:10E550004F8F16B1D4F8B4303360022394F8B8600A
:10E5600084F8B830F6B2B9F1040F1AD8DFE809F030
:10E570000E0309061500D4F8B4100D43C4F8B450C6
:10E5800004E0D4F8B4300133C4F8B430012E12D012
:10E59000012088F31188BDE8F883022EEED1002017
:10E5A000F7E7D4F8B4300133F0D041F2CF21184866
:10E5B000F7F7E2FFEAE7A36A23B141F2DA21144850
:10E5C000F7F7DAFF134B1B68EBB9251D284600F05F
:10E5D00058FA01231049E26A086893400343142063
:10E5E0000B6029460D4B00FB023000F027FA0C4B64
:10E5F000E26A1B68DB6A9A42CAD9012307B13B6011
:10E60000084A1360C4E7084804F11801EDE700BFA9
:10E610008AE501081817002020170020A8160020FE
:10E620009C1600209C1700205817002010B50446A7
:10E6300008B9084B1C68FDF785FE002094F8B83037
:10E64000022B0ABF84F8B80004460124FDF798FEA7
:10E65000204610BD9C160020F8B50F4CFDF772FE49
:10E660002568ADB90D4F0E4E384600F0D9F9304649
:10E6700000F0D6F90B4B2A461F600B4B0C210A20E9
:10E680001E60FEF77FF8206010B10849FEF73EFCDF
:10E69000BDE8F840FDF774BED4170020A81700208D
:10E6A000BC170020A0170020A417002065CD01088A
:10E6B000914208B5416000610AD8D21A83699A4232
:10E6C0000DD2084B011D186800F0C4F9002008BDE8
:10E6D0009A4201D2994202D2034B011DF3E7012075
:10E6E000F5E700BFA4170020A017002007B5FFF72B
:10E6F000B3FF0C4B1B6843B90B484FF48971F7F714
:10E700003BFF002003B05DF804FB084BC8220193D7
:10E7100001230749009307480023FEF711FF002853
:10E72000EAD0EFE7D41700208AE50108D8170020C7
:10E730006ACD010881E800082DE9F04180462C20CF
:10E740000D4617461E46FDF739FF044688B125B928
:10E750004FF4B6710848F7F70FFFFFF77DFF069BF0
:10E76000C4E90657C4F8008026626362201D00F0E9
:10E7700062F92046BDE8F0818AE501082DE9FF41F4
:10E780000C4690461E46054620B94FF4C3710F480B
:10E79000F7F7F2FE0E4F386878B1052CCDE9014845
:10E7A00003950DDCFFF7F4FC0023022814BF1A4682
:10E7B0000A9A386801A9FEF709F804B0BDE8F081AB
:10E7C0000023324601A9FEF7B9F8F6E78AE5010809
:10E7D000D41700202DE9F04F85B00646FFF7E8F882
:10E7E000DFF88C800546D8F8003083423DD94FF0E1
:10E7F0000009204FDFF880A03B681A685AB91F4A09
:10E80000116813600123396028463360C8F800504E
:10E8100005B0BDE8F08FDB68DC68D3F800B0211DDF
:10E820000846039100F02DF9636A20469847E36992
:10E830000399012BE0D1A3695B449B4505D238685D
:10E840006360246100F006F9D6E700235A461946B2
:10E850002046CDF80090FFF791FF0028CCD140F280
:10E8600072315046F7F788FEC6E70023CCE700BFB9
:10E87000D0170020A01700208AE50108A417002067
:10E880002DE9F047624F634E86B03B681D68002D4E
:10E8900068D00024DB681D68FFF782F803A8FFF743
:10E8A00099FF039B8246DFF87081002B78D1002C02
:10E8B0005AD1A8425ED3FFF71FF93B68DB68D3F853
:10E8C0000C9009F1040000F0DCF8D9F81C30012BA1
:10E8D00015D1D9F818102B46524648462944FFF75F
:10E8E000E7FE60B123462A46214648460094FFF7DA
:10E8F00045FF20B94FF4F4713046F7F73DFE484626
:10E90000D9F8243098470022D8F8000003A9FEF770
:10E91000B9F80028B9D0039B002BF4DB059C636990
:10E9200013B1201D00F0ADF802A8FFF753FF039BC1
:10E930000546092BE7D801A252F823F0A7E9000801
:10E94000A7E90008A7E9000807E90008E7E90008C7
:10E9500007EA0008A7E90008A7E9000807E9000896
:10E96000E7E90008012497E72C4B1B681C68B4FA00
:10E9700084F464092246D8F80000A5EB0A01FEF7EA
:10E98000FDFAFFF7B9F80028BDD14FF0E0234FF0B2
:10E990008052C3F8042DBFF34F8FBFF36F8FB2E7E0
:10E9A000FFF7AAF8AFE7A169049B02461944204685
:10E9B000FFF77EFE0028A6D0636A20469847E369E9
:10E9C000012BA0D10023A269049920460A44009398
:10E9D0001946FFF7D3FE002895D140F201313046A9
:10E9E000F7F7CAFD8FE7049BA36123B94FF4467183
:10E9F0003046F7F7C1FDA1692B462A462046294437
:10EA0000FFF756FE7FE72046FDF7DAFD7BE700BF04
:10EA1000A01700208AE50108D4170020A4170020C1
:10EA20004FF0FF3200F10803C0E9022343600361A5
:10EA300000230360704700230361704743689A68AE
:10EA40004B608A609A68516099600368086101337D
:10EA50000360704730B50C68631C0AD103695A68BB
:10EA60004A6091608B6059600368086101330360FC
:10EA700030BD00F10802134652681568A542FAD964
:10EA8000EDE70369D0E901128A605160596881425B
:10EA900008BF5A60002202611A68013A1A601868B9
:10EAA00070470000021E18BF012200210148F8F73C
:10EAB00055BB00BF00040240F8F7ACBF38B50546AF
:10EAC0000C460020FFF7EEFF45F08000FFF7F4FF53
:10EAD0002046FFF7F1FFBDE838400120FFF7E2BF15
:10EAE00008B50120F8F72AF90A20F8F727F90B20D2
:10EAF000F8F724F90720F8F721F90520F8F71EF9AF
:10EB0000BDE808400420F8F719B9000070B5204BA3
:10EB100004469D78EDB958B902211E48F8F719FB53
:10EB200023461A460221BDE870401A48F8F746BA53
:10EB3000012805D102211748F8F706FB2B46F0E71C
:10EB4000022823D102460146BDE870401148F8F77B
:10EB500075BA012D14D138B904210E48F8F7F9FA25
:10EB6000002304211A46DEE7012804D104210948C4
:10EB7000F8F7EAFAF4E7022808D102460421E3E7AD
:10EB80006A21BDE870400448F7F7F6BC70BD00BFCD
:10EB9000DC170020000002408AE5010808B50020CB
:10EBA000FFF7B4FFF8F70CF80120FFF7AFFFF8F715
:10EBB00007F80220FFF7AAFFBDE80840F8F700B801
:10EBC00008B500210120F8F7A5FE0120FFF76AFF34
:10EBD0000023094819461A46F8F7F0F9B5214020F4
:10EBE000FFF76CFFA0214120FFF768FFBDE8084058
:10EBF00000210120FFF762BF0004024010B5FFF7BB
:10EC00006FFF0120FFF74EFF00233A4819461A46CE
:10EC1000394CF8F7D3F900210120F8F77BFE23786F
:10EC20007BB1002306211A463248F8F7C7F90621BE
:10EC30003048F8F789FAF7F7C3FF19215820FFF792
:10EC40003DFFFFF7ABFFFFF7BBFF63785BB100232E
:10EC500004211A462948F8F7B1F900230D211A4674
:10EC60002748F8F7ABF9002201212248F8F7E6F926
:10EC700000220A211F48F8F7E1F900220B211D4864
:10EC8000F8F7DCF9002207211A48F8F7D7F9002233
:10EC900005211848F8F7D2F9002204211548F8F7A1
:10ECA000CDF90523022201211248F8F765F8052362
:10ECB00002220A210F48F8F75FF8052302220B21F0
:10ECC0000C48F8F759F80523022207210948F8F7FC
:10ECD00053F80523022219460648F8F74DF8094B68
:10ECE0001B782BB9BDE81040BE210748F7F744BC9C
:10ECF00010BD00BF00040240DC17002000000240ED
:10ED000000080240DF1700208AE5010882B0019068
:10ED1000064B9DF80620BDF804109A700122198058
:10ED2000034B1A7002B0FFF769BF00BFDC17002069
:10ED3000DF1700201A4B10B55B78D3B10128194CAE
:10ED400018D104211848F8F7FFF90D211748F8F7F2
:10ED500000FA23786BB1002304211A461248F8F711
:10ED60002DF900230D211A461048F8F727F9002342
:10ED7000237010BD40B904210B48F8F7EAF90D21C2
:10ED80000A48F8F7E1F9E4E7022204210648F8F717
:10ED900055F902220D210548F8F750F90123E7E75C
:10EDA000DC170020C80200200000024000080240DA
:10EDB00008B5FFF795FEFFF7F1FEFFF701FFF8F743
:10EDC00005FE012200211F48F8F738F90220FFF75D
:10EDD000B1FF0220FFF79AFE022201211948F8F73D
:10EDE0002DF902220A211748F8F728F902220B21EF
:10EDF0001448F8F723F9022207211248F8F71EF900
:10EE0000022205210F48F8F719F9022204210D48C2
:10EE1000F8F714F90C4B1B781BB9E2210B48F7F7F4
:10EE2000ABFB0B4B1B785BB1002306211A46054850
:10EE3000F8F7C4F8BDE8084006210248F8F789B998
:10EE400008BD00BF00040240DF1700208AE501086A
:10EE5000DC17002010B5064C022220460021F8F7EE
:10EE6000EDF82046BDE8104002220121F8F7E6B88F
:10EE700000140240F8B5104CD4F88032984723466D
:10EE8000002210F5617541F10006D3E90874B8421B
:10EE900071EB0404B8BFC3E90801D3E90674BD42AD
:10EEA00076EB040402F10102B8BFC3E90656102A4A
:10EEB00003F12803E9D1F8BDE817002010B5044696
:10EEC00018B9BB210748F7F757FB074BD3F8803237
:10EED0009847D4E90632984271EB0202ACBF002099
:10EEE000181A10BD8AE50108E81700202DE9F84F2F
:10EEF000054628B9BDE8F84FDC213148F7F73CBB9F
:10EF00000026304C33462246117A0133A94208BF0D
:10EF10000136102B02F12802F6D1002E4ED0062D1C
:10EF200003D940212648F7F727FB274B53F83570C4
:10EF3000002F41D1E7212248F7F71EFB7E4310271F
:10EF4000DFF87C80237AAB4231D163687BB32369DD
:10EF5000012B03D1D0214046F7F70EFBD4E906017F
:10EF600050EA010322D0D4E908A9B0EB0A0061EB12
:10EF7000090108F087FD83462069013808F068FD23
:10EF80000146584608F070FE8346304608F060FDA2
:10EF9000594608F0B5FD594608F0A8FC08F09CFF5A
:10EFA00010EB0A0049F10003C4E906032661013FA2
:10EFB00004F12804C6D101E0012FBFD1BDE8F88FCC
:10EFC0008AE50108E817002084CF01084FF47A731E
:10EFD000B0FBF3F341F65832A3F55223A3F61833EE
:10EFE00093422DD81B4B1C4A0344934228D91B4BF8
:10EFF0001B4A0344934223D94CF24E32194B03442B
:10F0000093421DD9184B98421CD903F5371303F5C9
:10F01000D863984218D903F5122303F5F863984290
:10F0200014D903F5122303F5F863984210D903F5B8
:10F03000DB2303F5BA6398428CBF06200520704796
:10F04000002070470120704702207047032070475E
:10F05000042070473F373ACC9E8601007F0F31CCA9
:10F060003E0D0300AF312ACC40DA8E332DE9F04358
:10F0700085B0E0B1D0E903984FF47A710D4B446844
:10F08000D3F88C62037AB4FBF1F4062B96BF0A4ADC
:10F090000A4D52F823500778FFF710FF3B46CDE9A1
:10F0A00001902A4621460648CDF80080B04705B0B9
:10F0B000BDE8F083E8170020BCCF010872CD01083D
:10F0C0007FCD010870B5154C054694F894320E4674
:10F0D00023B94FF496711248F7F74EFA25B940F26A
:10F0E0002D110F48F7F748FA26B94FF497710C48DD
:10F0F000F7F742FA0023094A1178A94202D1516870
:10F10000B14206D00133102B02F12802F4D10020C5
:10F1100070BD282000FB0340FAE700BFE81700207D
:10F120008AE501082DE9F04FDFF8B8B099469BF861
:10F13000943293B09246019123B940F241112A488A
:10F14000F7F71AFA0026FFF795FEB0464FF0FF37A3
:10F150003446244DEB68019A934218DBBAF1000F54
:10F1600010D12846FFF7AAFE80B3B84236D30ED19D
:10F17000D4E90823D5E90801FAF7DDFE002818BF15
:10F180002C4604E000212846D0470028E9D101366A
:10F19000102E05F12805DDD1B9F1000F01D0C9F815
:10F1A00000707FB9B8F1010F0CD9384608F1FF3172
:10F1B000FBF7BAF812AB03EB8000282350F8404C61
:10F1C00003FB04B4204613B0BDE8F08F12AB03EB91
:10F1D000880343F8406C08F10108C6E707462C464F
:10F1E000D5E700BFE81700208AE50108000000000D
:10F1F0002DE9F0470F46044620B94FF4C27120486C
:10F20000F7F7BAF9236923B940F285111C48F7F7DB
:10F21000B3F9DFF87080D8F880329847C4E9080164
:10F2200005462069894608F013FC394608F068FC59
:10F23000394608F05BFB07F0F3FF0FA3D3E9002387
:10F2400008F070F907F044FD08F0DCFA451949F1BF
:10F250000001C4E906510646384608F017FED8F802
:10F260008C5202463346AC4661680748BDE8F04719
:10F27000604700BFAFF300800000000080842E4193
:10F280008AE50108E8170020C6CD01082DE9F04104
:10F290000E461746054620B94FF4C8711348F7F7D4
:10F2A0006BF926B940F291111048F7F765F9002182
:10F2B000384608F0E1FD20B94FF4C9710B48F7F763
:10F2C0005BF94FF010080A4C2378AB4206D1636813
:10F2D000B34203D139462046FFF78AFFB8F101084F
:10F2E00004F12804F0D1BDE8F08100BF8AE50108EF
:10F2F000E817002008B5FFF769FE003818BF0120A5
:10F3000008BD00002DE9F0413E4D074695F89432C6
:10F310000E4694B023B94FF4D9713B48F7F72CF956
:10F320003046FFF7E7FF044658B94FF47A71D5F835
:10F330009032B6FBF1F135489847204614B0BDE84D
:10F34000F08131463846FFF7BDFE04460028F4D16F
:10F3500080462C4B5A683AB108F10108B8F1100FF9
:10F3600003F12803F6D1E8E795F894321BB9772129
:10F370002548F7F701F91FB978212348F7F7FCF87A
:10F38000282200210DEB020009F0E4F93046FFF7D6
:10F390001DFE062804468DF8300003D940211A4886
:10F3A000F7F7EAF80B966E4619488DF8287050F872
:10F3B000343000EBC40042680AACCDE90D230FCC19
:10F3C0000FC60FCC0FC694E80300282404FB085492
:10F3D000EC46274686E80300BCE80F000FC7BCE8F0
:10F3E0000F000FC796E80300D5F88C3287E80300BA
:10F3F0004146084898472046FFF738FE207AFFF735
:10F4000075FD9AE7E81700208AE5010806CE010895
:10F4100084CF010835CE01080D4B10B593F8943216
:10F42000044623B94FF4EA710A48F7F7A5F86CB11E
:10F4300063685BB10848FAF72BFE2046FFF716FE1B
:10F440000023207A63602372FFF750FD002010BD77
:10F45000E81700208AE5010856CE0108144B2DE973
:10F46000F04193F8943205460F4623B94FF4F671F4
:10F470001048F7F781F825B940F2ED110D48F7F77C
:10F480007BF800260A4C04F520782378AB4208D19B
:10F490006368BB4205D12046FFF7BEFF002818BFB6
:10F4A000064628344445F0D13046BDE8F08100BF1F
:10F4B000E81700208AE501082DE9F041114F0546C3
:10F4C00097F8943223B94FF4FE710F48F7F754F8C8
:10F4D00025B940F2FD110C48F7F74EF81026094CFB
:10F4E0002378AB4204D1636813B12046FFF794FF41
:10F4F000013E04F12804F3D1D7F88C320348BDE86B
:10F50000F0411847E81700208AE5010866CE010897
:10F510002DE9F04105460E461746134C04F52078B8
:10F520002378AB4207D162682AB100239F420BDCEB
:10F530002046FFF771FF28344445F1D10024A7424B
:10F5400008DC0120BDE8F08156F823108A42F2D091
:10F550000133EBE7284656F82410FFF7D3FE0028C6
:10F56000F0D00134EBE700BFE8170020014B93F81F
:10F5700094027047E817002010B5074C2378FA2B47
:10F5800004D94FF40D710548F6F7F6FF20780130E5
:10F59000C0B2207010BD00BFE01700208AE501084E
:10F5A00084B070B504AC84E80F001C4C94F894123D
:10F5B00031B1D4F890321A48BDE8704004B0184711
:10F5C0004FF42672204604F5207504AE09F0C2F807
:10F5D0000FCE0FC533682B6013B9124BC4F89032AD
:10F5E000D4F88C3213B90F4BC4F88C32D4F888326B
:10F5F00013B1D4F884324BB9D4F88C320A48984706
:10F600000A4BC4F888320A4BC4F88432012384F8C8
:10F610009432BDE8704004B0704700BFE817002086
:10F6200082CE010889A00008BBCE0108B986010876
:10F63000A986010830B400250E4BD3E9082452EA0C
:10F64000040C04D0121844EB0104C3E90824D3E9E4
:10F65000062452EA040C04D0121844EB0104C3E956
:10F6600006240135102D03F12803E6D130BCFFF745
:10F6700001BC00BFE817002070B50446044E4518D1
:10F6800014F8011B3046FAF703FDAC42F8D170BD07
:10F6900004DB01082DE9F8430025DDE90878C0E91D
:10F6A0000112164639464246C0E90335C0E9055500
:10F6B000C0E9075505704562044600F11C0904F0D5
:10F6C00063FB38B931460848FAF7E2FC2B210748BA
:10F6D000F6F752FF43463A464946204604F042FBBD
:10F6E0002046BDE8F88300BF20B201088AE5010882
:10F6F00010B504461C30F0F7C0FE04F11000F0F71E
:10F70000BCFE204610BD000070B5044690B0014616
:10F71000924A01A805F0B3FA2146914A04A805F0DF
:10F72000AEFA21468F4A07A805F0A9FA8E4A21466B
:10F730000AA805F0A4FA8D49204605F097FA054677
:10F740008B48FAF7A5FCDDE901239B1A082B06D0AC
:10F750008848FAF79DFCB1218748F6F70DFFDDE9EF
:10F7600004239B1A082B06D08448FAF791FCB52194
:10F770008148F6F701FFDDE90A239B1A102B06D01A
:10F780007F48FAF785FCB9217B48F6F7F5FEDDE9FD
:10F7900007135B1A102B0CD101234A1E01F10F0035
:10F7A00012F8016F002E18BF00239042F8D1002BF1
:10F7B00053D07448FAF76CFC5DB37348FAF768FCF1
:10F7C000674A21460DA805F05AFA7048FAF760FC1E
:10F7D00008210198FFF750FF6D48FAF759FC0821FE
:10F7E0000D98FFF749FF6B48FAF752FC10210A9871
:10F7F000FFF742FF6848FAF74BFC0D980A9A019907
:10F8000000F0E8FF0DA8F0F738FE6448FAF740FC76
:10F8100061E06348FAF73CFC6248FAF739FC0A9960
:10F82000019800F035FF6048FAF732FC0421019896
:10F830000844FFF721FF5D48FAF72AFC10215C48D5
:10F84000FFF71AFF5B48FAF723FC10215A48FFF72D
:10F8500013FF5148FAF71CFCD7E710220A9808F06A
:10F8600041FF564A4449002808BF11465448FAF758
:10F870000FFC002D40D04448FAF70AFC384A2146D4
:10F880000DA805F0FCF94F48FAF702FC0821019891
:10F89000FFF7F2FE4C48FAF7FBFB08210D98FFF743
:10F8A000EBFE4A48FAF7F4FB10210798FFF7E4FE55
:10F8B0004748FAF7EDFB10210A98FFF7DDFE3648BE
:10F8C000FAF7E6FB0D98079B0A9A019900F096FF5C
:10F8D0000DA8F0F7D2FD3048FAF7DAFB0AA8F0F7E6
:10F8E000CCFD07A8F0F7C9FD04A8F0F7C6FD01A8F4
:10F8F000F0F7C3FD10B070BD2948FAF7C9FB3548D1
:10F90000FAF7C6FB079A0A99019800F005FF264806
:10F91000FAF7BEFB042101980844FFF7ADFE2E481C
:10F92000FAF7B6FB10212248FFF7A6FE2B48FAF79C
:10F93000AFFB10212A48FFF79FFE2A48FAF7A8FBE1
:10F9400010212948FFF798FE2848FAF7A1FB1A482A
:10F950001021FFF791FE104858E700BFEFCF0108D4
:10F96000F6CF0108FECF010805D001086DC30108DC
:10F970000CD0010823D001088AE5010833D0010822
:10F9800044D0010854D001086FD0010875D0010897
:10F9900086D0010898D0010889E5010840D1010806
:10F9A000B8D00108BDD00108EFD0010801D101088D
:10F9B0006C0400202DD101089C040020D8CF010840
:10F9C0005FD101087CD101088ED10108A1D10108C5
:10F9D000C1D101080CD2010846D20108B2D20108F7
:10F9E0007C040020C9D201088C040020E0D2010868
:10F9F0002DE9F04100259DF81870C0E90112C0E919
:10FA000003353946C0E90555C0E90755057045621B
:10FA10000446164600F11C0804F086F838B9314651
:10FA20000748FAF735FB20210648F6F7A5FD3A46C8
:10FA30004146204604F066F82046BDE8F08100BF4C
:10FA400020B201088AE501082DE9F0410025069F52
:10FA5000C0E90112C0E903353946C0E90555C0E9DE
:10FA60000755057045620446164600F11C0804F06F
:10FA7000EFF838B931460748FAF70AFB2021064863
:10FA8000F6F77AFD3A464146204604F0CBF8204688
:10FA9000BDE8F08120B201088AE50108F0B5012631
:10FAA000044608270D468DB0564B574A31460096FE
:10FAB00002A8FFF79DFF02A9204605F0C3FA02A89D
:10FAC000FFF716FE514BCDE900571A460DEB070024
:10FAD0000421FFF7DFFD0DEB0701204605F0B2FA28
:10FAE0000DEB0700FFF704FEEB19494A019700935D
:10FAF0000DEB0700474B0421FFF7CCFD0DEB070191
:10FB0000204605F09FFA0DEB07001027FFF7F0FDE8
:10FB1000EB190093404B04211A46019702A8FFF706
:10FB2000B9FD02A9204605F08DFA203502A8FFF79D
:10FB3000DFFD3A4B3A4A00950421019702A8FFF7EE
:10FB4000A9FD02A9204605F07DFA02A8FFF7D0FD25
:10FB50000C230025334A00930221334B02A8FFF700
:10FB600073FF02A9204605F06DFA02A8FFF7C0FD59
:10FB70002E4B2F4A3146009602A8FFF739FF02A903
:10FB8000204605F05FFA02A8FFF7B2FD294B2A4A8A
:10FB90000221009502A8FFF757FF02A9204605F0B1
:10FBA00051FA02A8FFF7A4FD244B254A0221009533
:10FBB00002A8FFF749FF02A9204605F043FA02A870
:10FBC000FFF796FD1F4B204A3146009602A8FFF72B
:10FBD0000FFF02A9204605F035FA02A8FFF788FDBD
:10FBE00007231A4A00930221194B02A8FFF72CFFA2
:10FBF000204602A905F026FA02A8FFF779FD0DB00C
:10FC0000F0BD00BFF7D201086DC30108EFCF0108B6
:10FC1000F6CF010885D3010805D001089ED301085D
:10FC2000FECF010849C3010811D301086AD30108B6
:10FC30004CC30108C8D3010850C3010806D4010809
:10FC400059C3010841D4010862E4010862C30108F4
:10FC50005DD4010810B5084CD4F834321BB95C21CE
:10FC60000648F6F789FCD4F834020023BDE81040BA
:10FC700003222021FEF7E4BBD00200208AE5010820
:10FC8000F0B51F461446C7B005460E46F1220021C6
:10FC900009A808F05FFD09AA1021384602F0ECFF20
:10FCA000204609F077FD07461022002101A808F040
:10FCB00051FD102F3A46214628BF102201A808F016
:10FCC00021FD09AA05A901A803F050F832462846EB
:10FCD00005A908F017FD47B0F0BD000037B50E4C80
:10FCE0000E4D94F82F30022B12D194F821300120C0
:10FCF00094F8F321D4F8F4110093082302F06CFF78
:10FD00006B6B00209847042384F82D3003B030BD7E
:10FD1000EB6A98470123F7E7D00200201CCC0108CA
:10FD2000044B5A7F22B993F8330080F001007047EA
:10FD300000207047D0020020F0B570279DB0054626
:10FD40000E463A460021684608F004FD0821334675
:10FD50000DEB010004AC0B4AFFF792FF334620463F
:10FD60001021094A08AEFFF78BFF94E80F0086E8E0
:10FD70000F003A466946284608F0C4FC28461DB0E4
:10FD8000F0BD00BF8CD4010894D4010808B5054823
:10FD9000FAF77EF9044A92F8F831013382F8F83123
:10FDA00008BD00BF9BD40108D00200200022024BF6
:10FDB00083F8F821704700BFD002002084B070B5EE
:10FDC0008AB00EAC84E80F00724C4FF410722546D6
:10FDD000002120460EAE08F0BDFC0FCE0FC596E800
:10FDE000030014AB85E803000FCB04F1180585E888
:10FDF0000F000E9B0BB9684B23600F9B0BB9664B32
:10FE00002360109B23B94FF4C3716448F6F7B4FB29
:10FE1000129B23B94FF4C5716048F6F7ADFB119BF7
:10FE200023B94FF4C7715D48F6F7A6FB139B23B9BE
:10FE30004FF4C9715948F6F79FFBA3690BB9032327
:10FE4000A36101F0D3FE94F8203013B9012384F8A4
:10FE5000203001F0C3FE94F8213013B90E2384F84A
:10FE60002130636A0BB94E4B636201F0ABFEFAF7C7
:10FE700045FCC4F830020138033008D949486368AA
:10FE8000984700200AB0BDE8704004B070470022D7
:10FE900004210120FCF776FC0322C4F83C02002177
:10FEA0000120FCF76FFCC4F8380220B940F2BB1106
:10FEB0003A48F6F761FB002204210120FCF762FCBE
:10FEC000C4F83C0120B940F2BF113448F6F754FBA6
:10FED000002204210120FCF755FCC4F8400120B9A0
:10FEE0004FF4E1712D48F6F747FB4FF48163A4F816
:10FEF0000032002384F83430012384F80432FFF701
:10FF000035FB05AD70B9A368226905932368079294
:10FF10000893E268636806920993009395E80F00DE
:10FF2000FFF73EFBFFF728FB84F8320001F09EFE4E
:10FF300023681D4E0793636831460893236904962E
:10FF40000693E368059306F1A00318468DE80300C5
:10FF50000393F03695E80F0002F0D8F80196A369F4
:10FF60004FF4CD720093114901231148FDF7E8FACF
:10FF7000012804D040F2E7110848F6F7FDFA002303
:10FF800003220421D4F83402FEF75AFA012084F83F
:10FF9000310077E7D002002089A000088AE5010837
:10FFA00008E6D333CFD401081404002002D5010899
:10FFB0008D04010810B50F4CD4F8343223B94FF436
:10FFC000F8710D48F6F7D8FA002303220421D4F87B
:10FFD0003402FEF735FA42F21071D4F83802FCF719
:10FFE000E3FD0023D4F838021A46BDE81040194654
:10FFF000FCF7ECBBD00200208AE5010838B50E4DB5
:020000040801F1
:10000000D5F8383223B940F201210C48F6F7B4FA9A
:100010000021D5F83802FCF7C7FD0128044608D1B5
:100020000023D5F838021A461946FCF7CFFB2046C4
:1000300038BD0020FCE700BFD00200208AE501089F
:1000400010B5FFF7DBFF68B1074C0023D4F834028A
:1000500003220821FEF7F4F9D4F83402BDE8104079
:10006000FDF712BC10BD00BFD0020020002307B571
:100070004EF65E2201934EF66023411E91428CBFE4
:1000800002461A46044B01A9D3F84001FCF7FAFCDA
:10009000019803B05DF804FBD002002070B5FFF7B3
:1000A000ADFF1A4B28B15B681948984700242046D9
:1000B00070BDD3F83C01FCF703FF04460028F5D1DE
:1000C000014602F035F906460028EFD0047001F031
:1000D0008FFC054618B9304602F07AF9E7E70D4A79
:1000E00013680133136073B91368013313606B60D5
:1000F000042328462B7001F09FFC10B9284601F01C
:1001000089FC6C68D3E71368F1E700BFD0020020D8
:100110000AD50108801A00202DE9F0418AB0044672
:10012000884615460193FFF769FF20B1002738463E
:100130000AB0BDE8F0814D4ED6F83C01FCF7C0FE98
:1001400007460028F2D1002D5DD1B8F1000FEDD1A6
:100150002046414602F0ECF804460028E6D09DF81F
:100160000530002B52D004230370FFF70FFE0F223F
:1001700006A903A80AF078FF9DF804303BB10D23CF
:10018000012202A903A88DF808300AF07BFF9DF830
:1001900006303BB10223012202A903A88DF80830E2
:1001A0000AF070FF96F82E2096F82F30934203D174
:1001B00096F83030934217D02023022A18BF00222D
:1001C0008DF8083094F8783002A90BBF43F004038F
:1001D00043F001038DF809208DF8092003A80222BD
:1001E00084F878300AF04EFF96F81432059996F8A4
:1001F000F0011944C9B201F0B9FE804509D9204681
:1002000002F0E6F893E7E02D90D8A1E7022303700F
:10021000ADE7059A32B120460399D2B200F086FFCD
:100220000028ECD06577204601F0E2FB0546002867
:10023000E5D000230E4A836013680133136083B94D
:100240001368013313606B60022328462B7001F0A2
:10025000F3FB40B9284601F0DDFB73680548984779
:1002600065E71368EFE76F6861E700BFD002002021
:10027000801A002036D50108034B93F8141293F826
:10028000F00101F073BE00BFD00200200E2808BFAD
:100290000120024BD87783F8F0017047D00200208C
:1002A000024B83F8200083F8F1017047D002002050
:1002B000014B83F821007047D002002008B5F9F700
:1002C000D3FF024BC3F8480108BD00BFD002002095
:1002D000034630B5054C00F11005224618685968F0
:1002E000083303C2AB421446F7D130BD8C04002062
:1002F000034630B5054C00F11005224618685968D0
:10030000083303C2AB421446F7D130BD7C04002051
:10031000034630B5054C00F11005224618685968AF
:10032000083303C2AB421446F7D130BD6C04002041
:10033000034630B5054C00F110052246186859688F
:10034000083303C2AB421446F7D130BD9C040020F1
:1003500010B50446FFF7BCFF2046FFF7C9FF204653
:10036000BDE81040FFF7D4BF30B51025C3B0224C14
:10037000F122002105A808F0EDF92A46002101A884
:1003800008F0E8F994F85B3129468DF8053094F8C7
:100390005A3105AA8DF8063094F8593104F5B67033
:1003A0008DF8073094F858318DF8083094F85731AB
:1003B0008DF8093094F856318DF80A3094F855319B
:1003C0008DF80B3094F854318DF80C3002F054FC59
:1003D000052305AA04F5C67101A88DF8043002F0C2
:1003E000C5FC062305AA04F5BE7101A88DF80430EA
:1003F00002F0BCFC43B030BDD00200200246024BEC
:100400000068516803C370471C0400200246024B79
:100410000068516803C3704724040020034630B5C8
:10042000054C00F11005224618685968083303C2CC
:10043000AB421446F7D130BD2C040020034630B542
:10044000054C00F11005224618685968083303C2AC
:10045000AB421446F7D130BD3C040020014B9877E5
:10046000704700BFD0020020014B83F82E00704778
:10047000D002002038B5044600680D46884203D0FB
:1004800008B101F0C7FA256038BD000080B5F9F762
:1004900063FF0123754DDFF8D881764F85F82D3045
:1004A0000A234FF0FF310020714AFDF77FFF01283A
:1004B00064D1D8F80000430716D53B7833B1FAF77A
:1004C00067F80020FAF7BAF800233B70022385F89A
:1004D0002D300023D5F838021A461946FCF776F974
:1004E0000020FDF73BFCDBE710F0080621D03B784D
:1004F0007BB941F28830FAF777F818B99B215E484A
:10050000F6F73AF85D48FAF799F801233B70FFF7E0
:10051000E5FB0020FEF78AF84FF4FA61D5F83802BF
:10052000FCF742FB0028BBD1A2215348F6F724F880
:10053000B6E710F0200041D03B78E3B195F82D30BC
:10054000042B18D14E4C32462146D5F83002FCF728
:10055000D9FB01280DD12378072B2CD03246214618
:10056000D5F83002FCF78EFA012802D12046FAF7BE
:100570006BF8FFF7B3FB0020FEF758F83B78002B31
:100580008ED001F06BFA0446002889D00378012B45
:100590001AD195F82C10AA6A01B192B9B2FA82F276
:1005A00038485209F9F774FD204601F0B9FA20469F
:1005B00001F030FA74E701F0E3F9DAE7FEF736F814
:1005C0006EE701F027FAAC6A032385F82D30237813
:1005D000032B06D8012B19D88BB16B682A48984792
:1005E00009E0043B012BF8D828480021FFF742FF1F
:1005F000204600F037FE204601F00CFA03E0D62139
:100600001D48F5F7B9FFFFF769FB49E71F48214689
:10061000FFF730FFFFF784FB68B101F031FA0446C1
:1006200018B9E2211448F5F7A7FF022320462370EA
:1006300001F050FAE7E701F023FA064618B9E9217C
:100640000D48F5F799FF3146204600F001F9737E19
:1006500053B14FF47A70FDF703FB3146204600F0AA
:10066000F7F87368002BF2D03046E1E7D0020020A3
:10067000941A0020841A00208AE5010855FC00081D
:10068000881A002050D5010890D50108F8020020F2
:1006900010B50430C6B00C46FFF710FE1C4B0DF130
:1006A000050203F10C0153F8040B8B4242F8040BD2
:1006B000F9D11B881021138000238DF813300223F9
:1006C00009AA20468DF8043002F0D6FA09AA05A935
:1006D00001A802F04BFB05A8FFF72AFE012309AA97
:1006E000102120468DF8043002F0C6FA09AA05A9A7
:1006F00001A802F03BFB05A8FFF72AFE4FF4887221
:10070000044B9A83102283F8442146B010BD00BFE9
:10071000B4D50108D002002030B50430C7B00D4672
:100720001446FFF7CBFD294B0DF1050203F10C0137
:1007300053F8040B8B4242F8040BF9D11B8828466E
:10074000138000238DF813300223012509AA1021FC
:100750008DF8043002F090FA09AA05A901A802F068
:1007600005FB05A8FFF7E4FD09AA102120468DF836
:10077000045002F081FA09AA05A901A802F0F6FACC
:1007800005A8FFF7A5FD032309AA05A901A88DF86F
:10079000043002F0EBFA05A8FFF7AAFD042309AA2A
:1007A0000DEB030005A98DF8043002F0DFFA05A86F
:1007B000FFF7AEFD40F21112054B9A83112283F828
:1007C000FD5183F8442147B030BD00BFB4D50108C6
:1007D000D002002038B50D461446FFF70FFE28461C
:1007E000FFF714FE2046FFF719FE2046FFF726FE0E
:1007F0001022014B9A8338BDD002002070B50E46FE
:1008000015461C46FFF7FAFD3046FFF7FFFD284668
:10081000FFF704FE2046FFF711FE1122024B9A83D8
:10082000BDE87040FFF7A0BDD00200201023416852
:10083000064A106C884202D192F83C0020B9013B74
:1008400002F11002F5D11846704700BFD002002017
:100850002DE9F04306460C4687B019B918216748C0
:10086000F5F78AFE16B13378022B03D01A216348BC
:10087000F5F782FE33691BB91B216048F5F77CFE52
:1008800033691B78042B05D0022B03D01D215B4854
:10089000F5F772FE33785A4D63700023D5E97C87F3
:1008A0000393584A95F8F11195F8320003ABFEF71F
:1008B00039FC814620B90123237007B0BDE8F083DD
:1008C000039B33B101F0D2FB03232370039B6360CE
:1008D000F3E7B3680133012BB36011D1D5F8E421FC
:1008E00030690132C5F8E421B5F8FE2185F82C30D5
:1008F0000132A5F8FE2100F0D3F8306900F036FC93
:10090000D5F8482133695A60D5F8E4215A8195F821
:10091000F92142B1002285F8F9211A7A42F0040245
:100920001A72B5F8FA21A3F87A20484601F0C6F900
:10093000014695F8F03130694FF47A7C80F87C30CC
:1009400080F87D1095F804224FF0000902F00F02A4
:10095000012A38BF012205AB05EB0111019304AB5D
:1009600000933C3102FB0CC30CFB02F2CDF810905B
:1009700000F0DAFE00289ED0FDF71AF8F060D4F8F7
:10098000A00084F8009008B101F022FD049B0598B6
:10099000C4F8A03022463146C4F80A001A4800F0D4
:1009A0005BF88022316904F1200007F0ABFE4FF0C4
:1009B000000CC4E9048784F800C095F8333005982A
:1009C000C4F888C0C4F80A002376B26895F80232E9
:1009D000D4F8A0109A4200D261B184F819C085F809
:1009E0002CC0003918BF01210091617E0748F9F73A
:1009F0004FFB62E701206076F3E700BF8AE501085C
:100A0000D00200202D080108F8020020C3D50108FB
:100A100008B5104A10B10023A2F8FE31937FBBB194
:100A2000B2F8FE3192F800128B4211D992F80122ED
:100A30005B1A93FBF2F102FB11334BB901F0DEF8C4
:100A400030B901F0E9F818B9BDE8084001F0F4B890
:100A500008BD00BFD002002070B5D2F8A040064605
:100A6000154674B10021204601F080FBFFF79EF986
:100A70002378052B01BF012386F8D1316389A6F8BD
:100A8000D2312046FFF7C4FF2046D5F80A1000F007
:100A9000A3FB24B1237A5B0744BF01232B7270BDF3
:100AA000134B10B49A7F02B3027A42F00102027231
:100AB00093F8F011DA7F914208D193F83C40A4B149
:100AC00093F84C408CB193F85C4074B1B3F8FE419C
:100AD00093F800329C4208D9914206D0037A10BCA8
:100AE00043F002030372FFF751B910BC704700BF17
:100AF000D0020020431EDBB21F2B11D80D4A0A285A
:100B0000D35C0ED8012202FA00F010F4A46F08D0D2
:100B1000094A92F814221A440E2A02DD0020704776
:100B20000023064A107818440E28CCBF002001206C
:100B3000704700BF7FD60108D0020020A71A00200E
:100B400010B504782046FFF7D5FF78B1084A094868
:100B50001378C4540133137041B1074A92F8143228
:100B6000D118013381F8054282F8143210BD00BF5C
:100B7000A71A0020981A0020D00200202DE9F04F7B
:100B8000002593B0CDE90A129DF87090A34E059010
:100B900006934D4502D313B0BDE8F08F069B5C5D14
:100BA0005F192046FFF7A6FF019028B99C4813B0B3
:100BB000BDE8F04FF9F76CBA631E1F2B00F29C8260
:100BC000DFE813F020009A022C004C02700155015E
:100BD000BB013A024C02E2019A024E023201640267
:100BE00066029A029A029A029A029A029A029A0259
:100BF0009A029A029A029A029A029A029A029A0215
:100C00009A028702A9EB0503DBB2012B4FF0000427
:100C100000F0008186F8FD410224FBE04FF0000B5C
:100C2000A9EB0503DBB2039307235C468DF83C3048
:100C3000039A231D934202DA3B5D032B11D0BBF1D3
:100C4000000F05D09DF83C306FF300038DF83C3069
:100C50009DF83C30072B40F0CF800024DFF8C481A2
:100C6000C3E03B19D3F80180053408F00F03089363
:100C7000C8F303130493C8F30F230993C8F30313B2
:100C8000062B4FF0000AE4B2CDF8408003D908F0FB
:100C9000F003F02B35D14FF6FF71C8F3076303F073
:100CA0007003C8F30F22602B08BF0A460023079287
:100CB0005A4A02930799D8B20D920C9301F06EF83C
:100CC000DDE90C32014698B1106C88B106EB031CCB
:100CD0009CF844C004984FEA1C1E0CF00F0C84458D
:100CE00006D80298DDF810C0E64528BF08460290F5
:100CF0000133102B02F11002DCD1029B0BB14FF03B
:100D0000020A089B072B05D99DF8403003F00F031A
:100D10000F2B01D14AF0040AC8F3076808F07008E5
:100D2000B8F1600F0AD14AF0010AB8F1000F0ED0F5
:100D3000019BB8F1600F18BF9B4608E0B8F1000FA7
:100D400040F0DC81099801F007F80028EBD19DF80C
:100D50003C300AF0070A23F0070343EA0A0A8DF839
:100D60003CA065E73B19D3F801A09DF83C30053461
:100D700003F00703072BCDF840A0E4B235D19DF86E
:100D80004030C3F3031186F8F0110AF00F010F2968
:100D90004FEA131205D000293ED003F00F0386F866
:100DA000F1319DF84310CAF30F20C1F3021100F096
:100DB000FBFF20B940F275114046F5F7DDFB96F8D0
:100DC0004431102B09D11AF0706F01BF01229DF838
:100DD000433062F303038DF843309DF843301A0724
:100DE00003D0C3F3030386F80232039A231D9A4209
:100DF00002DD3B5D032BB5D054B10323002110A8C5
:100E00008DF84030FFF79CFE00210FA8FFF798FEF9
:100E100001F02CF92C443FE00123C0E7D002002070
:100E200000D601088AE50108A9EB0503DBB2052B12
:100E300040F26081781CF9F71EFA002397F905202B
:100E40009A42ACBFAF4AB04A801843F1000296F80C
:100E5000043218180B9B42F10002022B02D1013020
:100E600042F10002059BC3E91C020624D2E70623D7
:100E700000210FA88DF83C30FFF762FE0A9B00218D
:100E800003F01F03A1488DF84030FFF759FE002101
:100E900010A8FFF755FE6C1CE4B2A5423FF47BAEF0
:100EA000254676E6A9EB0503DBB2042B4FF00002E2
:100EB00040F22081D7F801308DF83820C3F30211B9
:100EC000DAB210930B4605299FBF9DF8383086F89B
:100ED000F21143F004038DF83830C2F3030302F03B
:100EE0000F02062A9CBF86F8F3319DF838300DF1C9
:100EF00041009CBF43F002038DF838306427F9F7B6
:100F0000BCF947433846FEF7F5F99DF8383088B10B
:100F1000C6F8F47143F001038DF8383005230FA8AB
:100F200001218DF83C30FFF70BFE01210EA8FFF7E1
:100F300007FE6FE760F30003EEE7A9EB0503DBB202
:100F4000052B40F2D780D7F801007B7910900DF186
:100F500041008DF8443000F0A7FE9DF84420014682
:100F60009DF8400000F0BEFE8DF8380001F07EF8DC
:100F700007230FA800218DF83C30FFF7E1FD002189
:100F80000EA8FFF7DDFD70E7A9EB0503DBB2042B2C
:100F90004FF000047FF63EAFD7F801300DF141006D
:100FA00010938DF8384000F07FFE044602469DF80D
:100FB00040105748F9F76CF82046FEF79BF928B126
:100FC0009DF8383043F001038DF838309DF84030FB
:100FD0000F2B2FD80133DAB206EB031393F82C1042
:100FE00006EB02122C3239B11B6B2BB19DF8383055
:100FF00043F002038DF838309DF83830012103F0BA
:101000000303032B4FF00A0308BFD4600FA88DF829
:101010003C30FFF795FD01210EA8FFF791FD9DF8EB
:1010200038103C48C1F3400201F00101F9F730F8F3
:101030000524EFE60022DFE7A9EB0503DBB2012B75
:1010400058D07B78012103F00F0386F8043208237F
:101050008DF8403010A8FFF773FDDDE5AC1C1BE7F1
:10106000A9EB0503DBB2012B44D001237A781109E7
:1010700002F00F0203FA01F1934086F801320C23CB
:1010800086F800128DF840300021E3E7EC1C03E7FE
:10109000A9EB0503DBB2012B2CD0B3687C78984711
:1010A000012223090A3302FA03F3C6F820320F2380
:1010B000C6E9860104F00F04002110A8C6F82442F6
:1010C0008DF83C208DF84030FFF73AFD00210FA845
:1010D000C1E7A9EB0503DBB2012B0BD07B780BB189
:1010E000022B07D196F830209A423FF495AD86F84E
:1010F000303091E500248DE62C46CEE6DDF804B0D4
:1011000025E600BF6E3DD5126F3DD512D3040020F9
:1011100037D6010856D6010838B10078032803D025
:10112000431F58425841704701207047037A70B5F9
:1011300004460C301E0900EB131002EB13130F2BA7
:10114000154609DC07F0DEFA0120237A05EB1315BA
:1011500065F30713237270BDC6F10F0207F0D2FAD0
:10116000237A002043F0F0032372F4E773B5134EA3
:1011700004463278124DC2B11249FFF7D7FF0F2251
:101180000021104807F0E6FA0023337095F8FD318E
:101190004BB101230222204601A98DF804308DF8BD
:1011A0000530FFF7C3FF02B070BD95F81422002A86
:1011B000ECD005F20521FFF7B9FFE7E7A71A0020F9
:1011C000D0020020981A0020024B00F00F0083F894
:1011D00004027047D0020020F0B585B004460391A8
:1011E00010B3FFF799FFF8B10020144B9DF90E10D2
:1011F00083F8050283F81402207A93F81EC09DF844
:101200000F20677F257F0609BCF1000F05D010F085
:10121000010018BF012083F8FC013EB1009604F1E3
:101220000C032046FFF7AAFC05B0F0BD002FFBD150
:10123000002DF9D00095A36EF3E700BFD002002087
:1012400003234168064A106C884202D192F83C00A0
:1012500020B9013B02F11002F5D11846704700BFDA
:10126000D00200202DE9F047054686B018B103787A
:10127000043B012B03D91B21B548F5F77DF92B69F8
:101280000BB11B781BB11C21B148F5F775F9B14CB6
:1012900094F8F161D4E97C8700F0A0FC00F0A6FC92
:1012A000002331460393AC4A94F8320003ABFDF7B8
:1012B00039FF28B9284600F033FC06B0BDE8F087B6
:1012C00000F0FCFC04EB0019039809F13C0998B10B
:1012D00000F0CCFE00F0D4FB044618B938219C483D
:1012E000F5F74AF92B782046637003232370039B9C
:1012F000636000F0EFFBE0E7AB680133AB60227F97
:10130000102A3AD1012B0AD1D4F8E4314FF6FF71FB
:101310000133C4F8E431F9F707F8A4F8DC01B4F8B4
:10132000DC310133A4F8DC3100262A69B4F8DC3161
:1013300004969382894B03CBD06011612A69103BDC
:1013400003CB05AB9160506094F8F3A184F8F3618E
:10135000019304AB009341F2883241F27073494625
:10136000286900F0E1F9B0B9284600F0D9FB0498EB
:1013700001F02EF884F8F3A19FE7112A06D16369E2
:1013800004F5A6709847A4F8DC01CDE74B2170481E
:10139000F5F7F2F8C8E7049B84F8F3A113B11A78C3
:1013A000012A06D0284600F0BBFB049801F010F893
:1013B00083E7227F102A00F09480112A40F08D806C
:1013C00093F82230049AD16802F15306C4F8481108
:1013D00002F1630E002B00F08680112384F8443163
:1013E0003346DFF87C91CC46186859680833ACE87E
:1013F00003007345E146F6D1DFF868E102F123030B
:1014000002F13309F446186859680833ACE8030060
:101410004B45E646F6D1DFF850E102F14309F446C8
:10142000186859680833ACE803004B45E646F6D126
:10143000DFF838E1F446186859680833ACE803006F
:10144000B342E646F6D19368A363137CC3F3030368
:1014500084F8F331137CC3F3021384F8F231507C27
:10146000FFF7B2FE002394F82E20049812F0FD0F2F
:1014700000F1120018BF84F82E30C4E97A33C4F8A2
:10148000E43184F82F3084F8303000F0CDFC00F0E7
:10149000EDFD012384F8333000F0F2FA064618B966
:1014A000CB212B48F5F768F88022296906F1200046
:1014B00007F028F90023049A0598C6F8A02094F8AC
:1014C0003320C6E90487C6F80A00C6F888303276A9
:1014D00033702B78304673700BE77D211C48F5F78D
:1014E0004BF833466EE7102384F844313346DFF877
:1014F00070C0664618685968083303C67345B44619
:10150000F7D102F123063346DFF8589002F1330E8B
:10151000CC46306871680836ACE803007645E14691
:10152000F6D11E46DFF84090CC4630687168083628
:10153000ACE803007645E146F6D1DFF830C06646F8
:1015400018685968083303C67345B446F7D17AE77B
:101550008AE50108D002002041120108240400207D
:101560009C0400208C0400207C0400206C040020DB
:101570002DE9F04385B006460C468DF80F202BB1BF
:10158000012200200DF10F01F9F73CFCFCF710FAE5
:101590001E4B1F4DDFF87C809DF80F109B6A07469D
:1015A0002046984741F288322946D8F83002FBF7A6
:1015B00069FA044600B32B78012B21D12846AC6888
:1015C000F9F742F84FF47A70A4EB070909FB000021
:1015D00006F03EFA7168024698F83200FDF756FEB2
:1015E00000F044FD3B46CDE90049D8F80050726850
:1015F0009DF80F100848A847204605B0BDE8F083C5
:101600002846F9F721F80024F6E700BF1CCC0108B2
:10161000B41A0020D00200209FD601082DE9F84F0F
:10162000DFF8E8B01E46DBF834300546894614463C
:1016300040F6B8379847DFF8D8A0DFF8D8804FF4E5
:101640007A7307FB05F23249B2FBF3F2D8F83002A5
:10165000FBF718FA28B9DBF8303098474FF0FF3025
:101660002DE09AF80030072B07D15046F8F7ECFF31
:101670004FF47A65F9F754FBE1E7032BDBF83070A0
:101680001FD1DAF8045028792968844228BF04461B
:101690004846224607F036F8D8F8008095F9083019
:1016A000B5F90620A9881C48C0471EB1EB883380D5
:1016B0002B7AB3701648F8F7C7FFB8472046BDE845
:1016C000F88F042B0CD11248F8F7BEFFB847D8F8B2
:1016D0000040FCF76DF901461048A0470020EEE7F6
:1016E000052B0AD10A48F8F7AFFFB847D8F80040F1
:1016F000FCF75EF901460A48EFE7F1210948F4F7E3
:101700003BFF0348F8F7A0FFB847A7E71CCC010848
:10171000A81A0020D0020020D2D60108FCD6010869
:1017200014D701088AE501082DE9F04F8E4CC9B0A5
:101730000E4691469846FF2294F8443108A9539FDB
:10174000029000F05DFE824618B9002049B0BDE865
:10175000F08F94F8F01194F8F25172688D4298BFAE
:101760004D1B08468CBF0025EDB2D4F800B00592A1
:10177000049100F0A9FB039094F8F10100F0BAFB8A
:10178000DDE90412039B00907848D847F2682846A8
:10179000D4F800B0039200F097FB29460346039A61
:1017A0007348D84794F8F311D4F8F4210846D4F8D4
:1017B00000B00492039100F087FBDDE903120346B9
:1017C0006C48D8474246236849466B4898470121F0
:1017D000029800F0CBFC94F821300020009394F89C
:1017E000F13194F8F021716801F0F6F952460023C6
:1017F000304608A9FFF7BCFE82460028A5D0029B10
:10180000594C93F8783013F0050F09D013F0040306
:1018100018BF022394F82F209A4218BF84F82F3063
:10182000FF22002108A806F095FF94F821302A46EF
:101830000093F1680823012001F0CEF9A9F114000A
:1018400005F0CCFC44A3D3E9002305F041FD05F0ED
:10185000D9FF054609F2AB2005F0C0FC40A3D3E94F
:10186000002305F035FD05F0CDFF8146A8F11400F9
:1018700005F0B4FC38A3D3E9002305F029FD05F0F9
:10188000C1FFA0F114034B4594BFC5EB030BC5EB9F
:10189000090B4FF47A7909FB05F10646B1FBF9F122
:1018A00007A8CDF81CA0FCF79BF9FF223B46584641
:1018B00008A9FFF7B3FE421C05463FF446AF0028D7
:1018C0001ADD2468FCF774F85346024629462B4873
:1018D000A0470FB10123FB700023529A9D42136071
:1018E00008DD214BE9B293F8442108A801F008F97A
:1018F000529B1860012029E794F8213001200093C1
:1019000094F8F3210823D4F8F41101F065F909FBE8
:1019100006F107A8B1FBF9F1CDF81CA0FCF760F9BE
:1019200008F2AB2005F05AFC0DA3D3E9002305F023
:10193000CFFC05F067FF3B46FF2208A9801BFFF79D
:101940006DFE431C05463FF400AF0028C4DD002FA8
:10195000C2D00223BFE700BF0AD7A3703D0AEF3F02
:10196000A4703D0AD7A3F03FD00200202AD7010877
:101970005CD7010882D70108A8D70108C3D701089E
:1019800030B5C3B06B46FF224FF47A6002A9FFF76F
:1019900045FE041E24DD0023144D0193D5F8482193
:1019A00095F84431E1B202A800F06CFE03460190C4
:1019B000B0B10278052A01D0032A14D118460021BB
:1019C00000F0D4FB0198FFF723F8DDE90010FFF7E2
:1019D00003FC00230122D5F83C0201A9FAF7F6FE28
:1019E000204643B030BD00F0F3FCF9E7D002002000
:1019F00038B5074B0546DB6814209847044620B1EC
:101A00001422002106F0A6FE2561204638BD00BF45
:101A1000D002002010B5044650B1006900F0D8FC97
:101A200000232361034B2046BDE810401B69184783
:101A300010BD00BFD0020020002307B5019006486A
:101A40001A4601A9D0F83C01FAF7C0FE431E5842DD
:101A5000584103B05DF804FBD0020020002307B515
:101A60000193064B93F8342022B9D3F83C0101A925
:101A7000FBF708F8019803B05DF804FBD0020020E2
:101A8000064B10B5A820DB689847044618B1A82279
:101A9000002106F05FFE204610BD00BFD0020020EE
:101AA00010B5044698B1D0F8883013B1203000F05A
:101AB00079FCD4F8A00020B100F08AFC0023C4F81F
:101AC000A030034B2046BDE810401B69184710BDED
:101AD000D00200201FB5104C0190D4F84001FBF754
:101AE00001FA024640B9D4F8400103A9FAF7CAFF47
:101AF00010B10398FFF7D4FF0023D4F840011A4631
:101B000001A9FAF763FE20B94FF4BA710348F4F75C
:101B100033FD04B010BD00BFD00200208AE50108EB
:101B200038B50546FFF7ACFF044620B940F27911FD
:101B30000548F4F721FD012323702B7820466370BC
:101B4000BDE83840FFF7C6BF8AE5010810B50D4C67
:101B5000031D04EB031319719A600123013004EB98
:101B60000010026380F82C30114694F83200FDF723
:101B7000C9FB28B9BDE810400B210348F4F7FCBCB1
:101B800010BD00BFD00200208AE501080C4B0146C1
:101B900070B4102000221D4693F83C401CB11E6C0E
:101BA0008E4208BF2246013803F11003F4D122B956
:101BB00095F8320070BCFDF751BC70BC704700BF97
:101BC000D0020020044B93F8222083F8F3215A6AB4
:101BD000C3F8F421704700BFD0020020024B93F8F5
:101BE000202083F8F1217047D0020020024BDA7FD9
:101BF00083F8F021704700BFD0020020054B93F816
